:020000041000EA
:1000000000B5324B212058609868022188439860DF
:10001000D860186158612E4B002199600221596106
:100020000121F02299502B49196001219960352056
:1000300000F044F80222904214D00621196600F024
:1000400034F8196E01211966002018661A6600F04E
:100050002CF8196E196E196E052000F02FF8012189
:100060000842F9D1002199601B49196000215960AB
:100070001A491B48016001219960EB211966A021F2
:10008000196600F012F800219960164914480160C1
:100090000121996001BC002800D000471248134993
:1000A000086003C880F30888084703B5996A0420EC
:1000B0000142FBD001200142F8D103BD02B5186610
:1000C0001866FFF7F2FF186E186E02BD00000240BE
:1000D000000000180000070000035F00212200005C
:1000E000F4000018222000A00001001008ED00E03C
:1000F00000000000000000000000000074B24E7A12
:1001000000200420F7010010C3010010C5010010F9
:10011000C1010010C1010010C1010010C101001097
:10012000C1010010C1010010C1010010C701001081
:10013000C1010010C1010010C9010010CB01001065
:10014000CD010010CD010010CD010010CD01001037
:10015000CD010010CD010010CD010010CD01001027
:10016000CD010010CD010010CD010010CD01001017
:10017000CD010010CD010010CD010010CD01001007
:10018000CD010010CD010010CD010010CD010010F7
:10019000CD010010CD010010CD010010CD010010E7
:1001A000CD010010CD010010CD010010CD010010D7
:1001B000CD010010CD010010CD010010CD010010C7
:1001C00000BE00BE00BE00BE00BE00BEEFF3058054
:1001D000103800BEF2EB8871D0850010F885001051
:1001E0003402001090A31AE700201F49086006C8D7
:1001F00081F3088810471D48006800282FD10DA4FE
:100200000ECC002902D000F012F8F9E71849194A7B
:10021000002000E001C19142FCD1174988471749ED
:1002200088471749884700BEFDE701C901C29A42C5
:10023000FBD37047F8850010C0000020B4E2002016
:10024000EC6701100000042000000420EC6701109E
:10025000001004200010042000000000704709482E
:1002600005F05EFB0047000008ED00E0000000D054
:10027000B8E20020209702201D410010CD0300109D
:10028000654200105756000006005250ABB3605351
:100290001485001006005250861C030224850010AD
:1002A000060052505422A29D3C8500100500525079
:1002B000DE65F468EC670110F8B5C0460448054BEC
:1002C00010B5834203D0044B002B00D0984710BDDB
:1002D000B4E20020B4E20020000000000648074914
:1002E000091A8B10C90FC91810B5491003D0044B57
:1002F000002B00D0984710BDB4E20020B4E20020EB
:100300000000000010B5074C2378002B09D1FFF73F
:10031000D5FF054B002B02D0044800E000BF0123AD
:10032000237010BDE8E5002000000000F871001007
:10033000054B10B5002B03D00449054800E000BF71
:10034000FFF7CCFF10BDC04600000000ECE5002028
:10035000F871001010B500F037FC012010BDC04648
:1003600010B50B0707D503000A3B012B18D90C3831
:10037000012826D910BD4907FCD50C281BD008D868
:100380000A2812D00B28F5D10121012000F030FC01
:10039000F0E70D28EED10121022000F029FCE9E769
:1003A0000021012000F024FCE4E701210120494262
:1003B00000F01EFCDEE701210220494200F018FC9B
:1003C000D8E70021022000F013FCD3E710B58AB073
:1003D00006F044FC0221012002F060F80221002016
:1003E00002F05CF8D02380221B0612025A622648D3
:1003F00006F036FB254806F033FB254806F030FBB7
:10040000012100220E2002F061F800F0DFFB02F073
:10041000C5FD04AB0293002301931E4B1E4A0093BB
:10042000002302F083FE002201210A2002F04EF890
:10043000002201210B2002F049F8002201210C20AA
:1004400002F044F8002201210D2002F03FF8134C85
:10045000012223000C210A2002F04AF82300012285
:100460000C210B2002F044F8230001220C210C2067
:1004700002F03EF8230001220C210D2002F038F892
:1004800000F0B2FBFCE7C046F871001010720010DB
:100490003C7200105503001010270000610300108B
:1004A000074B10B51C68074B1B689847064B20612B
:1004B0001A681F231A401E3B9340044A136010BD64
:1004C000489602204C9602209801002080E200E02D
:1004D000F0B5DE46454657464E46E0B58DB0039230
:1004E000934A040010609346924A88461360924BE8
:1004F000984200D10BE1914B9A46052003F09CFDF8
:1005000005F038FD8E4A8F4B05F0B1FC00228E4B72
:1005100005F0ADFC05F07AFD8146052003F08CFD69
:1005200005F028FD894A8A4B05F0BFFC05F06EFDF9
:10053000FE2102908905484606F004F9002800D003
:10054000EBE0484606F032F906000F0032003B00AF
:10055000804806F077FB029806F028F902000B00AD
:100560007D4806F06FFB7D49200006F06DFC7C495C
:100570000600200006F068FC002380220793F82381
:1005800052025B0204920593C02307001B03102252
:1005900004A908A8069306F081F93B1DFA011B0384
:1005A000134308A9102204A8099306F077F94346DB
:1005B0006C4A5B011340424613438222D204134328
:1005C0004846079306F0ECF885B20020002D0ED0C7
:1005D000280006F0BDF8011C484606F06AF887219D
:1005E000C90506F080F806F0DBF8C0B200025E4BE9
:1005F0002D04E3185A1E9341054304959D1D404662
:10060000290001F04BFF0123424600212000009306
:10061000994606F091FC8023069A9B021343002121
:100620003A002000069304AB06F0DAFC4F4B504A28
:100630002361D823E2504F4AE2504F4AE2504A46E3
:1006400023681343236033001833F2011B03134361
:100650004A4A13400993C0231B030A93039B9A023F
:1006600080239B0513430B93029B181C984606F0AE
:1006700097F887B20020002F0ED0380006F068F8F7
:10068000011C404606F015F88721C90506F02BF835
:1006900006F086F8C0B200022900039D3F0407431C
:1006A0002800089701F0FAFE01232A002000009399
:1006B000012106F041FC3200200008AB012106F0C8
:1006C0008FFC20232A4AFF3363612F3BE250022232
:1006D00023680121134323605346186801F0C4FFC7
:1006E00053462749186801F0D9FF5346002118687E
:1006F00002F0DAF95B461A689C2310215B00D150A6
:100700000DB0F0BCBB46B246A946A046F0BD0B4BAF
:100710009A460A2352461360EFE6484606F046F82A
:1007200006000B00320017480F0006F08BFA0DE7A9
:10073000489602204C96022000003050980100207C
:10074000D9899DD8892B6C41000018408DEDB5A04A
:10075000F7C6C03E9C720010B0720010D872001034
:10076000C4720010E0FF0FFC0000E0AFFF020000C9
:10077000A080000027A0000060600000FFFFFF9F36
:10078000A10400106072001070B5214C214920684E
:10079000214E0B684200121835689B0052019B18CD
:1007A00058590B6801330B600B68182B07D01B4B93
:1007B0005B68DB0102D50122194B1A7070BD002263
:1007C0000A602368023323602168164B994214D0D3
:1007D000902322689B009A42E9D101232360124BA7
:1007E0001B78002B0ED0114B1A78002A02D0012161
:1007F0000F4A117001221A70D9E70B4B22601B7847
:10080000002BF0D10B4B1A681D603260EBE7C0463D
:100810004096022044960220A001002000002050B3
:1008200019970220410200001A9702201E97022009
:100830001B9702209C010020F0B54546DE46574636
:100840004E46E0B58BB08046059008000F21404D24
:10085000194014001B098A0052182D685900C91844
:10086000AC4652008900002C6AD01D01EB1A00250D
:100870000F002E00DB0199460C374B1C9F426E4146
:100880000B2377423B4001335B189900CB185B0187
:100890009B18A0440493434691440693531C0A3288
:1008A0009A426D416B42079307232A499B461833AE
:1008B0004E469A4605008946069B6F0098460923D6
:1008C0007F19FF003900079A6746134001339B19CF
:1008D000039309954B4635008C46059A0896584671
:1008E000E908595C284001410120884399461600D7
:1008F00003000195029252461800002532409040B4
:10090000720962449200BA181168013501431160FE
:100910006032A542F8D101364645ECD1B046019D82
:10092000029A039901354B46A04412198D42D6D143
:10093000089E099D049BA036BC462D19B342BBD12D
:100940000BB0F0BCBB46B246A946A046F0BDC046BF
:100950009C0100203C73001070B5D825124B2D026D
:100960002A0004000021186805F092FF0F4B2A00AE
:100970000021186805F08CFF002301210C4A0D4866
:1009800013700D4A13700D4A13700D4A13700D4AFF
:1009900014600D4A11600D4A0131136003220C4BA3
:1009A000FFF796FD70BDC046A00100209C0100200D
:1009B00019970220000020501A9702201E9702204B
:1009C0001B9702209896022040960220449602200F
:1009D00089070010124B70B51A78002A1AD1114BF2
:1009E0001A78002A01D000221A700F4D2B78002BA4
:1009F0000FD00123D8220D4C002123700C4B120282
:100A0000186805F045FF0B4B1B68984700232370BF
:100A10002B7070BD002208481A7006F021F8DEE73E
:100A2000199702201B9702201E9702201A97022076
:100A30009C0100209896022014730010F0B54546E2
:100A4000DE4657464E46E0B587B001901000109A3A
:100A500002919046274A1278002A43D0002B41D0B9
:100A6000254A146800283DD00722914602004946D5
:100A70008A4308320392012293461E320025924691
:100A800004900593029B039A59196A43049B4E00F4
:100A90009C46019B76189F1AF60031003B00944457
:100AA000664647468C46984600954D46D008385CC9
:100AB000154028415D464346854328005546991810
:100AC0004B0929408840010063449B0018590132BA
:100AD000014319519642E8D1009D059B0135B84666
:100AE0009D42CFD107B0F0BCBB46B246A946A04656
:100AF000F0BDC0461A9702209C010020F8B5474679
:100B0000CE4680B50F002E49150008AA1C000978B2
:100B100008CA06001278002908D0012A0AD0022A41
:100B200034D0002A1FD0274805F09AFFC0BCB94630
:100B3000B046F8BD002BF9D09A00D2189846520161
:100B40009146A0444A461009684323782A00390098
:100B5000301AFFF771FEA0235B429C460134E1444A
:100B6000A045EFD1E2E7002BE0D0AA005219984649
:100B700052009146A044300023782A003900013405
:100B8000FFF75AFE4E444445F5D1CFE7002BCDD0B8
:100B9000290059438A00521852015209861AAA00A4
:100BA0005219984652009146A044300023782A00FA
:100BB00039000134FFF740FE4E44A045F5D1B5E7BA
:100BC0001A970220247300107047C046002210B507
:100BD000034B04481A60FFF7BFFE06F04DFA10BD44
:100BE000C4960220E11C001010B5FFF7F3FE10BD03
:100BF00010B5012823D0022800D010BD114B1A686F
:100C0000012AFAD00029F8D101241C600E4B0F4AAA
:100C10001B680C331360FA220D4B52001A6006F069
:100C20002BFA1422F0210B4B490018600A4B0F20BD
:100C30001A600A4B0A4A1C7001F0DEFADDE7094B24
:100C40001960DAE7C4960220C0960220B49602200A
:100C5000B8960220A4960220A80100201D97022029
:100C60004C1D0000BC9602201E23F0B5DE469B46BC
:100C70003E3357469A463E334E4699463E334546A6
:100C800098467C339C4684446346E0B587B0039322
:100C9000C9235B009C46A84C070084442600634699
:100CA000143117370D00A0368344824481448044B8
:100CB000FF370593C30700D597E0D130FF3004908C
:100CC00030E0022B00D12FE16368012B38D0022BDA
:100CD00000D127E1A368012B3DD0022B00D11FE1F9
:100CE000E368012B42D0022B00D113E12369012BD1
:100CF00047D0022B00D10BE16369012B4CD0022BB2
:100D000000D103E1A369012B51D0022B00D1FBE0FC
:100D1000E369012B56D0022B00D109E120342135A3
:100D2000B4425BD02368012BCBD1844B00932222A9
:100D3000192329005846FFF781FE6368012BC6D1AD
:100D40007E4B00932222192329005046FFF776FE9E
:100D5000A368012BC1D1794B0093222219232900CA
:100D60004846FFF76BFEE368012BBCD1734B009341
:100D70002222192329004046FFF760FE2369012B38
:100D8000B7D16E4B00932222192329003800FFF7B8
:100D900055FE6369012BB2D1684B009322221923BF
:100DA00029000398FFF74AFEA369012BADD1634BDD
:100DB00000932222192329000598FFF73FFEE369DB
:100DC000012BA8D15D4B29000093222219230498FE
:100DD0002034FFF733FE2135B442A3D107B0F0BC75
:100DE000BB46B246A946A046F0BDD130FF300490C4
:100DF00029E0022B00D181E06368012B31D0022B66
:100E00007AD0A368012B37D0022B7BD0E368012B6B
:100E10003DD0022B74D02369012B43D0022B7DD00F
:100E20006369012B49D0022B76D0A369012B4FD0E7
:100E3000022B7BD0E369012B55D0022B7AD02034D2
:100E40002135A642CAD02368012BD2D13C4B009356
:100E50002222192329005846FFF7F0FD6368012B71
:100E6000CDD1374B00932222192329005046FFF79A
:100E7000E5FDA368012BC7D1314B00932222192332
:100E800029004846FFF7DAFDE368012BC1D12C4B5E
:100E900000932222192329004046FFF7CFFD236942
:100EA000012BBBD1264B00932222192329003800A5
:100EB000FFF7C4FD6369012BB5D1214B00932222BA
:100EC000192329000398FFF7B9FDA369012BAFD1BE
:100ED0001B4B00932222192329000598FFF7AEFD32
:100EE000E369012BA9D1164B009322221923290073
:100EF0000498FFF7A3FDA2E7124BB3E7114BA6E757
:100F0000104BC5E70F4BB8E70F4B51E70E4B44E7CB
:100F10000D4B37E70C4B2AE70A4BCFE7094BC2E7EB
:100F2000094B19E7084B0CE7074BFFE6054BD0E7E9
:100F3000054B48E7034BD7E798030020F005002056
:100F40007005002070040020F0040020F0B5574622
:100F50004E464546DE46614BE0B51C68604B85B0A9
:100F60001E681E239A463E3399463E3398463E33CA
:100F70009C467C339B46B3445B460093C9235B008D
:100F80009B46B3445B460193E8235B009B463700D6
:100F9000B3445B4600251737FF37524A2D34B2441D
:100FA000B144B044B444039302972300193B9942DF
:100FB00059DB1368002B06D0824504DC4027BB4672
:100FC000B344584569DB5368002B06D0484504DB21
:100FD0007E27BB46B34458455ADB9368002B06D0A6
:100FE000404504DBBC27BB46B34458455FDBD368B0
:100FF000002B06D0604504DBFA27BB46B3445845B6
:1010000050DB1369002B08D0029FB84205DB9C27F8
:101010007F00BB46B34458454EDB5369002B08D0D4
:10102000009FB84205DBBB277F00BB46B344584551
:1010300047DB9369002B08D0019FB84205DBDA2714
:101040007F00BB46B344584540DBD369002B0AD030
:10105000039FB84207DBF9277F00BB46B3448345B3
:1010600001DDA14237DB013520322134052D9CD131
:1010700000210025002200231B480160456082609A
:10108000C36005B0F0BCBB46B246A946A046F0BD61
:10109000A142A2DA01210122EEE7A14293DA012165
:1010A0000022E9E7A142ACDA01210322E4E7A142F0
:1010B0009DDA01210222DFE7A142AEDA01210422FA
:1010C000DAE7A142B5DA01210522D5E7A142BCDA6F
:1010D00001210622D0E701210722CDE7AC01002043
:1010E0002CE6002098030020E0960220F0B5DE46B2
:1010F00057464E464546E0B5D5B005F0BDFFD44C49
:1011000023681433984200D935E3D24BD24E994626
:10111000D24D2B68002B00D0EDE1D14B1C68002C88
:1011200004D0002000210124049005915A68002A6F
:1011300007D000200121E20004AFBA18106051600E
:1011400001349A68002A07D000200221E20004AF8F
:10115000BA18106051600134DA68002A07D0002004
:101160000321E20004AFBA181060516001341A691B
:10117000002A07D000200421E20004AFBA18106052
:10118000516001345A69002A07D000200521E2008D
:1011900004AFBA181060516001349A69002A07D070
:1011A00000200621E20004AFBA181060516001343B
:1011B000DA69002A07D000200721E20004AFBA183C
:1011C0001060516001341A6A002A07D00120002102
:1011D000E20004AFBA181060516001345A6A002A64
:1011E00007D001200121E20004AFBA18106051605D
:1011F00001349A6A002A07D001200221E20004AFDC
:10120000BA18106051600134DA6A002A07D0012050
:101210000321E20004AFBA181060516001341A6B68
:10122000002A07D001200421E20004AFBA181060A0
:10123000516001345A6B002A07D001200521E200D9
:1012400004AFBA181060516001349A6B002A07D0BD
:1012500001200621E20004AFBA1810605160013489
:10126000DA6B002A07D001200721E20004AFBA1888
:101270001060516001341A6C002A07D0022000214E
:10128000E20004AFBA181060516001345A6C002AB1
:1012900007D002200121E20004AFBA1810605160AB
:1012A00001349A6C002A07D002200221E20004AF28
:1012B000BA18106051600134DA6C002A07D002209D
:1012C0000321E20004AFBA181060516001341A6DB6
:1012D000002A07D002200421E20004AFBA181060EF
:1012E000516001345A6D002A07D002200521E20026
:1012F00004AFBA181060516001349A6D002A07D00B
:1013000002200621E20004AFBA18106051600134D7
:10131000DA6D002A07D002200721E20004AFBA18D4
:101320001060516001341A6E002A07D0032000219A
:10133000E20004AFBA181060516001345A6E002AFE
:1013400007D003200121E20004AFBA1810605160F9
:1013500001349A6E002A07D003200221E20004AF74
:10136000BA18106051600134DA6E002A07D00320E9
:101370000321E20004AFBA181060516001341A6F03
:10138000002A07D003200421E20004AFBA1810603D
:10139000516001345A6F002A07D003200521E20072
:1013A00004AFBA181060516001349A6F002A07D058
:1013B00003200621E20004AFBA1810605160013426
:1013C000DA6F002A07D003200721E20004AFBA1821
:1013D00010605160013480229A58002A07D00420FE
:1013E0000021E20004AFBA18106051600134842279
:1013F0009A58002A07D004200121E20004AFBA184D
:1014000010605160013488229A58002A07D00420C5
:101410000221E20004AFBA181060516001348C223E
:101420009A58002A07D004200321E20004AFBA181A
:1014300010605160013490229A58002A12D0042082
:101440000421E20004AFBA1810605160013409E0D1
:10145000A89602202CE60020AC01002028E60020FF
:101460009803002094229A58002A00D149E10420D0
:101470000521E20004AFBA181060516098229A5812
:101480000134002A06D004200621E200BA181060B8
:10149000516001349C229B58002B06D00420072168
:1014A000E300FB18186059600134002005F04EFE7F
:1014B00005F0FAFD05F002FE210004F063FAC90010
:1014C0007B587F185A017968D21833681432D218C1
:1014D0004B015B1A494609685B00D3485B1824330B
:1014E0000360D24B02909A461A6001232B6006E0FB
:1014F000002C00D0E2E3CC4B0293CC4B9A46CC4B71
:10150000CC4C1A680393CC4B21009846180004F089
:10151000C1F9CA4BCA4F210018003A681C0004F0F8
:10152000B9F9404605F0E4FD012302222821019388
:1015300000904346A020FFF7E1FA200005F0D8FD17
:10154000002300900193E620230002222821FFF7C8
:10155000D5FABC4BBC4C186823688000C018002822
:1015600000DC05E1B9239B00984200DBB4E00300F6
:101570002360B64B98461B68012B00D1B4E0B44BF6
:101580009B46029B1B685A1D82420ADB02001732EF
:10159000934206DC53461B68E43BFF3B1C2B00D800
:1015A00041E3FA214900FFF7D1FC3B68002B00DC46
:1015B000B7E0F52332685B009A4200DDB1E00368D2
:1015C000012B00D1A9E0A34A516813685B18916808
:1015D0005B18D1685B1811695B1851695B189169D8
:1015E0005B18D1695B18116A5B18516A5B18916AC4
:1015F0005B18D16A5B18116B5B18516B5B18916BB0
:101600005B18D16B5B18116C5B18516C5B18916C9B
:101610005B18D16C5B18116D5B18516D5B18916D87
:101620005B18D16D5B18116E5B18516E5B18916E73
:101630005B18D16E5B18116F5B18516F5B18916F5F
:101640005B18D16F5B18802151585B188421515869
:101650005B18882151585B188C2151585B189021D8
:1016600051585B18942151585B18982151585B18B8
:101670009C2152589B18002B00D159E1FA21764B3E
:1016800020681822009349000C23FFF7D7F94B4636
:1016900031681868FFF7E8FA5B4619681E2963DDB0
:1016A0000839196043461B68012B00D137E12B68CC
:1016B000002B06D05346196882239B00994200DA1A
:1016C00011E1002352462B60136055B0F0BCBB46BD
:1016D000B246A946A046F0BD180023605B4B984671
:1016E0001B68012B00D04AE7594B19689B465B4B9E
:1016F0001868FFF72BFC0368012B00D1C0E02068BD
:101700003FE798229A58002A00D084E09C229B58F8
:10171000002B00D1ECE604AFC0E6C368002B00D17B
:1017200051E7DC214E4A49000F2000F065FD64209E
:1017300001F06AFEBE214A4A49000F2000F05CFD1C
:10174000642001F061FEF021454A0F2000F054FDB5
:10175000642001F059FE002264210F2000F04CFDAE
:101760000322404B1A6089E70023424613609EE73C
:1017700001230120FCE605F07FFC3B4B20601A684A
:1017800099461300DE33FF33212B18D8314B1C0050
:101790001900A034C86900281FD12031A142F9D115
:1017A00011000839FF39212900D9A8E01800A0301C
:1017B000D969002911D120338342F9D130E21300D5
:1017C000A033FF33212B00D9F8E0224B1C00190075
:1017D000A0348869002800D180E0244C244E23687E
:1017E0005B42236033681433336005F045FC0A2202
:1017F000204BE6211860204B0F201A601F4B093A3E
:101800001A70174A00F0F8FC4B461A6823689B18B8
:101810004A4613607CE404200621E20004AFBA18B3
:1018200010605160013435E610E6002014E6002017
:10183000F09602203C82001054960220509602201E
:10184000B0960220BC960220C0960220C4960220C8
:10185000B8960220980300204C040020B496022081
:1018600088130000FC9602202CE60020B001002026
:10187000AC010020A4960220A80100201D970220A0
:10188000C368002B00D13AE7002143468268196003
:1018900094464368914ADB0063449B009950C368B7
:1018A000012B00D106E2022B00D1FFE1039B1B6854
:1018B000F533FF33039A136005F0DEFB1422884BE7
:1018C0001E211860874B0F201A60874B133A1A703D
:1018D000FA22D20000F090FC206852E62031A142AA
:1018E00000D076E75CE7534604311960029B06227C
:1018F00018687E4B00931223FFF7A0F8E5E611006D
:101900004639FF39212900D9FEE01800A030996935
:10191000002900D061E720339842F8D180E1744B70
:1019200006221868714B00931223FFF787F8BEE672
:10193000DC21704A89000F2000F05EFCC82001F015
:1019400063FDF7216B4A89000F2000F055FCC82089
:1019500001F05AFD674A68490F2000F04DFCC8208D
:1019600001F052FDC421634A49000F2000F044FCFD
:10197000C82001F049FD5F4A60490F2000F03CFC9F
:101980009620400001F040FD002264210F2000F06D
:1019900033FC58495A4A8C46136801331360039A42
:1019A00013686344136096224E4B92001A60012222
:1019B0004D4B1A70534B03321A605FE63E3B212BAE
:1019C00000D847E13E3B212B00D859E11500434B9D
:1019D0002B351968002902D0212D00D8FDE614000E
:1019E00059686934002902D0212C00D8F5E610008E
:1019F0009968A730002902D0212800D8EDE611000F
:101A0000DE68E531002E02D0212900D8E5E61E6A05
:101A1000002E02D0212D00D8DFE65E6A002E02D013
:101A2000212C00D8D9E69E6A002E02D0212800D8A9
:101A3000D3E6DE6A002E02D0212900D8CDE61E6C46
:101A4000002E02D0212D00D8C7E65E6C002E02D0F9
:101A5000212C00D8C1E69E6C002E02D0212800D88F
:101A6000BBE6DE6C002E02D0212900D8B5E61E6E42
:101A7000002E02D0212D00D8AFE65E6E002E02D0DF
:101A8000212C00D8A9E69E6E002E02D0212800D875
:101A9000A3E6DE6E002E02D0212900D89DE6802626
:101AA0009E59002E02D0212D00D896E684255D593E
:101AB000002D02D0212C00D88FE688241C59002C40
:101AC00002D0212800D888E68C201858002800D1A0
:101AD00066E6212900D880E662E6C0469803002029
:101AE000A4960220A80100201D970220380400209F
:101AF000B4960220881300000F0300004B02000080
:101B0000A4010020FC9602203E39212900D8ADE036
:101B10003E39212900D8BFE06A49551819680029C3
:101B200002D0212D00D858E6674954185968002979
:101B300002D0212C00D850E6644950189968002939
:101B400002D0212800D848E66149DE685118002EED
:101B500002D0212900D840E61E6A002E02D0212D95
:101B600000D83AE65E6A002E02D0212C00D834E676
:101B70009E6A002E02D0212800D82EE6DE6A002EB2
:101B800002D0212900D828E61E6C002E02D0212D7B
:101B900000D822E65E6C002E02D0212C00D81CE674
:101BA0009E6C002E02D0212800D816E6DE6C002E96
:101BB00002D0212900D810E61E6E002E02D0212D61
:101BC00000D80AE65E6E002E02D0212C00D804E672
:101BD0009E6E002E02D0212800D8FEE5DE6E002E7B
:101BE00002D0212900D8F8E580269E59002E02D087
:101BF000212D00D8F1E584255D59002D02D0212C3E
:101C000000D8EAE588241C59002C02D0212800D8ED
:101C1000E3E58C201B58002B02D0212900D8DCE5FD
:101C20002C4C2D4EF2E50023FA222B603B681E213E
:101C3000013B92000F203B6000F0DEFA642001F0CF
:101C4000E3FB0F200022642100F0D6FA282328208D
:101C50002360A6E4214B1C001900A0344869002829
:101C600000D0BAE52031A142F8D199E51800A030A2
:101C70005969002900D0B0E520338342F8D1CFE77D
:101C8000164B1C001900A0340869002800D0A4E5F8
:101C90002031A142F8D183E51800A030196900294C
:101CA00000D09AE520339842F8D1B9E7039B1B682E
:101CB0006433FFE5039B1B68C833FBE504AFFFF704
:101CC000F4FBC04647FDFFFF85FDFFFFC3FDFFFF9F
:101CD00001FEFFFFB0010020AC01002098030020AE
:101CE000F0B5C64600B5C34FA8B03B68042B3DD83D
:101CF000C14A9B00D3589F4602250A22BE20C82114
:101D0000BE4B00924000073A0195FEF7F7FE06220F
:101D10008221BE20BA4B00924900033A400001954F
:101D2000FEF7ECFEB74BB84C1A68B849200003F038
:101D3000B1FD200005F0DCF9A0210090BE202300B9
:101D40000322490040000195FEF7D8FE1122C82168
:101D5000BE20AF4B009201950F3A49004000FEF7BC
:101D6000CDFEAC4B1B68012B00D13EE1AA4D24E116
:101D700002250E22BE20C821A84B019500924000EA
:101D80000B3AFEF7BBFE06228221BE209C4B01953A
:101D900000924900033A4000FEF7B0FE994B9A4C7E
:101DA0001A689A49200003F075FD200005F0A0F99B
:101DB000A0210090BE20230001950322490040008D
:101DC000FEF79CFE944D2B78002B00D0F8E0944A4F
:101DD0001368022B00D1FBE1032B00D1F6E1012BAC
:101DE00001D0012313608F4B19685A68169117921E
:101DF0009968DA681A911B9219695A691C911D92A7
:101E00009969DA691E911F92196A5A6A10911192A2
:101E1000996ADA6A20912192196B5A6B2291239266
:101E2000996BDA6B24912592196C5A6C2691279242
:101E3000996CDA6C08910992196D5A6D0A910B929E
:101E4000996DDA6D18911992196E5A6E0E910F9262
:101E5000996EDA6E04910592196F5A6F029103928E
:101E6000996FDA6F129113921A00803211685268DA
:101E7000069107921A008832116852680C910D92EF
:101E80001A0098339032106851685C681B6814938C
:101E90001594169A179B644C260080362260636066
:101EA0001A9A1B9BA260E3601C9A1D9B22616361CE
:101EB0001E9A1F9BA261E361109A119B22626362CA
:101EC000209A219BA262E362229A239B226363638E
:101ED000249A259BA263E363269A279B226463646A
:101EE000089A099BA264E3640A9A0B9B22656365C6
:101EF000189A199BA265E3650E9A0F9B226663668A
:101F0000049A059BA266E366029A039B22676367B5
:101F1000129A139BA267E367069A079B326073606D
:101F20000C9A0D9B2600883632607360260090362E
:101F3000306071602100149B159C98310B604C60DF
:101F4000C8233A4C5B002360903BFF3B2B703B6007
:101F500037E00A2202248C21BE20354B00920194E6
:101F6000073A49004000FEF7C9FD2B4D2B78002BA6
:101F700026D1304A3C6013601E222F4B1A6028B0D5
:101F800080BCB846F0BD002264210F2000F034F977
:101F90000023214D294A2B70294B0021009300205A
:101FA000284BFEF74BFD0122D02314001B065B6873
:101FB00090469B0B1C401A4248D02B78002BDED059
:101FC0001A4C05F059F8204B22681B689B18984260
:101FD000D5D9002264210F2000F00EF900232B70C8
:101FE000CDE7FFF783F80C4DE7E700230A4D3B6090
:101FF000E3E7C046FC9602209C8200106482001039
:1020000070820010F0960220549602203C8200104C
:1020100078820010C49602201D9702208C82001046
:10202000A4010020F802002098030020A80100204D
:10203000588200102CE60020AC010020FE020000B7
:10204000700600203E020000A4960220614804F0C1
:10205000F9FD4246604B1C60604B614C1A60614B5D
:1020600002321A60C8239B0023605F4C434626005F
:1020700080362B70A268E368069207932169626933
:1020800008910992A069E16904900591216A626A48
:1020900002910392A06AE16A226B636B0A900B9132
:1020A0000C920D93A16BE26B0E910F92206C616C00
:1020B00010901191A16CE26C12911392206D616DE0
:1020C000A26DE36D1490159116921793216E626EB6
:1020D00018911992A06EE16E1A901B91216F626F98
:1020E0001C911D9232687368A06FE16F26008836DC
:1020F0001E901F91209221933168726826009036BD
:10210000229123923068716826009836326873688D
:10211000364E249225932268636832607360069A73
:10212000079BB260F360089B099C33617461049B58
:10213000059CB361F461029B039C336274620A9B49
:102140000B9CB362F4620C9A0D9B326373630E9B1B
:102150000F9CB363F463109B119C33647464129BF3
:10216000139CB364F464149B159C33657465169AD0
:10217000179BB265F365189B199C336674661A9BAE
:102180001B9CB366F4661C9B1D9C336774671E9B87
:102190001F9CB367F467209A219B3400803422602F
:1021A0006360229A239B3400883422606360340089
:1021B000903420606160249B259C642098363360B5
:1021C000746001F021F943463B60F6E6084B0BE6EC
:1021D000084B09E640820010F0960220A40100207E
:1021E000A8010020B0960220F802002098030020E9
:1021F000B801002058020020F8B5CE464746050039
:1022000080B50E000421140000F048F92B075B0F85
:102210000520984601F010FF04F09AFA814630003C
:10222000184F784304F094FA011C484604F047FA2A
:102230008321C90504F057FA04F0B2FA434600219D
:102240009B00114A43449B009A1811609160D16031
:1022500001311761506011600C4A944622046344B6
:10226000120C29420CD00A4912041868424011404D
:102270008022520113431960C0BCB946B046F8BD74
:102280000449F2E710270000000005400C0005405B
:102290000000FFFFFFFF0000D0231B061B687B4AE6
:1022A00099005258F0B5574692465A1E9341302233
:1022B000DE464E4645465B421A401300744AE0B57E
:1022C000944683B063440193724B884608260F27D7
:1022D0009B463500083DEA081300019908339B002E
:1022E0005C58002C22D0012399465346002B27D05E
:1022F00039002140274213D05B4642469A584B464C
:10230000AB401A420CD1072208002A4092009040AC
:102310000200EB0860483C339B001A502800D0476D
:1023200024090135002C01D0AE42E1D80836282E10
:10233000CFD103B0F0BCBB46B246A946A046F0BD23
:1023400039002140274206D00133AB404546514871
:102350004059184276D02309E8D00F2211001940C5
:102360001A420DD04546F31F0E3A9A40494840594B
:10237000104205D1DB08484A3C3309019B009950C3
:10238000230AD3D00F22110019401A420DD045461E
:10239000B31F0E3A9A403F484059104205D1DB081E
:1023A0003D4A3C3309029B009950230BBED00F22BB
:1023B000110019401A4236D1230CB7D00F22110058
:1023C00019401A4243D1230DB0D00F2211001940F9
:1023D0001A424BD1230EA9D00F22110019401A42E4
:1023E0000DD04546B31E0E3A9A402A484059104235
:1023F00005D1DB08284A3C3309069B009950240F7D
:10240000721E002C00D191E70123404693402149E0
:102410000958194200D089E7D3083C331E4A2407E3
:102420009B009C5082E74546731F0E3A9A4019481C
:1024300040591042C0D1DB08174A3C3309039B00C6
:102440009950B9E7144B3C329200D15083E745468E
:10245000331F0E3A9A400F4840591042B3D1DB085F
:102460000D4A3C3309049B009950ACE74546F31EE6
:102470000E3A9A40074840591042ABD1DB08064A51
:102480003C3309059B009950A4E7C04630960220D2
:1024900000410140D896022000400140094A10B591
:1024A00094464024830063441A68C000624080342C
:1024B00014408022520113431C60034B9C4660442D
:1024C000416010BD04C0014000400140074B800046
:1024D0009C4660440368C90092000A435A400C239A
:1024E0001A4080235B0103431A60704704C0014017
:1024F000F8B51D00D0231B061C680600604244414D
:102500002F20644284432748F70884460720304040
:10251000800081403800244E3C3064448000BF007D
:102520008151E419002A11D08022920122431160C6
:102530001C681E4EA400A359002B15D0002D25D0D9
:10254000A55101210D2000F08FF8F8BDC0229201A5
:10255000224311601C68154EA400A359002B0CD017
:10256000002D18D0A551F0E7002DEAD000220D2053
:102570000F49A55100F0BCF8E3E7002DE5D000229B
:102580000D200B49A55100F0B3F8DEE70D200849F6
:1025900000F0A8F9D4E70D20054900F0A3F9A551F2
:1025A000D3E7C04630410140004001403096022050
:1025B00099220010024B18688007C00F7047C04670
:1025C00000C00640EFF3108072B6034A1368002B78
:1025D000FCD0BFF35F8F70472C0100D0BFF35F8F3B
:1025E0000022024B1A6080F3108870472C0100D043
:1025F00070B5EFF3108C72B60D4D2B68002BFCD02C
:10260000BFF35F8F0724CB08C618C05C01230C40C2
:10261000A3401C000440034207D118433070BFF3AD
:102620005F8F2C608CF3108870BD100001F01EFECF
:102630002C0100D00021044B044ABFF35F8F02C37A
:102640009342FAD17047C046000100D0800100D00B
:10265000044A1078431CDBB2172B00D910231370E7
:102660007047C046B0DD002001238340002904D01C
:10267000034A1360034A13607047034A1360FBE781
:1026800080E200E000E100E080E100E0024B103079
:102690009B688000C058704700ED00E070B50D00E9
:1026A000EFF3108672B60F4A1368002BFCD0BFF30D
:1026B0005F8F0D4B10309B6884001B590B4A93426F
:1026C00003D09D4201D001F0E9FD074B9B681D51ED
:1026D000BFF35F8FBFF35F8F0022024B1A6086F358
:1026E000108870BD240100D000ED00E0CD01001085
:1026F000F0B557464E46DE464546E0B585B0060085
:1027000000911700EFF3108B72B66A4A1368002B22
:10271000FCD0BFF35F8F0025674B5D579A46002DB5
:1027200000DA8BE06B00654C01935B199B009846C7
:10273000A146C1444B4652469B7910361370604BFC
:10274000B6009B6899590B1B2F2B33D95D4B9942CF
:1027500000D0ACE0019B42469C465B4B6544AD001B
:1027600063535A4B0232A218043B9B1A1B05584A6A
:102770005B0D651913436B80564B0121AB80FF2322
:10278000AB71009BEF71AB604B460B4319004C4B98
:102790009B689951BFF35F8FBFF35F8F0022454B5A
:1027A0001A608BF3108805B0F0BCBB46B246A94650
:1027B000A046F0BD01200A008243D3798C46BB427B
:1027C00031D84546130044491B1B5B415943090D51
:1027D0003D4B63533D4B02356519043B5B1B1B05A9
:1027E0003B4D5B0D2B43AA464D466B800425AC4602
:1027F0005546E044131F44441B1B1B055B0D1D4342
:102800004B46997100999D8099604946DF71334B21
:1028100001431360BBE75800C01880002018C1793D
:10282000B94211D902000623D356002BF3DA0293E2
:10283000131D9A462A4B6146039319E001F02EFDC1
:10284000002553465D576DE7908802934005131DA0
:102850009A46031561469C464046D444634604307C
:102860002018181AE0230005400D1B02184303909E
:1028700004235B429C46E14450464B461B1A1B0511
:102880005B0D9C46124B9571984663464046034348
:102890009380019B5A199200039BA418A380029B6A
:1028A0000E4AA371009B2260E771A3606FE701F0FD
:1028B000F5FC4FE7240100D01C970220B4DD002076
:1028C00000ED00E0CD01001000A1FFFFE4DD0020DD
:1028D00000E0FFFF01BDFFFFAAAA000001488047FA
:1028E00001BD0000F0B5DE4657464E464546E0B510
:1028F0000C0083B0EFF3108872B65D4A1368002BAA
:10290000FCD0BFF35F8F5B4B5B499A6803001033C9
:102910009F00D5598D4239D0A5424AD0574EAA1BA7
:102920002F2A33D801229246824091464846544A83
:102930001268104001904846524A1060BFF35F8F02
:10294000EFF305829346002A35D0934201D001F07F
:10295000A5FC2A0053469A439068844208D175E04A
:102960004B005B189B00F3189868A04234D01A0003
:10297000062151560029F3DA844253D0019B002BE3
:1029800026D04A46404B1A603D4B1A60394B9B6833
:10299000DD51BFF35F8FBFF35F8F0022344B1A60AE
:1029A00088F3108803B0F0BCBB46B246A946A046E7
:1029B000F0BD0D00EAE72A0053469A43906884422E
:1029C000D6D1062010561300002809DA0D0031E098
:1029D0004A462C4B1A60D9E706201856002822DBFD
:1029E00042001118890074188A46A1689960E1793B
:1029F000D971062161569971002925DBA488F11A45
:102A00006405241554440919E0240905490D2402DC
:102A10002143998013181D4A9B001178F31899716E
:102A20001070ABE713005946002914D1FF319171A2
:102A30001749918015490A789A71164A9B1B5B4188
:102A40005A43120D0A7099E71349E2E7062010561F
:102A500013000028C4DA114A1149D21A083A500268
:102A6000400D014399800F4952080A43DA8085E7F7
:102A7000240100D000ED00E0CD010010B4DD002005
:102A800000E100E080E100E080E200E01C9702202D
:102A900001BDFFFFAAAA000001BD0000EEDD00207D
:102AA00000F0FFFF00F8FFFF032310B50400074A02
:102AB00018409446C0009C43FC3383406444226821
:102AC00081409A4313000B43236010BD00E400E0F3
:102AD00070B5EFF3058101240443EFF3108C72B657
:102AE000214A1368002BFCD0BFF35F8F1F4B0500FA
:102AF0001F4AED1A6D416A43120D1E4D8900AE68E2
:102B000052B27658A6421CD00621595691421CD08A
:102B100012215956914222D01E215956914220D05D
:102B20002A2159560324914210D0134B19781A7058
:102B30008171BFF35F8F00220B4B1A608CF31088FA
:102B400070BDAB680D4C5C50EFE7002461000919C3
:102B500089005B18FF21997109499980E5E70124F3
:102B6000F4E70224F2E7C046240100D0B4DD0020DF
:102B7000AAAA000000ED00E01C970220CD01001081
:102B800001BDFFFF054B064A1360064A1360536000
:102B90009360D3601361536193617047808080803C
:102BA00000E400E004E400E0024B9C46614489003C
:102BB000016070474000003410B50400FFF748FD85
:102BC00001002000FFF7F0FFFF232371BFF35F8FA9
:102BD00010BDC04610B50400FFF73AFD010020000B
:102BE000FFF7E2FFFF23A380BFF35F8F10BDC04656
:102BF00083680B4810B584466144624412010901A0
:102C000059189B185C684A680120944201D802D088
:102C10000020C0B210BD1A680B689A42F9D8F7E7D5
:102C2000FFFFFF0F10B508000B690C009847002844
:102C300002D02068616810BDE06000210020FAE742
:102C40000A4B1968EFF3108072B60A68002AFCD0AC
:102C5000BFF35F8F1B68BFF35F8F00221A6080F3A2
:102C6000108840BF002000217047C046F89602201F
:102C7000F8B5574645464E46DE46E0B598460CAB9D
:102C80001C780DAB1B78070091469A460568002C0E
:102C90005ED1AC7B002C3BD0660029683619033E20
:102CA00089194B78AB73002B00D1EB7300238B7029
:102CB0004B700B702D4BE218BB6812019B184A46F3
:102CC0001A6042465A600A9A9A600B9ADA600023A8
:102CD0008B704B700B706B7B9B46002B2BD02200B4
:102CE0005946A8686B6898472A68002816D05B4642
:102CF00058465B005B449619033BB070D118D35C17
:102D0000002B00D073705B460C706B735C4513D066
:102D1000F0BCBB46B246A946A046F8BD5B465B0088
:102D20005B44033BD3189C709119925D002A00D03C
:102D30005A705B460B706C734A464346387D00F010
:102D4000F3FC051E0AD10E9B002BE1D01D70DFE7BE
:102D5000660029683619033E8919ABE75346002BF4
:102D6000F1D12100386800F003FFECE7FFFFFF0F0F
:102D7000F0B5DE4657464E4645460023E0B58BB0DB
:102D80000893684B8200D45800239B46099000F0BA
:102D900037FC02000B006068EFF3108A72B65646EB
:102DA00001680029FCD0B246BFF35F8F21684F7BDA
:102DB0008C46002F2ED0A5685B49A94679180901D9
:102DC000894449460868496805000E00AD1A9E41CD
:102DD000002E5FDD02000B00099800F0A5FC002327
:102DE00000229946002306920793002398466368C1
:102DF000BFF35F8F5A461A608AF310884346002B50
:102E000012D10028C3D10BB0F0BCBB46B246A946D4
:102E1000A046F0BD002300229946002306920793A6
:102E2000002300209846E2E7089B494618023843F1
:102E3000C047626805000E00EFF3108A72B613688F
:102E4000002BFCD0BFF35F8F002E41DB2B00334300
:102E500002D02369002B56D12368D97B002905D0E5
:102E60001A68480041185218033A57709A7B002A92
:102E700000D19F73DF73E268013FD35D0133D35507
:102E80005B4623616368BFF35F8F5A461A608AF31B
:102E900010887CE7002E02D1002D00D09AE7002197
:102EA000604600F0E3FD4B461A685B6806920793A4
:102EB0004B469B6898464B46DB689946E368DB19AE
:102EC000013B1B7808931B020343236100208EE71C
:102ED0002369002BC0D0069A079B8021521BB34167
:102EE00009068B4202D30122104B52420021049169
:102EF000013103914946019141462000029700911A
:102F0000FFF7B6FEBCE700F07BFB2A003300121887
:102F10004B41802109068B42E8D30122034B5242E8
:102F2000E4E7C046C8960220FFFFFF0FFFFFFF7FC8
:102F300010B5144C6368002B04D00A211248FFF727
:102F400033FE10BD2300114A1021206800F0A4FCBC
:102F5000032000F049FB032000F04EFC03200C4945
:102F600000F09CFBFFF774FB0A4B9C460323237580
:102F7000D0231B061B6860446375074B80006060AC
:102F8000DC60DAE7FCDD0020F8960220F12B00106F
:102F9000712D001040000034C89602200048704790
:102FA000FCDD0020F0B557464E464546DE46E0B50E
:102FB00085B0019310AB1B780600039300239A465B
:102FC000984600927268EFF3108B72B61368002B6C
:102FD000FCD0BFF35F8F3568AC7B002C00D16FE075
:102FE00067002B683F19033FDB195A78AA73002A40
:102FF00000D1EA734B4AA118B2680901521800982F
:103000000199106051600E9991600F99D16042460C
:103010009A705A701A706B7B9946002B00D170E041
:1030200022004946A8686B6898472A6800285BD048
:103030004B4648465B004B44D719033BB870D11848
:10304000D35C002B00D07B704B460C706B734C45EF
:1030500058D0F3681B19013B18787368BFF35F8F72
:1030600042461A608BF310885346002B08D10002A9
:10307000204305B0F0BCBB46B246A946A046F0BD11
:10308000039B002B4BD00E9B00200F999847030009
:1030900004000D000B4342D000291ADA009A019B6C
:1030A000121BAB410092019380221206934204D37B
:1030B00001231D4C5B4200930194039B9A4681E7D8
:1030C0007368BFF35F8F1C608BF310880120404250
:1030D000CFE700F095FA802224184D4112060094A3
:1030E00001959542E9D3E3E74B465B004B44033B34
:1030F000D3189C70D119D25D002A00D05A704B466B
:103100000B706C73307D009A019B00F00DFB8246C2
:1031100000289ED02100306800F02AFD99E70020A9
:10312000A7E7C046FFFFFF0FFFFFFF7FF0B5574641
:103130004E46DE4645461100E0B585B006009C4689
:10314000109F194300D1EDE06146DB170193009316
:1031500053401C00019B4B401D0000980199241A0C
:103160008D4163460E997B600F9BBE607B61396128
:103170003A6000F045FA8023001969411B0600906F
:103180000191994204D301236B4C5B42009301945B
:1031900000239846694B1097039300239946109B90
:1031A0003700464698467A68EFF3108B72B613687C
:1031B000002BFCD0BFF35F8F3D68AC7B002C00D1AF
:1031C00079E063001B19033B1A00944602932B68B5
:1031D00063445A78AA73002A00D1EA73584AA118A6
:1031E000BA6809015218009801991060516003995A
:1031F00091604146D1604A469A705A701A706B7B52
:103200009A46002B00D17FE022005146A8686B68E7
:1032100098472A68002800D168E053465B00534471
:10322000033B9C46D118534602981018837063469E
:10323000D35C002B00D0437053460C706B73350089
:10324000544562D0FB687A681B19013B1B78BFF3B9
:103250005F8F494611608BF31088002D0CD14746D3
:103260001B02234301352800FB6005B0F0BCBB46C0
:10327000B246A946A046F0BD434640461B69984762
:10328000061E24D042461468556822002A434FD0B7
:10329000002D1FDA009A019B121BAB410092019393
:1032A00080221206934200D27DE70123224C5B422A
:1032B0000093019477E73E0047467368BFF35F8F42
:1032C0001C608BF31088012300255B42CBE7474647
:1032D0000023C8E700F094F9802224184D4112061B
:1032E00000940195954200D25DE7DEE753465B000E
:1032F0005344033B0298D3189C701118125C002AA7
:1033000000D05A7053460B706C73387D009A019B45
:1033100000F00AFA051E00D194E72100386800F099
:1033200027FC8FE700230124002501229C4618E793
:1033300047460500002396E7FFFFFF7F252C00107E
:10334000FFFFFF0FF0B504000D0006267642F717C9
:10335000C64636196F4100B584B08F4214D811D0DB
:1033600000F04EF932003B00121A8B41002B15DCA5
:10337000002B3ED02000290000F080F904B080BC72
:10338000B846F0BD8642EBD90026002700F038F998
:1033900032003B00121A8B41002BE9DD002302931F
:1033A0000193154B3200009314483B00FFF7FAFDE0
:1033B0000028DFDB00239846BC46114A114F7B6A88
:1033C0009C4504D8B96AB142D4D29C45D2D1116887
:1033D000EFF3108072B60B68002BFCD0BFF35F8F49
:1033E0001368BFF35F8F4146196080F3108820BFD8
:1033F000E5E7002ABED0D1E7412C0010FCDD00201B
:10340000F89602200040054070B5060000F0F8F87C
:10341000FA2204000D00002330000021920003F086
:103420002BF98023001969411B06994202D3012020
:1034300002494042FFF786FF70BDC046FFFFFF7F95
:10344000F0B5EFF30583CE46474680B505000C0086
:1034500085B0002B0DD0324A0020536A9C4203D81D
:10346000926A0130AA4232D305B0C0BCB946B04618
:10347000F0BD2C4E029301932B4B020000933000C1
:103480000B00FFF78FFD031EE5DD20BF7168EFF332
:10349000108772B60A68002AFCD0BFF35F8FDAB2D9
:1034A00094463068427B624516D0FF2201681A407C
:1034B00089465100884649469044414403398978F9
:1034C00000290BD13269934210D131610EE0E31A29
:1034D0005A1E9341D8B2C7E7FF221A40F1681B0A6F
:1034E0008A18013A1278DBB29A4214D07368BFF39B
:1034F0005F8F00221A6087F31088094B00205A6AF8
:103500009442B1D89B6A0130AB42ADD2A41A631E7B
:103510009C41E0B2A8E7614600F02AFBE6E7C0461E
:1035200000400540FCDD0020412C0010F0B5EFF319
:103530000582D6464F4646461000C0B51038EFF318
:10354000108872B6214C2368002BFCD0BFF35F8F2C
:103550000123190081401E4D1F006963AA461D4DBD
:1035600029601D4D2E78AC463500C5402F402B42BA
:1035700015D053465F6A194B8500EB589F4218D30C
:103580006246174B8E43EB581670BFF35F8F0022D5
:10359000226088F31088002B06D0984704E0BFF320
:1035A0005F8F276088F31088E0BCBA46B146A84612
:1035B000F0BD0C4B92009C46624413681360BFF34D
:1035C0005F8F0023236088F31088EDE7280100D087
:1035D000004005403C7005401F97022000970220E4
:1035E00018E60020D03F054010B5034B010018003D
:1035F000024AFEF7FDFF10BD18970220B0820010AE
:10360000034B596A0A00986A596A8A42FAD170478C
:103610000040054070B504000D00174A536A1900B8
:10362000966A536A8B42FAD13000190024184D4132
:10363000AB4216D813D0104B2A005B6A9D4203D9C7
:103640000D494B6A9342FCD3934207D10A4A02E0E8
:10365000516A994202D1916AA142F9D370BDA64242
:10366000E9D9054B5B6A1C005A1CEFD001220124EA
:103670006442E5175242E3E700400540064A536AB8
:103680009942FCD807D1044B02E05A6A914202D118
:103690009A6A8242F9D370470040054070B5040031
:1036A0000D00EFF3108672B61A4A1368002BFCD097
:1036B000BFF35F8F002D1BD02000FEF7E7FF1649F8
:1036C00081420AD02000FEF7E9FF01212000FEF729
:1036D000CBFF0123A340114A1360114BA400E55016
:1036E000BFF35F8F00220B4B1A6086F3108870BD0A
:1036F0000121A1400A4BA200D5500A4B20001A78A4
:103700008A4305491A70FFF7EDF800212000FEF703
:10371000ABFFE5E7280100D02D35001038600540EB
:1037200018E600201F970220F0B54F46D6464646C1
:10373000C0B507002B4C616A0D00A66A616AA942F8
:10374000FAD18B4208D805D00120E0BCBA46B14678
:10375000A846F0BDB242F7D9EFF3108A72B62248FC
:1037600001680029FCD0BFF35F8F0125BD401F49D0
:103770001C4C8846097889462943C9B28C46414683
:1037800060460870391D890065630A511849B80000
:103790004350216A0020294219D0616A0800A66AB4
:1037A000616A8142FAD18B4219D801D1B24216D84E
:1037B000CC450BD00B4B1F221D625D6301233A40A9
:1037C00093400C4A136043464A461A700120BFF3E7
:1037D0005F8F0022044B1A608AF31088B5E700203F
:1037E000F5E7C04600400540280100D01F970220A1
:1037F0000097022080E200E0EFF3108C72B60A49D5
:103800000B68002BFCD0BFF35F8F01238340074A76
:103810000748136202789A430270BFF35F8F002358
:103820000B608CF310887047280100D000400540E1
:103830001F97022070B505000E001400002923D048
:10384000002A12D080686B689847296800280ED03B
:1038500063001B197200033B9219CB18033A9E7048
:1038600088188A5C002A11D10470300070BD730082
:103870009B196200033B1219CB18033A9C708818FD
:103880008A5C002A05D106702000EFE75A700470A8
:10389000EBE75A700670F7E730B583600023CCB2CF
:1038A00043730133047342608373C4730D00006873
:1038B000012C06D9421C0133DBB2137003329C4247
:1038C000F9D1FF2129404B005B18C01800230338B1
:1038D000437030BD70B505000C1E07D06300016851
:1038E0001B19033BCB185A78002A01D1200070BD68
:1038F000500080180338091800204E7848702100C5
:1039000058702800FFF796FF310004002800FFF7E9
:10391000E1FF0600002C26D00028E7D0210032006D
:10392000A8686B689847296800280ED073009B1917
:103930006200033B1219CB18033A9C7088188A5C0A
:10394000002A00D05A700670D0E763001B1972007D
:10395000033B9219CB18033A9E7088188A5C002AA0
:1039600000D05A7004703400C0E7C046F0B5574626
:103970004546DE464E46E0B50D006F0001687F19F2
:10398000033F0400C85D83B00192CA19002850D0DB
:1039900043001B18033BCB185E78B446002E1AD1A7
:1039A000019E002E42D0E67B002E04D073009B19AE
:1039B000CB18033B5D70A37B002B00D1A573E5738F
:1039C00000282FD10023537003B0F0BCBB46B24691
:1039D000A946A046F0BD72006244033A8A185178A5
:1039E000884600215170894659703200010020003C
:1039F000FFF720FF43468246002B07D05B0021687B
:103A00004344033BCB185A78002A16D1424651460C
:103A10002000FFF70FFF2168019BCA19002BC2D1BC
:103A20000028CFD043001B18033BCB18002199700E
:103A3000C8E7019B002BB6D1C4E7500080180338BB
:103A40000918487883464846487058704146200017
:103A5000FFF7F0FE594680462000FFF73BFF414646
:103A600002002000FFF7E6FE8046CFE7F0B557469C
:103A70004546DE464E46E0B583B00191457B0400E5
:103A80006F0000687F19033FC15DC219002952D041
:103A90004B005B18033BC3185E78B446002E1CD164
:103AA000019E002E44D0E67B002E04D073009B19AB
:103AB000C318033B5D70A37B002B00D1A573E57396
:103AC000002931D1002328005370617303B0F0BC8A
:103AD000BB46B246A946A046F0BD72006244033A16
:103AE000821850788046002050708146587032000D
:103AF0002000FFF79FFE43468246002B07D05B0065
:103B000021684344033BCB185A78002A17D1424618
:103B100051462000FFF78EFE019B01002068C2196C
:103B2000002BC0D10029CDD04B005B18033BC3183C
:103B300000209870C6E7019B002BB4D1C2E750006B
:103B400080180338091848788346484648705870EA
:103B500041462000FFF76EFE594680462000FFF7E1
:103B6000B9FE414602002000FFF764FE8046CEE722
:103B700070B5050000292CD0437B8B422ED04C0021
:103B800000686418033C0419A278002A21D053006D
:103B90009B18033BC25CC6188A4202D11BE0002A74
:103BA00008D053009B18033BC3185A788A42F6D1B9
:103BB00062785A70002301222800A3706370FFF717
:103BC000D5FE697B02002800FFF734FE68730120F0
:103BD00000E0002070BD63783370EBE7012219002C
:103BE000FFF7C4FEF2E7C046F8B5CE4647460400EC
:103BF00080B506200E0000F01FFA051E51D0524B72
:103C00005249E21853425A418023DB039C469205F5
:103C10004F4B62441A604F4B1A6010008B689843F8
:103C2000FBD1494B4C4AE31859424B4180215B0080
:103C300049000620995200F0FFF93100C00001F060
:103C4000C9FEC30932D14022012190466162A362BC
:103C5000256BEB0736D427008026E36A00232C3738
:103C600076013E4333600620256300F0E5F94146C6
:103C7000800001F0AFFE236B05009846DB073BD4C4
:103C80006023E26A5A400E33134033604346236395
:103C9000802310229B013B431A60304B2363032394
:103CA000A3642800C0BCB946B046F8BD2C4A934274
:103CB0003FD900232B492C4A6162A362256B9046B1
:103CC000EB07C8D52200C02330329B011343234A9F
:103CD00006201A60666AA36AB601F61800F0ACF90D
:103CE000224901F077FEB6020100300001F072FEB9
:103CF0000021FFF78FFCAEE72200C02330329B018A
:103D00001343164A06201A60636AA26A9B01994609
:103D1000914400F091F94B4614499B02994601F0F9
:103D200059FE0100484601F055FE0021FFF772FCE4
:103D3000A6E77F2299018846024001325208190005
:103D40009044130082E7C0460080FCBF00C00040E2
:103D500000E0004000F00040109702200103000046
:103D6000FEFF0000FFFF0000C0FF3F004E0E0000FE
:103D700010B50C2082B000F0B5F9FEF71BFC00284E
:103D800010D08B4B8B488B498B4A186059609860D8
:103D9000D960186159619861D961186259625A6293
:103DA00002B010BD854CA06700F0A4F90122844B3D
:103DB0001A60636C012BFCD10322824B1A607F4A8C
:103DC000936B012BFCD1013301217F4A7F48009383
:103DD000043300F037F905237D4A009301217D4823
:103DE00000F030F97C4B5A68FF2A02D8802252003A
:103DF0005A608022734B6E4C12011A6021690029AF
:103E000007D0606901F0E6FD013043001B18033B59
:103E1000FDD2E022704B714819680A40026002220C
:103E20001968514001320A40042102609A68114227
:103E3000FCD080216A4A09011160802252005A6038
:103E4000684B2361684B5968FF2900D85A600322E8
:103E500001215B4B1A60644A93681942FCD0E0234D
:103E60001068034061480360126803234A4002213E
:103E700013405D4A036093681942FCD080215C4B7B
:103E80000901196080215B4B4900516063615A4B05
:103E90005A68FF2A00D859608022584B12011A60D4
:103EA000E169002907D0606901F094FD0130430009
:103EB0001B18033BFDD2E0234F4A11680B405049C9
:103EC0000B6080214F4B090119608021394B49005B
:103ED0005160E3614C4B5A68FF2A00D85960802238
:103EE0004A4B12011A60216A002907D0606901F06B
:103EF00071FD013043001B18033BFDD2E023424A11
:103F000011680B4042490B608021424B0901196046
:103F100080235B0053608022264BD20223623E4BFB
:103F20005968914200D25A6080223C4B12011A60BB
:103F3000616A002907D0606901F04CFD013043003F
:103F40001B18033BFDD2E023334A11680B40344970
:103F50000B608021334B090119608023DB02536021
:103F6000154B6362304B5A68FF2A02D880225200F8
:103F70005A6080222D4B12011A60A169002907D0D6
:103F8000606901F027FD013043001B18033BFDD29F
:103F9000E023254A11680B4025490B608021254B01
:103FA0000901196080235B005360124BA361F7E69F
:103FB000B8E20020006CDC021BB70000008000406B
:103FC0003CB0004030B00040002F685900800240F3
:103FD000008C864700C00240308000403090004096
:103FE00030A00040001BB7003C8000403C900040E7
:103FF0003CA00040405973075480004054B000403A
:104000005490004054A000406080004060B00040E8
:104010006090004060A000406C8000406CB00040A8
:104020006C9000406CA000404880004048B00040C8
:104030004890004048A00040014B8000C0587047A5
:10404000B8E20020F8B5040021481D0017000E005A
:1040500001F0C0FC0100380001F0BCFC069B290403
:104060001B0319432368002B20DB1A4B1A4DE2185F
:1040700053425A4180235B019C461203174B624412
:104080001A60174B1A601700AB689F43FBD1C02220
:10409000231D92011A4321232660A0601360236828
:1040A000002BFCDA0823E1601360F8BD3F2322688F
:1040B0001340B342D9D1A3681B051B0D8342D4D151
:1040C000EE22E368D20213408B42CED1EDE7C04628
:1040D000001BB7000040FDBF00C0004000E00040F2
:1040E00000F000408023024A9B000343D3627047E4
:1040F00000800540AA23064A1B0113602F230549AF
:10410000D360054B19605368002BFCDA7047C0463A
:104110000040024000B0FA00006002402C4B2D4AE3
:1041200070B51A602C4A2D4B2D491A6014008B680B
:104130009C43FBD12B4D2C4EB54208D2013E761B41
:10414000B60808CD984723000134B342F9D1FFF7F0
:104150000FFE264A214B1A60214A9368DB43DB019C
:10416000DD09002BF9D14022214B224C224E9A67C7
:104170005A671A67DA66B44208D223682000002B17
:1041800020D00834FEF726FDB442F6D31B4C1C4E5B
:10419000C022B168200002F081FBB460FEF74AFA49
:1041A000FEF7F0FCFEF7C4FE164C174EB44208D2E0
:1041B000013E361BB60808CC98472B0001359E42BD
:1041C000F9D170BD0834FEF7F7FCB442D5D3DDE772
:1041D00000E00040BFCDFBFEFE7F3C0000F0004051
:1041E00000C00040A0E20020B0E20020FFFFFF017D
:1041F00000F0014098E20020A0E200200000002032
:1042000000ED00E0B0E20020B4E2002000BEFDE7D7
:1042100010B5041E0DD0FFF7F3F9074B1A685B6861
:10422000801A99410023054A01F0FAFB2060616081
:10423000A260002010BDC046E0E3002040420F0015
:1042400010B50400FFF7DCF90023054A01F000FC7B
:104250000023206063600020A360E36010BDC046BF
:104260001027000010B5FFF7D1FFC0460FB400B50E
:10427000084883B002F0F4FB049B002B07D005A98B
:104280001800019101F02CFB034802F0E9FB01202A
:10429000FFF7BCFFD4820010E482001010B5014883
:1042A000FFF7E4FFE88200109A4200D2885470477A
:1042B0007047C046F8B557464546DE464E46E0B51F
:1042C00098460A9B06009A460D9B0F0093461500E0
:1042D0009B0710D10B9B0C9A93420CD213005C46A7
:1042E0000B9A9D1A5D442200434601343900202078
:1042F000B047A542F7D10B9C6319002C09D01D00D3
:1043000053462A1B013C185D39004346B047002C38
:10431000F6D10D9B9B070ED55B46EC1A0C9BA34276
:1043200009D999462A004346390020200134B04774
:104330000135A145F6D82800F0BCBB46B246A946D7
:10434000A046F8BDF0B54F464646D646C0B584B047
:1043500098460EAB1B7894469946129B0D9C109F75
:10436000119E9A0724D4002E6AD1BC4220D2012289
:104370001A409246202C00D1CBE00C9A551E3022D8
:1043800001E0202C30D001342A55A742F9D85246FA
:10439000002A0DD0B4420BD20C9A551E3022202C8C
:1043A00002D126E0202C61D001342A55B442F9D143
:1043B000DA0634D55A0562D4002C5CD10F9A102A43
:1043C00000D191E0022A00D1A1E030220C9C2270A1
:1043D00001244A46002A5CD15A0700D47DE02B22F2
:1043E0000C9D2A5501341CE05246002A02D0202E92
:1043F0003CD92024DA0614D55A0512D4202F00D136
:1044000097E0202E3BD120261F2234000F9D102D37
:1044100000D181E0022D4CD030250C9FBD54202CC2
:10442000D7D103930C9B62460093029643460194B6
:10443000FFF740FF04B0E0BCBA46B146A846F0BD65
:10444000012215001D40AA461A4227D04A46002ADA
:1044500033D10C321A4230D1BC429BD2202C00D036
:104460008BE7202EC5D8DA06A4D4DAE72024DA06B2
:10447000D7D55A0503D4A74221D0B4421FD00F9AF2
:10448000102A21D0022A10D0202CCAD022000134B8
:10449000C2E72D220C9D2A550134C2E7BC4200D34D
:1044A00086E7202C00D068E7E1E7202CB9D0220075
:1044B000013462250C9FBD54E6E7013ECCE7621E45
:1044C000012C00D17AE7A1E79A0616D4202CA8D0B7
:1044D00078220C9D2A550134D6E71A07A1D520224F
:1044E0000C9D2A5501349CE79A060ED478220C9C28
:1044F00022703022627002246BE7202C91D0582564
:104500000C9A121915700134BEE75822EFE76222A7
:10451000EDE7002AA7D1AAE7023C9D0604D478253E
:104520000C9F3D551400B1E758250C9F3D551400D4
:10453000ACE71F226AE7C04610B5002800D110BDC5
:1045400002F042FAFBE7C0460B0010B5002802D08B
:1045500049681B68984710BDF0B557464E4645461A
:10456000DE46E0B599B08246894690460993229A84
:10457000239B1000190001F0EEFC002800D0C8E0D9
:10458000229823990122D54B524201F0DFFC0028EA
:1045900000D0BEE0229823990122D14B524201F073
:1045A000C7FC002800D0B4E0229823990022002301
:1045B00001F0BEFC002800D0E9E1229E239F802369
:1045C000269ADB001A400D92269A1A4201D1062340
:1045D00024933B00334300D0B4E0269B1B0500D559
:1045E000BFE1002300240A930B94002304250C93BD
:1045F000259B0024AB4200D95C1B0223269A1A405B
:104600000D92269A134203D06B426B415B421C40D1
:104610000C9B002B07D00A9A0B9B3000390001F04D
:1046200026FC06000F00229823990022002301F0A7
:104630007FFC002803D0802109067B181F00269AE2
:10464000A84B009601971340099E0493249B039462
:104650000293424633004946504600F0A7F9040051
:10466000002D67D02020269A4946024013005A4266
:1046700053415B42621C18400A92330022004530CD
:10468000D0470C9A6F1ED317D4185C40D30F9B46AB
:10469000002501E0202D13D008AA94461F232000F6
:1046A00063440A2101355E1901F094F9303131700B
:1046B00020000A2101F08EF926000400092EE9D815
:1046C00005230693002304930A3303935B46099E54
:1046D000029310AB0A9A009349463300504605975F
:1046E0000195FFF72FFE0D9A0400002A22D04246C2
:1046F000851A259AAA421DD9B046574616002200AF
:104700004346494620200135B8470134AE42F6D829
:1047100010E0269B42460493259B49460393249B25
:1047200050460293229B239C00930194099B00F026
:104730003DF90400200019B0F0BCBB46B246A946C2
:10474000A046F0BD684B78009C46400D604401F0E7
:1047500015FC664A664B01F0A8FB664A664B01F001
:104760007DFB664A3B031B0B1A4304000D00644BA0
:1047700011003000002201F068FB624A624B01F038
:1047800094FB02000B002000290001F067FB01F000
:104790000DFC0C9001F0F2FB5C4A5D4B04000D0037
:1047A00001F083FB00225B4B01F058FB01F0FEFBA4
:1047B000594A8346594B2000290001F076FB04003A
:1047C00058460D0001F0DAFB554A564B01F06DFBDF
:1047D00002000B002000290001F037FB02000B0053
:1047E0000A900B9101F061FB04000D000A980B99EF
:1047F00002000B0001F032FB00220E900F914A4B99
:104800002000290001F033FB0022484B01F026FB79
:1048100002000B002000290001F029FB0022444B7C
:1048200001F01CFB02000B002000290001F01FFB1F
:104830000A9A0B9B0D0080210400C905002001F09D
:1048400004FB02000B002000290001F007FB394C9B
:1048500002000B000E980F9901F009FB5C44002246
:10486000264B01F0FBFA2305002201F01EFB040099
:104870000D0002000B00300039000A940B9501F086
:1048800057FB00285ED123002A00C6250C9963310E
:104890008D42AD4126996D420435090500D4A7E645
:1048A000134364D030003900234A244B01F046FB07
:1048B000002807D0002230003900214B01F038FBDE
:1048C000002854D1249B002B00D191E60D9B5A1E49
:1048D0009341249AD31A24938AE6C046FFFFEF7FC0
:1048E000FFFFEFFFFFF7FFFF01FCFFFFFB799F508A
:1048F0001344D33FB3C8608B288AC63F0000F03F03
:104900000000F83F61436F63A787D23F71A3790925
:104910004F930A400000E03F1655B5BBB16B024013
:10492000EF39FAFE422EE63F00002C400000244002
:1049300000001840FF0300002D431CEBE2361A3F35
:1049400080842E410C9B0022013B0C932000164BCF
:10495000290001F08CFA0A00010003000A910B9271
:1049600093E7002300240A930B9400230C93249ACA
:104970000C9B9A4214DDD31A013B24938023269A80
:10498000DB001A430023002526920C9330E6802298
:1049900012069446229B1E00239B63441F000EE6D2
:1049A00000232493EAE7C04600002440F0B54546C2
:1049B000DE464E465746E0B595B08B469046994642
:1049C0001E9A1F9B0A9019001000209D01F0C3FA47
:1049D000002800D0B0E11E981F990122C74B524217
:1049E00001F0A6FA002800D037E11E981F99012295
:1049F000C34B524201F0AAFA002800D0A7E01E984B
:104A00001F990022BF4B01F0A1FA002800D088E0D6
:104A10001E981F990022BC4B01F08AFA002800D092
:104A20007FE01E981F990022002301F081FA0028E0
:104A300000D0FAE000230B938023229C229ADB0013
:104A40001C401A4200D102E1092D00D87EE106A9DE
:104A50008C462C00172200233021093C624401338C
:104A6000D154EF1A202B00D132E1A342F7D100221A
:104A7000A44B069207931E981F9901F097FA050020
:104A800001F07CFA02000B001E981F9901F0DDF97D
:104A9000069A079B01F009FA0890099101F0AAFA19
:104AA000060001F067FA02000B000898099901F06E
:104AB000CCF90022954B0890099101F047FA0028A3
:104AC00000D1D2E00136300001F054FA069A079B7B
:104AD00001F034FA002801D000260135AA46002F43
:104AE00000D098E0280001F049FA02000B001E985F
:104AF0001F9901F0AAF9854B002206000F0001F072
:104B000017FA0CAB9A46002845D100223000390034
:104B10007E4B01F01BFA00283DD1EB073BD5013558
:104B200039E0229B42460493219B594603930A98FD
:104B30001E9B1F9C0295009301944B46FFF70CFDB2
:104B400015B0F0BCBB46B246A946A046F0BD229BBC
:104B50005B0767D403226E4B22990192039121993E
:104B60000291009342464B4659460A98FFF7A2FB32
:104B7000E6E706AA94461723280063440A21013475
:104B80001E1900F0FFFE3031280031700A2100F0BC
:104B9000F9FE051E76D0202CEBD10323229A134078
:104BA000012B1DD1219B002B1AD00B9B002B00D079
:104BB000BBE0229A0C33134200D0B6E0219BA34203
:104BC00000D887E006AB9C4617223023624404E0FD
:104BD0002199013413558C4259D0202CF8D120242E
:104BE000229B01940393219B02935346B9E706AAA3
:104BF000944617230A216344300001341D1900F044
:104C0000E9FE3031297030000A21013F00F0E2FE58
:104C1000092E46D90600202CE9D155460CAB20249C
:104C20009A46B8E704223B4B96E71E9A1F9B00204A
:104C3000002101F00AF901230B938023229C229A80
:104C4000DB001E901F911C401A4200D0FCE600229F
:104C5000314B0627069207930DE7229B0393219B76
:104C60000293042301932D4B7BE7002208980999B6
:104C7000264B01F05DF9002800D02FE7002E4FD120
:104C800001362BE70323229A1340012B68D0202CF6
:104C9000A6D00B9B002B1FD02D2352461355013459
:104CA0009EE75546202CB9D030223B19002F4BD01F
:104CB000172006A9013409180A55202CAED09C42B1
:104CC000F6D10CAA92462E2251465C1CCA5462E7C9
:104CD0002024CCE6202C83D0229B5B0708D4229B87
:104CE0001B0700D47CE7202352461355013477E795
:104CF0002B2352461355013472E7C046FFFFEFFFE6
:104D0000FFFFEF7F65CDCD4165CDCDC10000E03F18
:104D1000FC820010F482001080842E410483001075
:104D2000F30700D4DAE60136D8E6219B013B219354
:104D3000A34200D946E7AAE7229B0393219B029353
:104D400003230193084B0CE72300BAE7074BEA0063
:104D50009B185C681B682F000693079400248AE662
:104D6000219B002B93D020E700830010A884001023
:104D7000F0B5DE4657464E464546E0B59FB01C00AE
:104D8000289B93460A93CC4ACC4B8A4609901A60DA
:104D9000002900D14DE1002320789946002800D158
:104DA0004FE1C74B4D460893C64B0D930AE02A00CE
:104DB0006E1C5B46099D5146A8473500013420789A
:104DC000002872D02528F2D110239946083B984636
:104DD000043B00219C460227013420782600030072
:104DE000203BDBB2102B03D8089A9B00D3589F4678
:104DF0000300303B092B6ED900272A2800D18AE016
:104E000000230B932E2800D176E00300683BDBB231
:104E1000122B1BD8AC4C9B00E3589F460123013456
:104E20001943DAE739430134D7E7634601341943BC
:104E3000D3E74B4601341943CFE7434601341943C6
:104E4000CBE780235B0070781943013667280AD8C6
:104E500024281FD90300253BDBB2422B1AD80D9A18
:104E60009B00D3589F460300693BDBB20F2B11D840
:104E700001249C40954AA446904614400C946246F6
:104E80004446224200D025E20A2B00D101E1072B43
:104E900000D1D8E0099C2A005B465146A0477078B3
:104EA0006F1C741C3D0000288CD1A9462C00CB45FA
:104EB00003D801235B425B4499465B464A46514610
:104EC0000020099DA84720001FB0F0BCBB46B24699
:104ED000A946A046F0BD0027BB00DF1901367F00C0
:104EE0003F183078303F0300303B092BF4D90023C2
:104EF0000B932E2800D088E780237078DB001943BD
:104F00000300303B741C092B00D82CE12A2800D167
:104F100038E1260079E70A9B80CB002F03DB60781D
:104F20000A93661C6CE70222607811437F420A9361
:104F3000661C65E7672800D1C8E1472800D104E274
:104F4000452800D104E207200A9B049107338343DC
:104F500019000B9A039702920CC9099800920193C9
:104F60000A912A005B465146FFF7F6FA741C0500C9
:104F700025E770786C2800D10DE280235B0019438F
:104F8000013663E780239B007078194301365DE7A3
:104F90007078682800D1F9E180230136194355E77C
:104FA000462800D18FE107200A9B049107338343F1
:104FB00019000B9A039702920CC909980092019369
:104FC0000A912A005B465146FFF7F0FC741C05006D
:104FD000F5E62A00099C5B46514625206F1CA04738
:104FE0003D00741CEBE6890700D4DEE10A9B2A0031
:104FF00098466B1C9946434601CB51469846099CFE
:105000005B46C0B2A047ED19012F00D893E24C4691
:10501000B1465646099F22005B46013431002020EC
:10502000B847AC42F7D1B24643464E460A93741C89
:10503000C5E6274B2078099300239946002800D025
:10504000AFE6002433E70A9B1A0008CA9046002BFB
:1050500000D1A7E0212008430EA98C461F226244FC
:105060000F27AC46814615000C9C02E0202C0CD08A
:1050700013003800184001003731092800D80739DB
:10508000013429551A090F2BF0D8654648460C946F
:1050900094E00A9B1A0008CA12920B9A002A7BD14C
:1050A00002241A786442002A1DD0013418199C4643
:1050B0001C00030010E0C046714D0010AC960220A9
:1050C0000C8300109C83001050830010419000005E
:1050D000B14200109C4203D0607801340028F9D11D
:1050E0006346E01A0C908020C00084460840804649
:1050F0006046014204D00B980C9C844200D90C906D
:105100000220844608400A906046084200D189E1A6
:10511000101E00D170E14246002A00D11BE10B9A1B
:105120005B1B9046A84444462A00B8469946574619
:10513000B246099E09E05B463900551CB0474B4614
:10514000585D002800D12CE12A009442F3D1564644
:105150002500BA4647460A9B002B00D04CE1129B23
:10516000741C0A932BE6002293009B185B00013409
:105170001A182078303A0300303B092BF4D9260066
:105180000B9242E60A9B023604CBD043C017024082
:105190000B9230780A9338E61A78002AA3D00B983D
:1051A000441E82E7102308008027984311331843D8
:1051B0000B00FF003B40394200D14DE70823059327
:1051C0000B9B2A00049310230393002302930C9B50
:1051D0000690019316AB009351465B460998FFF782
:1051E000B1F843460500741C0A93E8E5622800D133
:1051F000A6E1582800D1B1E180230A00DB001A4063
:105200009046194200D189E1112399438C468023AD
:1052100062469B001A40100062461A4200D023E109
:10522000802364465B001C401A4200D032E2634691
:105230005B0600D56BE163460A991B0600D4DBE2EE
:1052400008C91BB2DA179818504080B20A91DA0FD9
:105250000C92002B00D118E280460EAA91461F2323
:105260004B441395E14645461297B0461E0001E0B7
:10527000202C0FD028000A2100F0ACFB0134371994
:105280003031397028000A2100F0A4FB2F000500FE
:10529000092FEDD84646CC46129F139D63460693D0
:1052A0000B9B059704930A2303930C9B029316AB65
:1052B0002A000194009351465B460998FFF742F893
:1052C000741C05007BE5202319436CE680231B0139
:1052D000194338E6782800D07CE180230A00DB00FF
:1052E0001A409146194200D1A5E20D2399430800C6
:1052F00003330C93802302009B001A40904618420F
:1053000000D078E1802304005B001C40184200D0EC
:1053100007E2430600D453E2FF210A9B04CB0A4074
:1053200090460A934346002B00D026E11033984361
:105330004B46002B00D120E100240B9B06900493E8
:105340000C9B059703930023B0E780231B011943AF
:1053500020231943F7E55B1B99460C9B099C984653
:105360005B46B3465646BA461F002A003B00310052
:10537000A0474B460135585D0028F6D143460C93B3
:105380003B005746B2465E469B46E4E6C023B078F3
:10539000194302365AE5C0239B00B0781943023600
:1053A00054E55646BA464746D5E6012F00D832E2C4
:1053B0006B1E9846B8442C00A9464546B846574649
:1053C000B246099E22005B46013439002020B047D6
:1053D000AC42F7D10A9B564601CBBA46474698469F
:1053E00022005B46099C5146C0B2A0474D46434649
:1053F000ED190A93741CE2E40C9BA8469F4200D866
:10540000ADE64446B04656467D19099FED1A220086
:105410005B46013431002020B847AC42F7D1B24698
:1054200046469CE60C98874200D8F0E142469846F2
:105430007919B9465746B246099E0C1A0C922A00B1
:105440005B46013539002020B047A542F7D15646CA
:10545000BA464F4643460C9A90467A1C0C921A78EC
:10546000101E00D057E67AE60822072191460A9BD3
:1054700007338B4399444A460ACB0C000A921C43DB
:10548000DA0F002C4ED0D817040010904C40119029
:105490000E94109811990C005C400F940E9B0F9C79
:1054A0001B1A8C410E930F940EA988461F230024CB
:1054B00043441297B046270013951E000E9C0F9D83
:1054C000E1460C9201E0202F10D0200029000A2292
:1054D000002300F0BDFA013730322B00F2550D00E9
:1054E00022000400002BEED1092AECD84646CC4617
:1054F0000E940F950C9A3C00139D129F63460693E1
:105500000B9B059704930A2302920393CFE6FF2394
:105510000A9904C9134018000A9198E61023994388
:105520008C4674E643460024002BE7D10023002478
:105530000E930F94B8E743464D460A93741C3EE41D
:1055400080230A00DB001A409146194200D140E155
:105550000D2399430B3B08000C93CBE680230A00F4
:10556000DB001A409146194200D162E10D23202050
:105570009943033308430C93BCE66123810600D5AD
:1055800041230EA91F228C46DBB262440A3B1397CB
:105590001495814645460C9FB0461293160008E0CC
:1055A0003033DBB201343355BD420ED3202C0CD046
:1055B00005003900280000F00DFACBB20929EFD917
:1055C000129A94466344DBB2ECE746464846139F82
:1055D000149DB2E66F2800D03CE10C2308009843EC
:1055E00080230A00DB001A409146194200D02AE1CC
:1055F00008230C937EE60A99FA3BFF3B0731994357
:1056000001339C468C4463464A680A930B68904673
:105610009C461343191E06D14B4610310024884383
:10562000002B00D089E66121830600D541210EAA16
:1056300091461F234B449946C9B20C9B0A391397D4
:105640001495159645464E46002467469846814671
:1056500012910CE03032D2B2002301343255AB4209
:1056600000D1BCE0202C00D1BCE007000D00424678
:1056700000233800290000F0EBF9D2B2092AE9D959
:10568000129B9C466244D2B2E6E74346002B00D010
:1056900004E6E2E50A9C08CCDA0F1392002B00D155
:1056A000A5E0D9175B184B4098460EAA91461F23D8
:1056B0004B440C95A14645461296E04606001C0058
:1056C0000A9701E0202E0FD028000A2100F082F96D
:1056D0000136A7193031397028000A2100F07AF913
:1056E0002F000500092FEDD8C4464C4630000A9F14
:1056F0000C9D129E634606930B9B2A0004930A237B
:105700000393139B0190029316AB009351465B46A3
:1057100009980597FEF716FE0A940500741CFFF71A
:105720004EFB0A9B10CB1493002C04D110239843FA
:105730004B46002B2CD16123810600D541230EA9B5
:105740001F228C46DBB262440A3B129713958146B6
:1057500045460C9FB0460A93160008E03033DBB292
:1057600001357355BC420ED3202D0CD004003900F6
:10577000200000F02FF9CBB20929EFD90A9A9446FC
:105780006344DBB2ECE748464646129FA846139DA9
:105790000B9B2A0004930C9B069003930023029317
:1057A0004346019316AB009351465B460998059713
:1057B000FEF7C8FD149B05000A93741CFFF7FFFA5F
:1057C00003061FD50A9B02CB09040A0C90460A93D4
:1057D000A8E50C2399430A3B08000C938AE5B845D9
:1057E00000D83FE74846139F149D159EA5E5434604
:1057F000002B00D07EE758E708C9DA179818504008
:105800000A9124E50A9B04CB90460A938AE501009D
:1058100001310C9124E60A9F6C1C01CF2A005B46E3
:10582000099D5146C0B2A84725000A97741CFFF78E
:10583000C6FA202319430C239943002399461033B9
:1058400008000C9356E508238C460C930D23604604
:1058500098434FE510230A009A439446692808D1DB
:1058600080230A00DB001A409046194200D1CEE4A2
:10587000CAE41C230800984380230A00DB001A4076
:105880009146194202D10A230C9333E50A230C9363
:10589000DCE7C0460EB4012230B584B007AC08CCBA
:1058A000064D01000094280052420394FFF760FA6D
:1058B00004B030BC08BC03B01847C046A942001071
:1058C00000B585B0039101210290009303481300B5
:1058D0004A4202A9FFF74CFA05B000BD4945001045
:1058E00010B5094A0300146884B0002C08D00122C6
:1058F00000910648524203A9A047012004B010BD00
:1059000001F0AEF80020F9E7AC960220394500100E
:1059100001480421014B184730DE00204159001096
:10592000142310B50100188804331B88984710BD54
:10593000162310B50100188802331B88984710BD44
:10594000F8B54746CE4680B50F1E19D014239946A8
:10595000043304000025012698464B461888434628
:1059600021681B88984701C4431E98410135404275
:105970000640AF42F1D13000C0BCB946B046F8BDD8
:105980000126F8E7124A936F9B0815D29066D166FC
:10599000002905D0FFE7FFE7FFE7516F106F704761
:1059A00004B580210906C2175140002800D0C84321
:1059B00001F012FC002104BDF0B5146E556E576F56
:1059C000166FFFF7E3FF1466556657671667F0BD5D
:1059D000000000D0114A936F9B0813D210665166E5
:1059E000002905D0FFE7FFE7FFE7516F106F704711
:1059F00004B5002801D00020C04301F0EDFB0021D8
:105A000004BDC046F0B5146E556E576F166FFFF7A4
:105A1000E5FF1466556657671667F0BD000000D0B5
:105A200094464A4A926F9208624601D228E0C046E4
:105A3000F0B5464E346E756E776F366F00F020F815
:105A40009446424A14665566576716676246F0BD2B
:105A500094463E4A926F9208624601D254E0C04694
:105A6000F0B53A4E346E756E776F366F00F04CF8C5
:105A70009446364A14665566576716676246F0BD07
:105A8000002B24DB11D000293EDA00B5C943404287
:105A900000D1013100F038F8C943404200D1013152
:105AA000DB43524200D1013300BD002AEBD1002874
:105AB00001D1002905D00020C90FC90701D1C04379
:105AC000410800B501F080FB0022002300BD00B5B5
:105AD00000290ADBDB43524200D1013300F014F805
:105AE000C943404200D1013100BDC943404200D109
:105AF0000131DB43524200D1013300F005F8DB43B2
:105B0000524200D1013300BD002923D1002B18D10E
:105B1000002A0CD0BC460D4F38667A66002100235F
:105B2000FFE7FFE7FFE77A6F386F674670470028A7
:105B300001D00748010000B501F046FB0022002318
:105B400000BD02000B00002000217047000000D0C3
:105B5000FFFFFFFF002B00D0BFE0130C28D1002A6D
:105B6000E7D080B4114F39667A66FFE7FFE730B4BB
:105B7000040C7B6F396F1B0423433B667A66FFE797
:105B8000FFE7FFE7C04684B27B6F3D6F1B042343F2
:105B90003B667A66FFE7FFE7C04600232C042D0C26
:105BA0007A6F386F00196941B0BC7047000000D0AF
:105BB000F0B594460025140E01D112020835140FD9
:105BC00001D112010435940F01D192000235D40F96
:105BD00001D152000135D40B0134254F7C66254C90
:105BE0003C660E0C93B2FFE7FFE7FFE73C6F6643AE
:105BF000360C7703BE467343DF0B5B04C01AB94112
:105C0000130C7343DB18C91ACE086643360CB6442E
:105C100093B273431F0F1B01C01AB941130C734396
:105C20001F0B1B05C01AB941860D8F023E43664308
:105C3000360C092D24DB520A7243801A7703460A78
:105C40006643360C16235B1BDE40DF40BF196446FB
:105C50006643821B7046043506330100D940A840D4
:105C6000C01900D30131A24206D20023F0BD0000CA
:105C7000000000D0FFFFFFFF121B0130F3D3F1E75C
:105C800009277F1BFE406446A2B27243801A00D2ED
:105C90000139220C7243130C1204821A99410B0031
:105CA0007046043513370100F940A840801900D32D
:105CB0000131002B02D1A2420AD2F0BD013000D343
:105CC0000131121BFAD2013BF8D1A24200D2F0BD41
:105CD000013000D30131121BF7E7F0B51C0C00D0E6
:105CE00080E00CB400251C0A04D11B02160E3343BD
:105CF000120208351C0B04D11B01160F334312018D
:105D000004359C0B04D19B00960F3343920002355F
:105D1000DC0B02D192185B4101351C0097186441DD
:105D20000134464F7C66464C3C660E0CFFE7FFE7AD
:105D3000FFE7C0463C6F6643360C7703BE4697B21A
:105D40007743C01B00D20139C01B00D201399FB27A
:105D50007743C91BC91B170C77437E04FF0B801BBD
:105D6000B941CE086643360C0C2D33DBB644120B1A
:105D70001F053A431B0B97B27743C01B00D2013972
:105D80009FB27743C91B170C77433E043F0C801B1F
:105D9000B941860D8F023E43664329277F1BFE4093
:105DA0000C3D7746AF40BF1930BCA2B2ABB27243D4
:105DB0007343801A9941220C7243130C1204801A07
:105DC000994102000B000137001BA941F9D2781E4E
:105DD0000021F0BD0C277F1BFE4077467F0BAF40B4
:105DE000FF19E0E700245D1C07D0144F7D6639667B
:105DF000FFE7FFE7FFE7FFE73C6F95B29EB2654321
:105E00006643401BB141150C1E0C654366433604C6
:105E10002F0C3E432D04401BB141994204D2020095
:105E20000B0020000021F0BD01D19042F7D3801A71
:105E3000994101349942F2D3F6E70000000000D006
:105E4000FFFFFFFF48404140484018B41B4B5B68D0
:105E5000FC46019308BD04DFEF60001018B4174B37
:105E60001B68FC46019308BD00DFF96000109446F2
:105E7000134A926F920809D2624618B40F4BDB683E
:105E8000FC46019308BD0CDFB16300100C4AF0B56D
:105E9000146E556E576F166F6246FFF7EEFF084A95
:105EA0001466556657671667F0BD18B4034B9B68B8
:105EB000FC46019308BD08DF55620010E8E30020AE
:105EC000000000D0FFB550404240504059404B4088
:105ED000594000E0FFB5154F4C00640D03D0BC42A3
:105EE00004D10C0314D80020090D09055C00640DD1
:105EF00003D0BC4204D11C030AD800221B0D1B0591
:105F000001264B4009D44B4003D58B4200D182423D
:105F1000FFBD9942FCD19042FFBD0B43DB18034308
:105F20001343F5D0C9434918FFBD0000FF07000027
:105F300000B5FFF7CFFF804100BDC04600B5FFF7B9
:105F4000C1FF01D9002000BD012000BD00B5FFF751
:105F5000B9FF804100BD012040054A00121804D855
:105F60005A00121801D80020704701207047002005
:105F7000704700000021002805D17047C117484034
:105F8000401AFAD0C90713B5064B1B6898470CBCDA
:105F9000441CA2401005120B0349091B09051943B3
:105FA000114310BDF49602201F04000010B54C00F0
:105FB000620D8023D218DB00D21A5B057E2A10DD29
:105FC0009E3A13DACC170903490819435242D140CB
:105FD000640001341532202A05DAD04008436043BA
:105FE00010BD002010BD0846604310BDC80FC0188A
:105FF000013810BD18B4044B5B6AFC46019308BD20
:1060000024DF616500100000E8E3002018B4044BB1
:10601000DB6FFC46019308BD7CDFE16500100000EA
:10602000E8E30020132370B51D78012D15D010DD95
:106030001D48FFF77DFC1D4C01008022200000F070
:106040002DFC022D2DD01A48FFF76AFC194B186061
:1060500070BD194B154CA364F5E7174B134C236027
:106060006360A360E36023616361A361E361236212
:106070006362A362E36223636363A363E3632364F2
:106080006364A364E36423656365A365E3652366D2
:106090006366A366E36623676367A367E367A36436
:1060A000D1E7054BA364CEE753440000E8E30020AA
:1060B0004C330000F4960220BD60001007B5604626
:1060C00001880A0A0230DF2AFAD1C9B2820804D351
:1060D000028840880004104300E00068014A5050E4
:1060E000039007BDE8E300200FB403BC0CBCF0B57F
:1060F0000124E407634000E0F0B50C0DCF0F661EED
:106100003605891B640503D3C943404200D30131DE
:10611000640D03D0661CF60A07D0E41B00207F0044
:10612000791C89078912803C24031D0DDF0F6E1E28
:1061300036059B1B6D0503D3DB43524200D301336D
:106140006D0D03D06E1CF60A07D0ED1B00227F00F8
:106150007B1C9B079B12803D2D032F1B661B58D475
:10616000A446202E46DA20371400BC401D00BD4056
:10617000F24033412A4380185941CB0F05D0C9431F
:10618000C043002264425041514162464D0D28D126
:106190000D0D07D100281FD0241940414941013A73
:1061A0000D0DF9D0640006D3013000D30131002C6D
:1061B00001D140084000013A0BD4941CE40A04D1F8
:1061C00012051144DB071944F0BDD907204B1943D0
:1061D00000E0D9070020F0BD0029DDD1002CDBD183
:1061E000F0BD0132C6074008CD0728434908002EFC
:1061F000E1D0D9E73C2E29DA203E40371400BC40DC
:1062000000D00124F24014431A00BB401C43D317B2
:10621000ACE7AC46202F08DA20360400B4400D006D
:10622000B540F84039412843A5E73C2F0CDA203F20
:1062300040360400B44000D00124F8400443080074
:10624000B1400C43C117EAE710001900002494E79D
:106250000000F07FF0B50C0D661E3605891BE60ABE
:106260006405640D02D0651CED0A04D000200121F4
:106270000905803C2403A4461C0D671E3F05DB1B5B
:10628000E70A6405640D02D0651CED0A04D0002203
:1062900001231B05803C24037740644497B484B2F7
:1062A00096B27443070C7E43150C6F4380B268436B
:1062B000361802D3012000043F183004350C0019B1
:1062C0007D41844688B29AB250430C0C62431F0C45
:1062D0007C438EB27E43921902D301263604A41960
:1062E0001604170C3618674101BC81B29AB25143AB
:1062F000040C62431B0C5C4380B25843121802D357
:106300000120000424181004130C401863412D18B8
:106310005E410020474106BC88B293B258430C0C42
:106320006343120C544389B251435B1802D30121D9
:106330000904641819041A0C091862416D185641B1
:106340000020474118BCF902720D1143F0026A0D9A
:106350001043ED020A0D03D16D1940414941013B43
:10636000124E9B1B7600B3420ED26D0007D3013054
:10637000002671416646354301D1400840001B05A7
:10638000C918E4072144F0BD0BDA013306D101300E
:1063900004D101314F0D01D04908F2E7E107002097
:1063A000F0BD013631050020EBE70000FF030000DF
:1063B000F0B51C0D671E3F05DB1BE70A6405640D85
:1063C00002D0661CF60A04D0002201231B05803C83
:1063D0002403D0252D060026F6432E661E096E6680
:1063E000CE0FF619B44649004F0D02D07E1CF60AB6
:1063F00003D000200021403F3F033E1BB600B444C1
:10640000013F7F05C91B49082E6F013676089C02A3
:10641000950D25437543ED137543AD1301356D108F
:10642000F603761B0CB4CC02450D2C43A2B2B3B2DA
:106430005A43270C7B43350C6F43A4B26C431B19A2
:1064400002D3012424043F191C041D0CA4187D410F
:1064500024196D41009A91B2ACB26143170C7C4390
:106460002B0C5F4392B25A43A41802D301221204A8
:10647000BF182204230C52187B41019C6C431B194A
:10648000520ED9010A434401A01A81B2B2B251435B
:1064900003145A43360C734387B27743D617D21985
:1064A00000277E4136049B191704160C7F185E41A5
:1064B0007316ED18F301002680337541A90F06D13C
:1064C0006400690AE8055B0A184309D22FE0042238
:1064D000944480337541A90AA8059B0A184326D322
:1064E000404149412404009A019B0D005543641B1F
:1064F0004343E41A95B286B27543170C7E43030CEE
:106500005F4392B25A43B61802D301221204BF1855
:106510003204330C52197B4152429C41002C02D46C
:106520000022013051414008CA071043490802B017
:106530006246D7079210084BD218084B9A4203D2F2
:1065400012058918C919F0BD0020002A01DC3900A4
:10655000F0BD01331905F5E7FD030000FE0700005B
:10656000002200B5203200F004F8080000BD000051
:1065700000220B150AD410B5944600F05FF81414ED
:10658000013400DA0021CB17144C204700200021F1
:1065900070476244343A0CD40C2A07DA0400914064
:1065A000904052422032D440214310BDD843D943B9
:1065B00010BD203207D40C46944052422032114183
:1065C000D040204310BD0800C917203203D45242E6
:1065D0002032104110BD1800190010BD9365001045
:1065E0004A00520D144BD21A13DDFF2A1EDAD205CF
:1065F000CB0FDB071A43C300400F0903490A0843C6
:1066000010435B0001D301D0013070474308FBD237
:10661000704702D0C80FC00770470A031213013237
:10662000F8D1420F072AF5D1012200E0FF22C80F5E
:1066300000028018C0057047800300000A0DCC0FCF
:10664000531E1B05C91A520503D3C943404200D348
:106650000131520D03D0531CDB0A07D0121B00205E
:106660006400611C89078912803A1203014BD21A17
:1066700070470000FF03000051434343C9188C4694
:10668000110C83B24B4310B4040C614392B280B23C
:10669000504362431C041B0C001910BC59411304E5
:1066A000120CC018514161447047000048404140FD
:1066B00048400E4B5B6818470C4B1B6818470C4A48
:1066C000936F9B0802D2094BDB681847F0B5146E34
:1066D000556E576F166FFFF7F6FF054A146655663D
:1066E00057671667F0BD014B9B681847E8E4002028
:1066F000000000D007B548404140484001E0C04696
:1067000007B54200120E03D0FF2A03D1420218D867
:10671000C00DC0054A00120E03D0FF2A03D14A0261
:106720000FD8C90DC9050122414005D4414001D50A
:10673000814207BD884207BD0143491801D0C043CB
:10674000001807BD00B5FFF7DBFF804100BDC04664
:10675000491A002808D1084670470000C10FC90730
:1067600000D54042002817D0F44603B40B4B1B68F9
:10677000984706BC81409E384042803107D20B06C4
:1067800007D04900490AC00510430843604701305B
:10679000F8E7490A8902F5E770470000F4960220FD
:1067A000014B5B6A18470000E8E40020034BDB6FF5
:1067B000FC4618477CDF516800100000E8E4002028
:1067C000132310B512481C78FFF7B2F80100012C12
:1067D0000AD003DD80220F4800F060F80E48FFF772
:1067E0009FF80E4B186010BD0A4C5422200000F098
:1067F00055F80B4B6365A365E36523666366A36683
:10680000E36623676367A367E3672362E361E5E702
:1068100053460000E8E400204C330000F4960220C8
:106820002568001007B5604601880A0A0230DF2A91
:10683000FAD1C9B2820804D3028840880004104308
:1068400000E00068014A5050039007BDE8E40020D2
:10685000C30FDB0741000A0E07D0FF2A08D0090941
:10686000054A8918194340077047190000207047EE
:106870000249C918FAE70000000000380000F07F64
:1068800001480421014B184740DE00204159001007
:10689000014B1B681847000040DE0020014B5B687D
:1068A0001847000040DE0020F0B546464F46D64669
:1068B000C0B5437D80460E001700002B4BD0002A48
:1068C00032DD274B01259A464B1E002400209946B5
:1068D00007E0335D0A2B2CD02B0001340135BB427D
:1068E00013DA002CF5D133780A2BF5D143461B7D02
:1068F000002BF1D14346504602211B6898472800DF
:106900002B0001340135BB42EBDB874204DD4346FB
:10691000391A1B6830189847F619013E33780D3B39
:106920005A42534142461375E0BCBA46B146A846A6
:10693000F0BD4B461B5D0D2BCED0A042DADA4346AC
:10694000211A1B68301898474346504602211B689D
:1069500098472800D4E70368110030009847E3E720
:1069600078850010F0B5C6460B6806000C0000B52F
:10697000802B06D05A1C2260E418267180BCB846D1
:10698000F0BD0F4B1D68002D16D00B1D98460D4F06
:1069900002E02D69002D0FD02B68002BF9D03B6849
:1069A000002B01D0AB42F4D1280041462268FFF70A
:1069B0007BFF2D69002DEFD101220023DBE7C046CC
:1069C0009C960220A0960220F0B5CE46474680B5A0
:1069D00083B06B460600DD1D2870FCF711FE002316
:1069E0001A4A12184B41802109068B4202D3012218
:1069F000174B524217490800884600F0F5FB164B2A
:106A000081461C68002C14D0144F02E02469002C2D
:106A10000FD02368002BF9D03B68002B01D0A34294
:106A2000F4D1200001222900FFF73EFF2469002C49
:106A3000EFD14B46002B05D1300003B0C0BCB946A6
:106A4000B046F0BD404600F0B7FBF5E740420F000E
:106A5000FFFFFF7F98E200209C960220A096022074
:106A6000F0B5DE4657464E464546E0B585B00700D0
:106A700000F03EFB0600FCF7C3FD00232B4A121872
:106A80004B41802109068B4202D30122284B5242FE
:106A9000284908008B4600F0A7FB274B01901C6893
:106AA0009A46002C3BD0254B984602ABDD1D0A23AD
:106AB000994602E02469002C17D02368002BF9D0F6
:106AC00043461B68002B01D0A342F3D120003200C3
:106AD0003900FFF7E9FE4B462000012229002B7008
:106AE000FFF7E2FE2469002CE7D1019B002B18D1AF
:106AF00053461C68002C06D06368002B0BD09847C7
:106B00002469002CF8D1300005B0F0BCBB46B24679
:106B1000A946A046F0BD2469002CEDD1F3E700287A
:106B2000F1D0584600F048FBE2E7C04640420F0073
:106B3000FFFFFF7F98E200209C960220A096022093
:106B40000A4A1368002B05D10CE01A001B691032A9
:106B5000002B07D09842F8D1002902D103691360B5
:106B6000016170470029FCD01060FAE79C96022072
:106B7000F0B5CE46474680B5A3B004000D00FCF743
:106B80003FFD0023294A12184B41802109068B4200
:106B900002D30122264B5242264F380000F024FB3C
:106BA00000230600019322002B00234801A9FEF7D1
:106BB00087FE019B8046002B14D1204B1C68002CC3
:106BC00006D06368002B0BD098472469002CF8D1BD
:106BD000002E25D1404623B0C0BCB946B046F0BD1A
:106BE0002469ECE7154B1D689946002D1CD0144C08
:106BF00002E02D69002D0FD02B68002BF9D02368FF
:106C0000002B01D0AB42F4D12800019A02A9FFF772
:106C10004BFE2D69002DEFD14B4601951C68CEE748
:106C2000380000F0C9FAD5E70195D1E740420F00DE
:106C3000FFFFFF7F98E20020656900109C9602200C
:106C4000A09602200FB400B583B004A901C9019138
:106C5000FFF78EFF03B008BC04B0184710B500F072
:106C6000CFF8012010BDC046F0B5002915DD0E4B50
:106C70000D271A680D4B0E4CD3185D426B41451819
:106C800020215B001E5F0478A64207D09369194259
:106C9000FCD101301460A842F5D1F0BD93691942CE
:106CA000FCD11760F2E7C046149702200080FCBFB9
:106CB0001097022030B504000D1E30DD0020102199
:106CC000204B013C1A689369194217D1013093692E
:106CD0001942FCD1136823548542F4D11A4B1B6826
:106CE000002B09D0502338219363536B3432194061
:106CF00080235B011343196028000FE0124B1B68CF
:106D0000002B09D0502338219363536B3432194040
:106D100080235B011A431160002810D030BD0A4B5C
:106D20001B68002B0BD050223821064B1B689A633E
:106D30005A6B3433114080225201134319600320EF
:106D40004042EBE71497022038960220064B10B51C
:106D50001B68002B06D00021044A12689163044A84
:106D60001068984710BDC04638960220149702203C
:106D70003C9602201D4BF0B51A68C64698461C4B3F
:106D80000E00D31859424B411A4F14331C00050012
:106D900000B53B68002807D0002B11D0164B3D6092
:106DA0001E6080BCB846F0BD002BF7D09063002178
:106DB0002000FBF759FC20001049FBF793FDEDE79D
:106DC00020000E49FBF76AFC01212000FBF74CFC78
:106DD0004346502238211B689A635A6B3433114062
:106DE0008022520113431960D8E7C046149702204D
:106DF0000080FCBF389602203C9602204D6D0010AA
:106E00000C4B10B51B780C4B0C4C1B780C4B022117
:106E100000202360FBF742FB02210120FBF73EFB31
:106E2000E12120684902FCF7DFFE01210548FFF758
:106E300087FE10BDF4850010F08500101497022025
:106E40000040034050DE0020F0B5DE4657464E4677
:106E500045468846E0B583B006000524FBF7B2FB43
:106E600043461F791C57314B8246F3185A4253410F
:106E70009B009C462E4A1300934662469B58012273
:106E80009946BA402023013ADB1B002C36DB9C429A
:106E900046DCA2404B46134242D10192002F1CD047
:106EA0004246434652781B7812021A4343469B7867
:106EB00080251B0413434246D07800220006184365
:106EC000AD015300C15AA94200D20919A3181233C7
:106ED0009B0001329951BA42F3D34D46019B624661
:106EE0001D435B4650469D50FBF778FB200003B0E6
:106EF000F0BCBB46B246A946A046F0BD002B0FDB56
:106F00001100484699401C000191014206D1C5E795
:106F1000150049469D401C00294204D0013BF7D290
:106F20000448FDF7A3F90195B8E7C0460000D0AFCB
:106F300008E60020BC850010F0B557464E46454691
:106F4000DE468946E0B583B00CA90D784946490074
:106F500088464944C900461837003400DC37844667
:106F60003868CC3483462068C024CC31A401614405
:106F700021438024A4020C6069424D411E216D42D0
:106F80008D43164901908A465544052B0CD9A02003
:106F90001F214005D836540104430532053B3C60AF
:106FA0000A403560052BF6D852019B061343424632
:106FB0004A44D20062441000DC3213600300D8332C
:106FC0001D605B461360019BCC30036003B0F0BCD6
:106FD000BB46B246A946A046F0BDC0469FE00000B1
:106FE000F0B501258D400468AC430460002B2ED021
:106FF0004D006C18E400041926001F68C83637607D
:107000005F68DC3477609F68DB68B76023606B186B
:10701000DB001D008024D035451964012C438025F8
:107020002D06256025600125124C2E008C408460C1
:107030000C1DA640802408318D401F21A40104436B
:10704000C0180A40D830266025600260F0BD4D00AF
:107050006C18E400041926008027C8367F023760C8
:10706000F8277F027760C027DC343F03B7602360D6
:10707000CDE7C0460101010100B50A4B87B0186891
:1070800002A900F07DF8431C0AD0039B1800029B64
:107090009C46049B60449C460193059B6044C01839
:1070A00007B000BD68DE00200022034B1B68A83338
:1070B00018605A607047C04668DE0020094B10B562
:1070C0001C68094AA83420686168084BFFF7D4FAA5
:1070D0000122002380185941206061604800400867
:1070E00010BDC04668DE00202D7F954C2DF4515810
:1070F00010B583070AD00300032102E001330B42DD
:1071000005D01A78002AF9D1181A10BD03001968A1
:107110000C4A0D4C8A188A4322420FD15968094AF9
:1071200004338A188A43224208D15968054A043335
:107130008A188A432242F1D000E001331A78002AEB
:10714000FBD1E1E7FFFEFEFE8080808010B50B4B97
:1071500084B0040000226946186800F017F800287F
:1071600007DB00980199002C01D02060616004B019
:1071700010BD01204042C117F5E7C04668DE00207F
:1071800010B50800FDF75CF810BDC046002370B5CF
:10719000074D0400080011002B60FDF739F8431C6F
:1071A00000D070BD2B68002BFBD02360F9E7C046F0
:1071B00004E60020F8B5C04601B40248844601BC8C
:1071C000604700BF5D01002001B40248844601BC55
:1071D000604700BF8501002001B40248844601BC1D
:1071E000604700BF8501002001B40248844601BC0D
:0871F000604700BFC100002050
:1071F800537061636520496E7661646572732074AB
:107208006573740D000000004261736564206F6E41
:1072180020416C616E205265656473207069636FEC
:107228002D636F6D706F73697465206C696272612C
:1072380072790D005772697474656E20696E203218
:10724800303233206279206D75656C6C65725F6DC4
:10725800696E6B690D0000005741524E494E473A1E
:107268002050494F206461746120534D20636C6F36
:10727800636B2064697669646572202876616C7531
:107288006520256629206C657373207468616E20FB
:10729800310D0A004461746120636C6F636B64692B
:1072A800762025660D0A000053796E6320636C6FA3
:1072B800636B6469762025660D0A0000CC720010A5
:1072C80005FF000000E041A0C02001648300000029
:1072D800E072001019FF0000630023F0041D24FE73
:1072E80042A0441E24ED2911470D6C0022F00D1C0C
:1072F80023FD4AB042A04E1E30E142BE341E510169
:1073080027A142B200DD201C5501000044617461D0
:1073180020756E64657272756E210D00496E766116
:107328006C6964206A757374696669636174696FEE
:107338006E0D0000FFFFFFFFFFFFFFFFFFFFFFFFD6
:10734800FFFFFFFFFFFFFFFF01061860800106181F
:1073580060800106186080010618608079E69967E8
:107368009E79E699679E79E699679E79E699679E80
:1073780079E699679E79E699679E79E699679E7995
:10738800E699679E79E699679E79E699679E79E618
:1073980099679E79E699679E79E699679E79E69955
:1073A800679E79E699679E79E699679E79E6996777
:1073B8009E79E699679E79E699679E79E699679E30
:1073C80079E699679E79E699679E79E699679E7945
:1073D800E699679E79E699679E79E699679E79E6C8
:1073E80099679E79E699679E79E699679E79E69905
:1073F800679E79E699679E79E699679E0106186007
:1074080080010618608001061860800106186080F7
:10741800FFFFFFFFFFFFFFFFFFFFFFFFFFFFFFFF74
:10742800FFFFFFFFFFFFFFFFFFFFFFFFFFFFFFFF64
:10743800FFFFFFFFFFFFFFFF01061860800106182E
:1074480060800106186080010618608079E69967F7
:107458009E79E699679E79E699679E79E699679E8F
:1074680079E699679E79E699679E79E699679E79A4
:10747800E699679E79E699679E79E699679E79E627
:1074880099679E79E699679E79E699679E79E69964
:10749800679E79E699679E79E699679E79E6996786
:1074A8009E79E699679E79E699679E79E699679E3F
:1074B80079E699679E79E699679E79E699679E7954
:1074C800E699679E79E699679E79E699679E79E6D7
:1074D80099679E79E699679E79E699679E79E69914
:1074E800679E79E699679E79E699679E0106186016
:1074F8008001061860800106186080010618608007
:10750800FFFFFFFFFFFFFFFFFFFFFFFFFFFFFFFF83
:10751800FFFFFFFFFFFFFFFFFFFFFFFFFFFFFFFF73
:10752800FFFFFFFFFFFFFFFFFF3F3FF9CCCFCF7CFF
:10753800FCF39F9FFFFFFFFFFFFFFFCFFF3F3FF9D8
:10754800CC034F3EF9F38F1FFFFCFFFFFFFFFFCF78
:10755800FF3F3F7980037F3EF9F3CF3F9FE4F3FF7E
:10756800FFFFFFE7FF3FFFFFCCCB3F7FFCFFE77F3D
:107578003EF0F3FFFFFFFFE7FF3FFFFFCC033F3F76
:10758800F4FFE77F7EF8C0FF1FFEFFF3FF3FFF7F9A
:10759800804F9F9FF9FFE77F3EF0C0FFFFFFFFF39B
:1075A800FFFFFFFFCC039F9CF1FFE77F9EE4F3CF33
:1075B800FFFFFFF9FF3FFFFFCC03CF3CE4FFCF3FC6
:1075C800FFFCF3CFFFFFFCF9FF3FFFFFFFCFFFFFFB
:1075D800FFFF8F1FFFFFFFC7FFFFFCFCFFFFFFFF41
:1075E800FFFFFFFFFFFF9F9FFFFFFFE7FFFFFFFC7E
:1075F800FFFFFFFFFFFFFFFFFFFFFFFFFFFFFFFF93
:10760800FFFFFFFFFFFFFFFFFFFFFFFFFFFFFFFF82
:10761800FFFFFFFFFFFFFFFF873F7FF8C08F0F7C53
:1076280078C0871FFEFFFFFFFFFFFFE13B1F3FF30F
:10763800CE87CF3FFFCF3BEFFCFCF3FFFFFFFFCC34
:107648003B0FBFF3CF93CF3FFFC73BEFFCFCF33FAC
:10765800FF3FFFCE3B3FFFF3E7990F3EF8E787EF89
:10766800FCFFFFCF1FFEFCC73B3FFFF9E799FF3C3C
:10767800F7F33B1FFCFFFFF3FFFFF3E33B3F7FFC08
:10768800CF01FF3CF7F33BFFFCFCF3F31FFEF3F3E2
:107698003B3F3FFFCE9FEF3CF7F93BFFFCFCF3CFAE
:1076A800FFFFFCFF870F3CF0E19F1F7EF8F9871F63
:1076B800FEFFF13FFF3FFFF3FFFFFFFFFFFFFFFF6D
:1076C800FFFFFFFFFFFFF9FFFFFFFFF3FFFFFFFFD4
:1076D800FFFFFFFFFFFFFFFFFFFFFFFFFFFFFFFFB2
:1076E800FFFFFFFFFFFFFFFFFFFFFFFFFFFFFFFFA2
:1076F800FFFFFFFFFFFFFFFFFFFFFFFFFFFFFFFF92
:10770800FFFFFFFFFFFFFFFF873F3FF8E1830F3CCD
:10771800F0E1331F3EF0CCF3E739F3E17B1F3EF392
:10772800C013CF3CF3CC333FFFF3E4F3C738F3CCBB
:10773800CDCE3C73CE33CF3FFFCC333FFFF3E4F3E2
:107748000738F2CCB5CE3C78FE330F3EF8FC033F49
:10775800FFF3F0F32739F0CCB50E3C73FE33CF3F7F
:10776800FFC4333FFFF3E4F3E739F1CC4DCF3C736B
:10777800CE33CF3FFFCC333F3FF3E4F3E739F3CCCD
:10778800FBCF3CF3C013CF3CFFCC333F3FF3CCF3EC
:10779800E739F3CC07CE3CF8E1830F3CFFE1331F18
:1077A8007EF8CC03E739F3E1FFFFFFFFFFFFFFFFA0
:1077B800FFFFFFFFFFFFFFFFFFFFFFFFFFFFFFFFD1
:1077C800FFFFFFFFFFFFFFFFFFFFFFFFFFFFFFFFC1
:1077D800FFFFFFFFFFFFFFFFFFFFFFFFFFFFFFFFB1
:1077E800FFFFFFFFFFFFFFFFFFFFFFFFFFFFFFFFA1
:1077F800FFFFFFFFFFFFFFFF831F3EF8E103CF3CC2
:10780800739E39CF3CF0F1F31FFFFCFF33CF3CF3FD
:10781800DCCFCF3C739E93CFFCF3F9F33F7FF8FFA7
:1078280033CF3CF3FCCFCF3C739E931FFEF9F9E7AF
:107838003F3FF3FF33CF3CF3E1CFCF3C7392C71FF9
:10784800FEFCF9E73FFFFFFF83CF3CF8CFCFCF3CEB
:107858007392C73F7FFEF9CF3FFFFFFFF3CF3CF99D
:10786800CFCFCF3C7380933F3FFFF9CF3FFFFFFF60
:10787800F3CF3CF3CCCFCF7C7880933F3FF0F99F98
:107888003FFFFFFFF31F3EF3E1CF1FFEFCCC393F64
:107898003FF0F99F3FFFFFFFFF7FFEFFFFFFFFFF66
:1078A800FFFFFFFFFFFFF93F3FFFFFFFFFFFFCFF69
:1078B800FFFFFFFFFFFFFFFFFFFFF13F1FFFFFC0BD
:1078C800FFFFFFFFFFFFFFFFFFFFFFFFFFFFFFFFC0
:1078D800FFFFFFC0FFFFFFFFFFFFFFFFFFFFFF3FAF
:1078E800FFF9FFFFFFFFFFFFE7FF3FFFFF3FFFFF3E
:1078F800F8FFF33FFFF9FCC7FFFFFFFFCFFF3FFF94
:10790800FF3FFF7FF8FFF3FFFFFFFCCFFFFFFFFF05
:107918009F0F3FFFE13F1F7EFEC0831F7FF8CCCF44
:10792800073CF8E1FF7F3EF8CC07CF7C7EE6333F8B
:10793800FFF9E4CF2739F3CCFF0F3EF3FC33CF3CFC
:107948007CE6333FFFF9F0CF2739F3CCFF673EF3EE
:10795800FC330F7CFEF0333FFFF9F0CF2739F3CC2F
:10796800FF673EF3CC33CF7F7EFC333FFFF9E4CF94
:107978002739F3CCFF8F3CF8E1071F7E7EF0331FD9
:10798800FEF9CC872739F3E1FFFFFFFFFFFFFFFF79
:107998007FE6FFFF7FF8FFFFFFFFFFFFFFFFFFFF0F
:1079A800FFFFFFFFFFF0FFFF7FFCFFFFFFFFFFFF71
:1079B800FFFFFFFFFFFFFFFFFFFFFFFFFFFFFFFFCF
:1079C800FFFFFFFFFFFFFFFFFFFFFFFFFFFFFFFFBF
:1079D800FFFFFFFFFFFFFFFFFFFFFFFFFFE7FFFFC7
:1079E800FFFFFFFFFFFFE7CF9FFF7F80FFFFFFFF46
:1079F800FFE7FFFFFFFFFFFFFFFFF3CF3FFF7F9E84
:107A0800831F7CF8C1E7CF3C739E39CF3CF8F3CF96
:107A18003FFF7F9E33CF3CF6FC87CF3C739E93CFCE
:107A2800FCF9F3CF3F3F669E33CF3CFFE0E7CF3C06
:107A38007392C7CFFCFCF9CF7F9E649E33CF3CFF87
:107A4800C7E7CF3C7392C7CF7CFEF9CF7F9E719E6C
:107A580033CF3CFFC787CF7C788093CF3CFFF3CFF1
:107A68003FFF7F9E831F3CFFE08F1FFCFCCC391F2C
:107A78003CF8F3CF3FFF7F9EF3FFFCFFFFFFFFFFC4
:107A8800FFFFFFFFFCFFF3CF3FFF7F9EF3FFFCFFED
:107A9800FFFFFFFFFFFFFF1FFEFFE7CF9FFF7F8076
:107AA800FFFFFFFFFFFFFFFFFFFFFFFFFFFFFFFFDE
:107AB800FFFFFFFFFFFFFFFFFFFFFFFFFFFFFFFFCE
:107AC800FFFFFFFFFFFFFFFF010618608001061898
:107AD80060800106186080010618608079E6996761
:107AE8009E79E699679E79E699679E79E699679EF9
:107AF80079E699679E79E699679E79E699679E790E
:107B0800E699679E79E699679E79E699679E79E690
:107B180099679E79E699679E79E699679E79E699CD
:107B2800679E79E699679E79E699679E79E69967EF
:107B38009E79E699679E79E699679E79E699679EA8
:107B480079E699679E79E699679E79E699679E79BD
:107B5800E699679E79E699679E79E699679E79E640
:107B680099679E79E699679E79E699679E79E6997D
:107B7800679E79E699679E79E699679E010618607F
:107B88008001061860800106186080010618608070
:107B9800FFFFFFFFFFFFFFFFFFFFFFFFFFFFFFFFED
:107BA800FFFFFFFFFFFFFFFFFFFFFFFFFFFFFFFFDD
:107BB800FFFFFFFFFFFFFFFF0106186080010618A7
:107BC80060800106186080010618608079E6996770
:107BD8009E79E699679E79E699679E79E699679E08
:107BE80079E699679E79E699679E79E699679E791D
:107BF800E699679E79E699679E79E699679E79E6A0
:107C080099679E79E699679E79E699679E79E699DC
:107C1800679E79E699679E79E699679E79E69967FE
:107C28009E79E699679E79E699679E79E699679EB7
:107C380079E699679E79E699679E79E699679E79CC
:107C4800E699679E79E699679E79E699679E79E64F
:107C580099679E79E699679E79E699679E79E6998C
:107C6800679E79E699679E79E699679E010618608E
:107C7800800106186080010618608001061860807F
:107C8800FFFFFFFFFFFFFFFFFFFFFFFFFFFFFFFFFC
:107C9800FFFFFFFFFFFFFFFFFFFFFFFFFFFFFFFFEC
:107CA800FFFFFFFFFFFFFFFF013EFFFBE3FFCFFCEE
:107CB800FCF301FE1FE0FFFF07F87F80793E7FF0AD
:107CC800C9FDCEFCFCED791E9EE7FFFFE779789EA3
:107CD80079FE3FE0F94B1FFEFCFD79EE9DE799FF29
:107CE800E7B9779E793E9FE5FBB71FFEFCFB793627
:107CF8009BE7CCFFE7596C9E793E9FFDE07B3FFFF9
:107D0800FFF579D69B67E601E6596B9E793E9FFEA3
:107D1800FB7B0FFCFFEB79D69B67E67FE6596C9EF1
:107D2800793E9FE6F8B73FFFFCF779369BE7CC7FB3
:107D3800E6596B9E793E3F60B94B0FFCFCEF79EE3C
:107D48009DE7997FE6B9779E793E7FF0C4FD3EFFB7
:107D5800FCED791E9EE7FFFFE779789E01FE7FFF25
:107D6800FFFFFFFFFCF301FE1FE0FFFF07F87F8026
:107D7800FFFFFFFFFFFFFFFFFFFFFFFFFFFFFFFF0B
:107D8800FFFFFFFFFFFFFFFFFFFFFFFFFFFFFFFFFB
:107D9800FFFFFFFFFFFFFFFFCFFFFFFCE301FE7FB9
:107DA800E0FF017E1FE0FFFBEF1FFFF3B7FFFFFBC4
:107DB800EF79FE3FF4FF793E9FE7FFF9E67BEFF3AB
:107DC800B73FFFFDF779CE3CF4FF797E9F67E67BEE
:107DD800EFBDF7FFCF3FFFFEEF79CE7CF4FF797E52
:107DE8009FE7CCBBEF7EFBF3FF0FFCF8F379CEFCEB
:107DF800F4F3793E9EE799D1479FFDF1FF0FFCFF11
:107E0800FF79CEFCF4F379FE9FE799AFBEFCEAF860
:107E1800FF3FFFFFFF79CEFCF4FF79FE9FE7CCB769
:107E2800DE7BEBDCFF3FFFFFFF792EFAF4FF79FEE4
:107E38009F67E63BEEBDE3CCFF0FFCFFFF79EEFF4B
:107E4800FFFF79FE9FE7FFFDF6DEEFE1FFFFFFFF93
:107E5800FF01EEFFFFFF01FE1FE0FFFFFEF8EFFF4F
:107E6800FFFFFFFFFFFFFFFFFFFFFFFFFFFFFFFF1A
:107E7800FFFFFFFFFFFFFFFFFFFFFFFFFFFFFFFF0A
:107E8800FFFFFFFFFFFFFFFF0106186080010618D4
:107E9800E0FF0106186080010618608079E699679E
:107EA8009E79E699E7FF79E699679E79E699679E54
:107EB80079E699679E79E699E7DE79E699679E798A
:107EC800E699679E79E699679E79E699E7ED79E6FE
:107ED80099679E79E699679E79E699679E79E6990A
:107EE800E7F379E699679E79E699679E79E6996757
:107EF8009E79E699E7F379E699679E79E699679E10
:107F080079E699679E79E699E7ED79E699679E792A
:107F1800E699679E79E699679E79E699E7DE79E6BC
:107F280099679E79E699679E79E699679E79E699B9
:107F3800E7FF79E699679E79E699679E01061860DA
:107F480080010618E0FF01061860800106186080AD
:107F5800FFFFFFFFFFFFFFFFFFFFFFFFFFFFFFFF29
:107F6800FFFFFFFFFFFFFFFFFFFFFFFFFFFFFFFF19
:107F7800FFFFFFFFFFFFFFFF0106186080010618E3
:107F8800E0FF0106186080010618608079E69967AD
:107F98009E79E699E7F379E699679E79E699679E6F
:107FA80079E699679E79E699E7F379E699679E7984
:107FB800E699679E79E699679E79E699E7FF79E6FB
:107FC80099679E79E699679E79E699679E79E69919
:107FD800E7C079E699679E79E699679E79E6996799
:107FE8009E79E699E7FF79E699679E79E699679E13
:107FF80079E699679E79E699E7F379E699679E7934
:10800800E699679E79E699679E79E699E7F379E6B6
:1080180099679E79E699679E79E699679E79E699C8
:10802800E7FF79E699679E79E699679E01061860E9
:1080380080010618E0FF01061860800106186080BC
:10804800FFFFFFFFFFFFFFFFFFFFFFFFFFFFFFFF38
:10805800FFFFFFFFFFFFFFFFFFFFFFFFFFFFFFFF28
:10806800FFFFFFFFFFFFFFFF0106186080010618F2
:1080780060800106186080010618608079E69967BB
:108088009E79E699679E79E699679E79E699679E53
:1080980079E699679E79E699679E79E699679E7968
:1080A800E699679E79E699679E79E699679E79E6EB
:1080B80099679E79E699679E79E699679E79E69928
:1080C800679E79E699679E79E699679E79E699674A
:1080D8009E79E699679E79E699679E79E699679E03
:1080E80079E699679E79E699679E79E699679E7918
:1080F800E699679E79E699679E79E699679E79E69B
:1081080099679E79E699679E79E699679E79E699D7
:10811800679E79E699679E79E699679E01061860D9
:1081280080010618608001061860800106186080CA
:10813800FFFFFFFFFFFFFFFFFFFFFFFFFFFFFFFF47
:10814800FFFFFFFFFFFFFFFFFFFFFFFFFFFFFFFF37
:10815800FFFFFFFFFFFFFFFF010618608001061801
:1081680060800106186080010618608079E69967CA
:108178009E79E699679E79E699679E79E699679E62
:1081880079E699679E79E699679E79E699679E7977
:10819800E699679E79E699679E79E699679E79E6FA
:1081A80099679E79E699679E79E699679E79E69937
:1081B800679E79E699679E79E699679E79E6996759
:1081C8009E79E699679E79E699679E79E699679E12
:1081D80079E699679E79E699679E79E699679E7927
:1081E800E699679E79E699679E79E699679E79E6AA
:1081F80099679E79E699679E79E699679E79E699E7
:10820800679E79E699679E79E699679E01061860E8
:1082180080010618608001061860800106186080D9
:10822800FFFFFFFFFFFFFFFFFFFFFFFFFFFFFFFF56
:10823800FFFFFFFF256400005B44454255475D2072
:10824800436F696E20696E7365727465640000001F
:1082580047455420524541445921000047414D4566
:10826800204F56455221000053434F52453A0000D3
:108278005052455353204649524520425554544F75
:108288004E0000004C4556454C20434C4541524554
:1082980044210000861F0010521F0010E21F00102A
:1082A800F81C0010701D00104861726477617265D7
:1082B80020616C61726D20256420616C7265616457
:1082C8007920636C61696D65640000000A2A2A2AB6
:1082D8002050414E4943202A2A2A0A000A00000059
:1082E800486172642061737365727400666E692BED
:1082F80000000000666E69006E616E00666E692D92
:10830800000000003A4E0010F04D0010F04D001033
:10831800324E0010F04D0010F04D0010F04D0010DE
:10832800F04D0010F04D0010F04D0010F04D001011
:108338002A4E0010F04D0010244E0010F04D001091
:10834800F04D00101C4E0010904F00104C4E0010C5
:10835800844F00104C4E0010724F00104C4E00100D
:108368004C4E00104C4E00104C4E00104C4E00105D
:108378004C4E00104C4E0010424E00104C4E001057
:108388004C4E00104C4E00104C4E00104C4E00103D
:10839800424E0010D24F0010944E0010944E001020
:1083A800944E0010944E0010944E0010944E0010FD
:1083B800944E0010944E0010944E0010944E0010ED
:1083C800944E0010944E0010944E0010944E0010DD
:1083D800944E0010944E0010944E0010944E0010CD
:1083E800944E0010944E0010944E0010944E0010BD
:1083F800944E0010944E0010944E0010944E0010AD
:10840800944E0010944E0010944E0010944E00109C
:10841800944E0010344F0010A04F0010344F00103D
:10842800944E0010944E0010944E0010944E00107C
:10843800944E0010944E0010944E0010944E00106C
:10844800944E0010944E0010944E0010944E00105C
:10845800944E0010944E0010944E0010944E00104C
:10846800EC510010944E0010944E0010944E0010E1
:10847800944E0010944E0010944E0010944E00102C
:10848800944E0010944E0010EC510010E64F00106E
:10849800EC510010344F0010A04F0010344F001062
:1084A800000000000000F03F000000000000244031
:1084B80000000000000059400000000000408F400C
:1084C800000000000088C34000000000006AF84077
:1084D8000000000080842E4100000000D01263419B
:1084E8000000000084D797410000000065CDCD4111
:1084F80052656C6561736500626F6F74325F7732C5
:108508003571303830000000302E3100312E352ED4
:10851800310000007069636F000000007069636FCC
:108528002D636F6D706F736974652D766964656FFF
:1085380000000000417567203135203230323400A8
:1085480006005250D3F07542F884001006005250CD
:10855800E182887F00850010060052503ABCA911BC
:108568001085001006005250BBFF3CB61C85001059
:108578000D0A00005541525420737464696E00005E
:1085880055415254207374646F75740055415254A8
:1085980020737464696E202F207374646F7574007F
:1085A8000600525053B4F4A19485001008005250AC
:1085B800920000004E6F2070726F6772616D2073B9
:0885C800706163650000000012
:1085D0004885001054850010608500108802001046
:1085E0006C85001094020010A0020010AC02001074
:0885F000B4850010A8850010FD
:1085F800F0B5C646150000B504001E000268EFF38A
:10860800108172B61368002BFCD0BFF35F8F042370
:10861800E356002B2DDB2268BFF35F8F002010602C
:1086280081F31088D0221206127852B290469A42EC
:1086380003D1002080BCB846F0BD00270BE02368BA
:10864800BFF35F8F1F6081F310882800310000F0AE
:1086580033F80028EDD12268EFF3108172B6136861
:10866800002BFCD0BFF35F8F23797F2BE7D94346DC
:1086780002E0D0231B061B6823712368BFF35F8FBA
:1086880000221A6081F310880120D3E70268EFF313
:10869800108172B61368002BFCD0BFF35F8FFF23E5
:1086A80003710368BFF35F8F00221A6081F310889B
:1086B80040BF70477047C04601B40248844601BCB9
:1086C800604700BF413400100800000030BE0120A0
:1086D80030E60020010000000A0000001E00000033
:1086E800050000000000000001000000010000007B
:1086F800010000000100000001000000010000006E
:10870800010000000100000002000000010000005C
:108718000200000002000000020000000200000049
:10872800010000000200000002000000020000003A
:108738000200000002000000020000000200000029
:108748000200000002000000020000000200000019
:108758000200000002000000020000000200000009
:1087680002000000020000000200000002000000F9
:1087780002000000020000000200000002000000E9
:1087880002000000020000000100000001000000DB
:1087980001000000010000000100000001000000CD
:1087A80001000000010000000200000001000000BC
:1087B80002000000020000000200000002000000A9
:1087C800010000000200000002000000020000009A
:1087D8000000000000000000000000000000000091
:1087E8000200000002000000020000000200000079
:1087F8000200000002000000020000000200000069
:108808000200000002000000010000000200000059
:10881800010000000200000002000000010000004A
:10882800020000000100000001000000010000003B
:10883800010000000100000001000000010000002C
:10884800010000000100000002000000010000001B
:108858000200000002000000020000000200000008
:1088680001000000020000000200000002000000F9
:1088780002000000020000000200000002000000E8
:1088880002000000020000000000000000000000DC
:1088980002000000020000000200000002000000C8
:1088A80000000000000000000000000000000000C0
:1088B80000000000000000000000000000000000B0
:1088C800000000000000000001000000010000009E
:1088D800010000000100000001000000010000008C
:1088E800010000000100000002000000010000007B
:1088F8000200000002000000020000000200000068
:108908000100000002000000020000000200000058
:108918000200000002000000020000000200000047
:10892800020000000200000000000000000000003B
:108938000200000002000000020000000200000027
:10894800000000000000000000000000000000001F
:10895800000000000000000000000000000000000F
:1089680000000000000000003838380707073838D2
:10897800380707073838380707070000FF81FFFF67
:1089880081FFFF81FF0700E00700E00700E000002B
:1089980000000000000000000000000000000000CF
:1089A800FF3FF0FF03FF3FF0FF03FF3FF0FF03FF30
:1089B8000780FF03FF0780FF03FF0780FF03FF0017
:1089C80000FC03FF0000FC03FF0000FC031F3870DD
:1089D800E0031F3870E0031F3870E0031F0000E059
:1089E800031F0000E0031F0000E0031F0000E00376
:1089F800FFC78FFF03FFC78FFF03FFC78FFF03FF6B
:108A0800F87FFC03FFF87FFC03FFF87FFC03FFC738
:108A18008FFF03FFC78FFF03FFC78FFF030000000F
:108A2800FF3FF0FF03FF3FF0FF03FF3FF0FF03FFAF
:108A38000780FF03FF0780FF03FF0780FF03FF0096
:108A480000FC03FF0000FC03FF0000FC031F38705C
:108A5800E0031F3870E0031F3870E0031F0000E0D8
:108A6800031F0000E0031F0000E0031F0000E003F5
:108A7800FFC78FFF03FFC78FFF03FFC78FFF03FFEA
:108A88003870FC03FF3870FC03FF3870FC031FC705
:108A98008FE3031FC78FE3031FC78FE303000000A3
:108AA8003FFEFFF1033FFEFFF1033FFEFFF103F836
:108AB800F13F7E00F8F13F7E00F8F13F7E0038007C
:108AC80000700038000070003800007000000EC010
:108AD8000100000EC00100000EC0010000000000EF
:108AE800000000000000000000000000000000007E
:108AF8000700008003070000800307000080033F91
:108B0800FEFFF1033FFEFFF1033FFEFFF103C7FF46
:108B1800FF8F03C7FFFF8F03C7FFFF8F030000000E
:108B28003FFEFFF1033FFEFFF1033FFEFFF103FFAE
:108B3800F13FFE03FFF13FFE03FFF13FFE033F005D
:108B480000F0033F0000F0033F0000F003070EC0F1
:108B5800F103070EC08103070EC0810300000080E7
:108B680003000000000000000000000000000000FA
:108B780000000000000000000000000000000038B5
:108B8800FEFF710038FEFF710038FEFF7100FF81A3
:108B980007FE03FF8107FE03FF8107FE03000000B5
:108BA800FFFFFFFFFFFFFFFFFFFFFFFFFFFFFFFFCD
:108BB800FFFFFFFFFFFFFFFFFFFFFFFFFFFFFFFFBD
:108BC800FFFFFFFFFFFFFFFFFFFFFFFFFFFFFFFFAD
:108BD800FFFFFFFFFFFFFFFFFFFFFFFFFFFFFFFF9D
:108BE800FFFFFFFFFFFFFFFFFFFFFFFFFFFFFFFF8D
:108BF800FFFFFFFFFFFFFFFFFFFFFFFFFFFFFF3F3D
:108C0800FFFFFFFFFFFFFFFFFFFFFFFFFFFFFFFF6C
:108C1800FFFFFFFFFFFFFFFFFFFFFFFFFFFFFFFF5C
:108C2800FFFFFFFFFFFFFFFFFFFFFFFFFFFFFFFF4C
:108C3800FFFFFFFFFFFFFFFFFFFFFFFFFFFFFFFF3C
:108C4800FFFFFFFFFFFFFFFFFFFFFFFFFFFFFFFF2C
:108C5800FFFFFFFFFFFFFFFFFFFFFFFFFFFFFF3FDC
:108C6800FFFFFFFFFFFFFFFFFFFFFFFFFFFFFFFF0C
:108C7800FFFFFFFFFFFFFFFFFFFFFFFFFFFFFFFFFC
:108C8800FFFFFFFFFFFFFFFFFFFFFFFFFFFFFFFFEC
:108C9800FFFFFFFFFFFFFFFFFFFFFFFFFFFFFFFFDC
:108CA800FFFFFFFFFFFFFFFFFFFFFFFFFFFFFFFFCC
:108CB800FFFFFFFFFFFFFFFFFFFFFFFFFFFFFF3F7C
:108CC800FFFFFFFFFFFFFFFFFFFFFFFFFFFFFFFFAC
:108CD800FFFFFFFFFFFFFFFFFFFFFFFFFFFFFFFF9C
:108CE800FFFFFFFFFFFFFFFFFFFFFFFFFFFFFFFF8C
:108CF800FFFFFFFFFFFFFFFFFFFFFFFFFFFFFFFF7C
:108D0800FFFFFFFFFFFFFFFFFFFFFFFFFFFFFFFF6B
:108D1800FFFFFFFFFFFFFFFFFFFFFFFFFFFFFF3F1B
:108D2800FFFFFFFFFFFFFFFFFFFFFFFFFFFFFFFF4B
:108D3800FFFFFFFFFFFFFFFFFFFFFFFFFFFFFFFF3B
:108D4800FFFFFFFFFFFFFFFFFFFFFFFFFFFFFFFF2B
:108D5800FFFFFFFFFFFFFFFFFFFFFFFFFFFFFFFF1B
:108D6800FFFFFFFFFFFFFFFFFFFFFFFFFFFFFFFF0B
:108D7800FFFFFFFFFFFFFFFFFFFFFFFFFFFFFF3FBB
:108D8800FFFFFFFFFFFFFFFFFFFFFFFFFFFFFFFFEB
:108D9800FFFFFFFFFFFFFFFFFFFFFFFFFFFFFFFFDB
:108DA800FFFFFFFFFFFFFFFFFFFFFFFFFFFFFFFFCB
:108DB800FFFFFFFFFFFFFFFFFFFFFFFFFFFFFFFFBB
:108DC800FFFFFFFFFFFFFFFFFFFFFFFFFFFFFFFFAB
:108DD800FFFFFFFFFFFFFFFFFFFFFFFFFFFFFF3F5B
:108DE800FFFFFFFFFFFFFFFFFFFFFFFFFFFFFFFF8B
:108DF800FFFFFFFFFFFFFFFFFFFFFFFFFFFFFFFF7B
:108E0800FFFFFFFFFFFFFFFFFFFFFFFFFFFFFFFF6A
:108E1800FFFFFFFFFFFFFFFFFFFFFFFFFFFFFFFF5A
:108E2800FFFFFFFFFFFFFFFFFFFFFFFFFFFFFFFF4A
:108E3800FFFFFFFFFFFFFFFFFFFFFFFFFFFFFF3FFA
:108E4800FFFFFFFFFFFFFFFFFFFFFFFFFFFFFFFF2A
:108E5800FFFFFFFFFFFFFFFFFFFFFFFFFFFFFFFF1A
:108E6800FFFFFFFFFFFFFFFFFFFFFFFFFFFFFFFF0A
:108E7800FFFFFFFFFFFFFFFFFFFFFFFFFFFFFFFFFA
:108E8800FFFFFFFFFFFFFFFFFFFFFFFFFFFFFFFFEA
:108E9800FFFFFFFFFFFFFFFFFFFFFFFFFFFFFF3F9A
:108EA800FFFFFFFFFFFFFFFFFFFFFFFFFFFFFFFFCA
:108EB800FFFFFFFFFFFFFFFFFFFFFFFFFFFFFFFFBA
:108EC800FFFFFFFFFFFFFFFFFFFFFFFFFFFFFFFFAA
:108ED800FFFFFFFFFFFFFFFFFFFFFFFFFFFFFFFF9A
:108EE800FFFFFFFFFFFFFFFFFFFFFFFFFFFFFFFF8A
:108EF800FFFFFFFFFFFFFFFFFFFFFFFFFFFFFF3F3A
:108F0800FFFFFFFFFFFFFFFFFFFFFFFFFFFFFFFF69
:108F1800FFFFFFFFFFFFFFFFFFFFFFFFFFFFFFFF59
:108F2800FFFFFFFFFFFFFFFFFFFFFFFFFFFFFFFF49
:108F3800FFFFFFFFFFFFFFFFFFFFFFFFFFFFFFFF39
:108F4800FFFFFFFFFFFFFFFFFFFFFFFFFFFFFFFF29
:108F5800FFFFFFFFFFFFFFFFFFFFFFFFFFFFFF3FD9
:108F6800FFFFFFFFFFFFFFFFFFFFFFFFFFFFFFFF09
:108F7800FFFFFFFFFFFFFFFFFFFFFFFFFFFFFFFFF9
:108F8800FFFFFFFFFFFFFFFFFFFFFFFFFFFFFFFFE9
:108F9800FFFFFFFFFFFFFFFFFFFFFFFFFFFFFFFFD9
:108FA800FFFFFFFFFFFFFFFFFFFFFFFFFFFFFFFFC9
:108FB800FFFFFFFFFFFFFFFFFFFFFFFFFFFFFF3F79
:108FC800FFFFFFFFFFFFFFFFFFFFFFFFFFFFFFFFA9
:108FD800FFFFFFFFFFFFFFFFFFFFFFFFFFFFFFFF99
:108FE800FFFFFFFFFFFFFFFFFFFFFFFFFFFFFFFF89
:108FF800FFFFFFFFFFFFFFFFFFFFFFFFFFFFFFFF79
:10900800FFFFFFFFFFFFFFFFFFFFFFFFFFFFFFFF68
:10901800FFFFFFFFFFFFFFFFFFFFFFFFFFFFFF3F18
:10902800FFFFFFFFFFFFFFFFFFFFFFFFFFFFFFFF48
:10903800FFFFFFFFFFFFFFFFFFFFFFFFFFFFFFFF38
:10904800FFFFFFFFFFFFFFFFFFFFFFFFFFFFFFFF28
:10905800FFFFFFFFFFFFFFFFFFFFFFFFFFFFFFFF18
:10906800FFFFFFFFFFFFFFFFFFFFFFFFFFFFFFFF08
:10907800FFFFFFFFFFFFFFFFFFFFFFFFFFFFFF3FB8
:10908800FFFFFFFFFFFFFFFFFFFFFFFFFFFFFFFFE8
:10909800FFFFFFFFFFFFFFFFFFFFFFFFFFFFFFFFD8
:1090A800FFFFFFFFFFFFFFFFFFFFFFFFFFFFFFFFC8
:1090B800FFFFFFFFFFFFFFFFFFFFFFFFFFFFFFFFB8
:1090C800FFFFFFFFFFFFFFFFFFFFFFFFFFFFFFFFA8
:1090D800FFFFFFFFFFFFFFFFFFFFFFFFFFFFFF3F58
:1090E800FFFFFFFFFFFFFFFFFFFFFFFFFFFFFFFF88
:1090F800FFFFFFFFFFFFFFFFFFFFFFFFFFFFFFFF78
:10910800FFFFFFFFFFFFFFFFFFFFFFFFFFFFFFFF67
:10911800FFFFFFFFFFFFFFFFFFFFFFFFFFFFFFFF57
:10912800FFFFFFFFFFFFFFFFFFFFFFFFFFFFFFFF47
:10913800FFFFFFFFFFFFFFFFFFFFFFFFFFFFFF3FF7
:10914800FFFFFFFFFFFFFFFFFFFFFFFFFFFFFFFF27
:10915800FFFFFFFFFFFFFFFFFFFFFFFFFFFFFFFF17
:10916800FFFFFFFFFFFFFFFFFFFFFFFFFFFFFFFF07
:10917800FFFFFFFFFFFFFFFFFFFFFFFFFFFFFFFFF7
:10918800FFFFFFFFFFFFFFFFFFFFFFFFFFFFFFFFE7
:10919800FFFFFFFFFFFFFFFFFFFFFFFFFFFFFF3F97
:1091A800FFFFFFFFFFFFFFFFFFFFFFFFFFFFFFFFC7
:1091B800FFFFFFFFFFFFFFFFFFFFFFFFFFFFFFFFB7
:1091C800FFFFFFFFFFFFFFFFFFFFFFFFFFFFFFFFA7
:1091D800FFFFFFFFFFFFFFFFFFFFFFFFFFFFFFFF97
:1091E800FFFFFFFFFFFFFFFFFFFFFFFFFFFFFFFF87
:1091F800FFFFFFFFFFFFFFFFFFFFFFFFFFFFFF3F37
:10920800FFFFFFFFFFFFFFFFFFFFFFFFFFFFFFFF66
:10921800FFFFFFFFFFFFFFFFFFFFFFFFFFFFFFFF56
:10922800FFFFFFFFFFFFFFFFFFFFFFFFFFFFFFFF46
:10923800FFFFFFFFFFFFFFFFFFFFFFFFFFFFFFFF36
:10924800FFFFFFFFFFFFFFFFFFFFFFFFFFFFFFFF26
:10925800FFFFFFFFFFFFFFFFFFFFFFFFFFFFFF3FD6
:10926800FFFFFFFFFFFFFFFFFFFFFFFFFFFFFFFF06
:10927800FFFFFFFFFFFFFFFFFFFFFFFFFFFFFFFFF6
:10928800FFFFFFFFFFFFFFFFFFFFFFFFFFFFFFFFE6
:10929800FFFFFFFFFFFFFFFFFFFFFFFFFFFFFFFFD6
:1092A800FFFFFFFFFFFFFFFFFFFFFFFFFFFFFFFFC6
:1092B800FFFFFFFFFFFFFFFFFFFFFFFFFFFFFF3F76
:1092C800FFFFFFFFFFFFFFFFFFFFFFFFFFFFFFFFA6
:1092D800FFFFFFFFFFFFFFFFFFFFFFFFFFFFFFFF96
:1092E800FFFFFFFFFFFFFFFFFFFFFFFFFFFFFFFF86
:1092F800FFFFFFFFFFFFFFFFFFFFFFFFFFFFFFFF76
:10930800FFFFFFFFFFFFFFFFFFFFFFFFFFFFFFFF65
:10931800FFFFFFFFFFFFFFFFFFFFFFFFFFFFFF3F15
:10932800FFFFFFFFFFFFFFFFFFFFFFFFFFFFFFFF45
:10933800FFFFFFFFFFFFFFFFFFFFFFFFFFFFFFFF35
:10934800FFFFFFFFFFFFFFFFFFFFFFFFFFFFFFFF25
:10935800FFFFFFFFFFFFFFFFFFFFFFFFFFFFFFFF15
:10936800FFFFFFFFFFFFFFFFFFFFFFFFFFFFFFFF05
:10937800FFFFFFFFFFFFFFFFFFFFFFFFFFFFFF3FB5
:10938800FFFFFFFFFFFFFFFFFFFFFFFFFFFFFFFFE5
:10939800FFFFFFFFFFFFFFFFFFFFFFFFFFFFFFFFD5
:1093A800FFFFFFFFFFFFFFFFFFFFFFFFFFFFFFFFC5
:1093B800FFFFFFFFFFFFFFFFFFFFFFFFFFFFFFFFB5
:1093C800FFFFFFFFFFFFFFFFFFFFFFFFFFFFFFFFA5
:1093D800FFFFFFFFFFFFFFFFFFFFFFFFFFFFFF3F55
:1093E800FFFFFFFFFFFFFFFFFFFFFFFFFFFFFFFF85
:1093F800FFFFFFFFFFFFFFFFFFFFFFFFFFFFFFFF75
:10940800FFFFFFFFFFFFFFFFFFFFFFFFFFFFFFFF64
:10941800FFFFFFFFFFFFFFFFFFFFFFFFFFFFFFFF54
:10942800FFFFFFFFFFFFFFFFFFFFFFFFFFFFFFFF44
:10943800FFFFFFFFFFFFFFFFFFFFFFFFFFFFFF3FF4
:10944800FFFFFFFFFFFFFFFFFFFFFFFFFFFFFFFF24
:10945800FFFFFFFFFFFFFFFFFFFFFFFFFFFFFFFF14
:10946800FFFFFFFFFFFFFFFFFFFFFFFFFFFFFFFF04
:10947800FFFFFFFFFFFFFFFFFFFFFFFFFFFFFFFFF4
:10948800FFFFFFFFFFFFFFFFFFFFFFFFFFFFFFFFE4
:10949800FFFFFFFFFFFFFFFFFFFFFFFFFFFFFF3F94
:1094A800FFFFFFFFFFFFFFFFFFFFFFFFFFFFFFFFC4
:1094B800FFFFFFFFFFFFFFFFFFFFFFFFFFFFFFFFB4
:1094C800FFFFFFFFFFFFFFFFFFFFFFFFFFFFFFFFA4
:1094D800FFFFFFFFFFFFFFFFFFFFFFFFFFFFFFFF94
:1094E800FFFFFFFFFFFFFFFFFFFFFFFFFFFFFFFF84
:1094F800FFFFFFFFFFFFFFFFFFFFFFFFFFFFFF3F34
:10950800FFFFFFFFFFFFFFFFFFFFFFFFFFFFFFFF63
:10951800FFFFFFFFFFFFFFFFFFFFFFFFFFFFFFFF53
:10952800FFFFFFFFFFFFFFFFFFFFFFFFFFFFFFFF43
:10953800FFFFFFFFFFFFFFFFFFFFFFFFFFFFFFFF33
:10954800FFFFFFFFFFFFFFFFFFFFFFFFFFFFFFFF23
:10955800FFFFFFFFFFFFFFFFFFFFFFFFFFFFFF3FD3
:10956800FFFFFFFFFFFFFFFFFFFFFFFFFFFFFFFF03
:10957800FFFFFFFFFFFFFFFFFFFFFFFFFFFFFFFFF3
:10958800FFFFFFFFFFFFFFFFFFFFFFFFFFFFFFFFE3
:10959800FFFFFFFFFFFFFFFFFFFFFFFFFFFFFFFFD3
:1095A800FFFFFFFFFFFFFFFFFFFFFFFFFFFFFFFFC3
:1095B800FFFFFFFFFFFFFFFFFFFFFFFFFFFFFF3F73
:1095C800FFFFFFFFFFFFFFFFFFFFFFFFFFFFFFFFA3
:1095D800FFFFFFFFFFFFFFFFFFFFFFFFFFFFFFFF93
:1095E800FFFFFFFFFFFFFFFFFFFFFFFFFFFFFFFF83
:1095F800FFFFFFFFFFFFFFFFFFFFFFFFFFFFFFFF73
:10960800FFFFFFFFFFFFFFFFFFFFFFFFFFFFFFFF62
:10961800FFFFFFFFFFFFFFFFFFFFFFFFFFFFFF3F12
:10962800FFFFFFFFFFFFFFFFFFFFFFFFFFFFFFFF42
:10963800FFFFFFFFFFFFFFFFFFFFFFFFFFFFFFFF32
:10964800FFFFFFFFFFFFFFFFFFFFFFFFFFFFFFFF22
:10965800FFFFFFFFFFFFFFFFFFFFFFFFFFFFFFFF12
:10966800FFFFFFFFFFFFFFFFFFFFFFFFFFFFFFFF02
:10967800FFFFFFFFFFFFFFFFFFFFFFFFFFFFFF3FB2
:10968800FFFFFFFFFFFFFFFFFFFFFFFFFFFFFFFFE2
:10969800FFFFFFFFFFFFFFFFFFFFFFFFFFFFFFFFD2
:1096A800FFFFFFFFFFFFFFFFFFFFFFFFFFFFFFFFC2
:1096B800FFFFFFFFFFFFFFFFFFFFFFFFFFFFFFFFB2
:1096C800FFFFFFFFFFFFFFFFFFFFFFFFFFFFFFFFA2
:1096D800FFFFFFFFFFFFFFFFFFFFFFFFFFFFFF3F52
:1096E800FFFFFFFFFFFFFFFFFFFFFFFFFFFFFFFF82
:1096F800FFFFFFFFFFFFFFFFFFFFFFFFFFFFFFFF72
:10970800FFFFFFFFFFFFFFFFFFFFFFFFFFFFFFFF61
:10971800FFFFFFFFFFFFFFFFFFFFFFFFFFFFFFFF51
:10972800FFFFFFFFFFFFFFFFFFFFFFFFFFFFFFFF41
:10973800FFFFFFFFFFFFFFFFFFFFFFFFFFFFFF3FF1
:10974800FFFFFFFFFFFFFFFFFFFFFFFFFFFFFFFF21
:10975800FFFFFFFFFFFFFFFFFFFFFFFFFFFFFFFF11
:10976800FFFFFFFFFFFFFFFFFFFFFFFFFFFFFFFF01
:10977800FFFFFFFFFFFFFFFFFFFFFFFFFFFFFFFFF1
:10978800FFFFFFFFFFFFFFFFFFFFFFFFFFFFFFFFE1
:10979800FFFFFFFFFFFFFFFFFFFFFFFFFFFFFF3F91
:1097A800FFFFFFFFFFFFFFFFFFFFFFFFFFFFFFFFC1
:1097B800FFFFFFFFFFFFFFFFFFFFFFFFFFFFFFFFB1
:1097C800FFFFFFFFFFFFFFFFFFFFFFFFFFFFFFFFA1
:1097D800FFFFFFFFFFFFFFFFFFFFFFFFFFFFFFFF91
:1097E800FFFFFFFFFFFFFFFFFFFFFFFFFFFFFFFF81
:1097F800FFFFFFFFFFFFFFFFFFFFFFFFFFFFFF3F31
:10980800FFFFFFFFFFFFFFFFFFFFFFFFFFFFFFFF60
:10981800FFFFFFFFFFFFFFFFFFFFFFFFFFFFFFFF50
:10982800FFFFFFFFFFFFFFFFFFFFFFFFFFFFFFFF40
:10983800FFFFFFFFFFFFFFFFFFFFFFFFFFFFFFFF30
:10984800FFFFFFFFFFFFFFFFFFFFFFFFFFFFFFFF20
:10985800FFFFFFFFFFFFFFFFFFFFFFFFFFFFFF3FD0
:10986800FFFFFFFFFFFFFFFFFFFFFFFFFFFFFFFF00
:10987800FFFFFFFFFFFFFFFFFFFFFFFFFFFFFFFFF0
:10988800FFFFFFFFFFFFFFFFFFFFFFFFFFFFFFFFE0
:10989800FFFFFFFFFFFFFFFFFFFFFFFFFFFFFFFFD0
:1098A800FFFFFFFFFFFFFFFFFFFFFFFFFFFFFFFFC0
:1098B800FFFFFFFFFFFFFFFFFFFFFFFFFFFFFF3F70
:1098C800FFFFFFFFFFFFFFFFFFFFFFFFFFFFFFFFA0
:1098D800FFFFFFFFFFFFFFFFFFFFFFFFFFFFFFFF90
:1098E800FFFFFFFFFFFFFFFFFFFFFFFFFFFFFFFF80
:1098F800FFFFFFFFFFFFFFFFFFFFFFFFFFFFFFFF70
:10990800FFFFFFFFFFFFFFFFFFFFFFFFFFFFFFFF5F
:10991800FFFFFFFFFFFFFFFFFFFFFFFFFFFFFF3F0F
:10992800FFFFFFFFFFFFFFFFFFFFFFFFFFFFFFFF3F
:10993800FFFFFFFFFFFFFFFFFFFFFFFFFFFFFFFF2F
:10994800FFFFFFFFFFFFFFFFFFFFFFFFFFFFFFFF1F
:10995800FFFFFFFFFFFFFFFFFFFFFFFFFFFFFFFF0F
:10996800FFFFFFFFFFFFFFFFFFFFFFFFFFFFFFFFFF
:10997800FFFFFFFFFFFFFFFFFFFFFFFFFFFFFF3FAF
:10998800FFFFFFFFFFFFFFFFFFFFFFFFFFFFFFFFDF
:10999800FFFFFFFFFFFFFFFFFFFFFFFFFFFFFFFFCF
:1099A800FFFFFFFFFFFFFFFFFFFFFFFFFFFFFFFFBF
:1099B800FFFFFFFFFFFFFFFFFFFFFFFFFFFFFFFFAF
:1099C800FFFFFFFFFFFFFFFFFFFFFFFFFFFFFFFF9F
:1099D800FFFFFFFFFFFFFFFFFFFFFFFFFFFFFF3F4F
:1099E800FFFFFFFFFFFFFFFFFFFFFFFFFFFFFFFF7F
:1099F800FFFFFFFFFFFFFFFFFFFFFFFFFFFFFFFF6F
:109A0800FFFFFFFFFFFFFFFFFFFFFFFFFFFFFFFF5E
:109A1800FFFFFFFFFFFFFFFFFFFFFFFFFFFFFFFF4E
:109A2800FFFFFFFFFFFFFFFFFFFFFFFFFFFFFFFF3E
:109A3800FFFFFFFFFFFFFFFFFFFFFFFFFFFFFF3FEE
:109A4800FFFFFFFFFFFFFFFFFFFFFFFFFFFFFFFF1E
:109A5800FFFFFFFFFFFFFFFFFFFFFFFFFFFFFFFF0E
:109A6800FFFFFFFFFFFFFFFFFFFFFFFFFFFFFFFFFE
:109A7800FFFFFFFFFFFFFFFFFFFFFFFFFFFFFFFFEE
:109A8800FFFFFFFFFFFFFFFFFFFFFFFFFFFFFFFFDE
:109A9800FFFFFFFFFFFFFFFFFFFFFFFFFFFFFF3F8E
:109AA800FFFFFFFFFFFFFFFFFFFFFFFFFFFFFFFFBE
:109AB800FFFFFFFFFFFFFFFFFFFFFFFFFFFFFFFFAE
:109AC800FFFFFFFFFFFFFFFFFFFFFFFFFFFFFFFF9E
:109AD800FFFFFFFFFFFFFFFFFFFFFFFFFFFFFFFF8E
:109AE800FFFFFFFFFFFFFFFFFFFFFFFFFFFFFFFF7E
:109AF800FFFFFFFFFFFFFFFFFFFFFFFFFFFFFF3F2E
:109B0800FFFFFFFFFFFFFFFFFFFFFFFFFFFFFFFF5D
:109B1800FFFFFFFFFFFFFFFFFFFFFFFFFFFFFFFF4D
:109B2800FFFFFFFFFFFFFFFFFFFFFFFFFFFFFFFF3D
:109B3800FFFFFFFFFFFFFFFFFFFFFFFFFFFFFFFF2D
:109B4800FFFFFFFFFFFFFFFFFFFFFFFFFFFFFFFF1D
:109B5800FFFFFFFFFFFFFFFFFFFFFFFFFFFFFF3FCD
:109B6800FFFFFFFFFFFFFFFFFFFFFFFFFFFFFFFFFD
:109B7800FFFFFFFFFFFFFFFFFFFFFFFFFFFFFFFFED
:109B8800FFFFFFFFFFFFFFFFFFFFFFFFFFFFFFFFDD
:109B9800FFFFFFFFFFFFFFFFFFFFFFFFFFFFFFFFCD
:109BA800FFFFFFFFFFFFFFFFFFFFFFFFFFFFFFFFBD
:109BB800FFFFFFFFFFFFFFFFFFFFFFFFFFFFFF3F6D
:109BC800FFFFFFFFFFFFFFFFFFFFFFFFFFFFFFFF9D
:109BD800FFFFFFFFFFFFFFFFFFFFFFFFFFFFFFFF8D
:109BE800FFFFFFFFFFFFFFFFFFFFFFFFFFFFFFFF7D
:109BF800FFFFFFFFFFFFFFFFFFFFFFFFFFFFFFFF6D
:109C0800FFFFFFFFFFFFFFFFFFFFFFFFFFFFFFFF5C
:109C1800FFFFFFFFFFFFFFFFFFFFFFFFFFFFFF3F0C
:109C2800FFFFFFFFFFFFFFFFFFFFFFFFFFFFFFFF3C
:109C3800FFFFFFFFFFFFFFFFFFFFFFFFFFFFFFFF2C
:109C4800FFFFFFFFFFFFFFFFFFFFFFFFFFFFFFFF1C
:109C5800FFFFFFFFFFFFFFFFFFFFFFFFFFFFFFFF0C
:109C6800FFFFFFFFFFFFFFFFFFFFFFFFFFFFFFFFFC
:109C7800FFFFFFFFFFFFFFFFFFFFFFFFFFFFFF3FAC
:109C8800FFFFFFFFFFFFFFFFFFFFFFFFFFFFFFFFDC
:109C9800FFFFFFFFFFFFFFFFFFFFFFFFFFFFFFFFCC
:109CA800FFFFFFFFFFFFFFFFFFFFFFFFFFFFFFFFBC
:109CB800FFFFFFFFFFFFFFFFFFFFFFFFFFFFFFFFAC
:109CC800FFFFFFFFFFFFFFFFFFFFFFFFFFFFFFFF9C
:109CD800FFFFFFFFFFFFFFFFFFFFFFFFFFFFFF3F4C
:109CE800FFFFFFFFFFFFFFFFFFFFFFFFFFFFFFFF7C
:109CF800FFFFFFFFFFFFFFFFFFFFFFFFFFFFFFFF6C
:109D0800FFFFFFFFFFFFFFFFFFFFFFFFFFFFFFFF5B
:109D1800FFFFFFFFFFFFFFFFFFFFFFFFFFFFFFFF4B
:109D2800FFFFFFFFFFFFFFFFFFFFFFFFFFFFFFFF3B
:109D3800FFFFFFFFFFFFFFFFFFFFFFFFFFFFFF3FEB
:109D4800FFFFFFFFFFFFFFFFFFFFFFFFFFFFFFFF1B
:109D5800FFFFFFFFFFFFFFFFFFFFFFFFFFFFFFFF0B
:109D6800FFFFFFFFFFFFFFFFFFFFFFFFFFFFFFFFFB
:109D7800FFFFFFFFFFFFFFFFFFFFFFFFFFFFFFFFEB
:109D8800FFFFFFFFFFFFFFFFFFFFFFFFFFFFFFFFDB
:109D9800FFFFFFFFFFFFFFFFFFFFFFFFFFFFFF3F8B
:109DA800FFFFFFFFFFFFFFFFFFFFFFFFFFFFFFFFBB
:109DB800FFFFFFFFFFFFFFFFFFFFFFFFFFFFFFFFAB
:109DC800FFFFFFFFFFFFFFFFFFFFFFFFFFFFFFFF9B
:109DD800FFFFFFFFFFFFFFFFFFFFFFFFFFFFFFFF8B
:109DE800FFFFFFFFFFFFFFFFFFFFFFFFFFFFFFFF7B
:109DF800FFFFFFFFFFFFFFFFFFFFFFFFFFFFFF3F2B
:109E0800FFFFFFFFFFFFFFFFFFFFFFFFFFFFFFFF5A
:109E1800FFFFFFFFFFFFFFFFFFFFFFFFFFFFFFFF4A
:109E2800FFFFFFFFFFFFFFFFFFFFFFFFFFFFFFFF3A
:109E3800FFFFFFFFFFFFFFFFFFFFFFFFFFFFFFFF2A
:109E4800FFFFFFFFFFFFFFFFFFFFFFFFFFFFFFFF1A
:109E5800FFFFFFFFFFFFFFFFFFFFFFFFFFFFFF3FCA
:109E6800FFFFFFFFFFFFFFFFFFFFFFFFFFFFFFFFFA
:109E7800FFFFFFFFFFFFFFFFFFFFFFFFFFFFFFFFEA
:109E8800FFFFFFFFFFFFFFFFFFFFFFFFFFFFFFFFDA
:109E9800FFFFFFFFFFFFFFFFFFFFFFFFFFFFFFFFCA
:109EA800FFFFFFFFFFFFFFFFFFFFFFFFFFFFFFFFBA
:109EB800FFFFFFFFFFFFFFFFFFFFFFFFFFFFFF3F6A
:109EC800FFFFFFFFFFFFFFFFFFFFFFFFFFFFFFFF9A
:109ED800FFFFFFFFFFFFFFFFFFFFFFFFFFFFFFFF8A
:109EE800FFFFFFFFFFFFFFFFFFFFFFFFFFFFFFFF7A
:109EF800FFFFFFFFFFFFFFFFFFFFFFFFFFFFFFFF6A
:109F0800FFFFFFFFFFFFFFFFFFFFFFFFFFFFFFFF59
:109F1800FFFFFFFFFFFFFFFFFFFFFFFFFFFFFF3F09
:109F2800FFFFFFFFFFFFFFFFFFFFFFFFFFFFFFFF39
:109F3800FFFFFFFFFFFFFFFFFFFFFFFFFFFFFFFF29
:109F4800FFFFFFFFFFFFFFFFFFFFFFFFFFFFFFFF19
:109F5800FFFFFFFFFFFFFFFFFFFFFFFFFFFFFFFF09
:109F6800FFFFFFFFFFFFFFFFFFFFFFFFFFFFFFFFF9
:109F7800FFFFFFFFFFFFFFFFFFFFFFFFFFFFFF3FA9
:109F8800FFFFFFFFFFFFFFFFFFFFFFFFFFFFFFFFD9
:109F9800FFFFFFFFFFFFFFFFFFFFFFFFFFFFFFFFC9
:109FA800FFFFFFFFFFFFFFFFFFFFFFFFFFFFFFFFB9
:109FB800FFFFFFFFFFFFFFFFFFFFFFFFFFFFFFFFA9
:109FC800FFFFFFFFFFFFFFFFFFFFFFFFFFFFFFFF99
:109FD800FFFFFFFFFFFFFFFFFFFFFFFFFFFFFF3F49
:109FE800FFFFFFFFFFFFFFFFFFFFFFFFFFFFFFFF79
:109FF800FFFFFFFFFFFFFFFFFFFFFFFFFFFFFFFF69
:10A00800FFFFFFFFFFFFFFFFFFFFFFFFFFFFFFFF58
:10A01800FFFFFFFFFFFFFFFFFFFFFFFFFFFFFFFF48
:10A02800FFFFFFFFFFFFFFFFFFFFFFFFFFFFFFFF38
:10A03800FFFFFFFFFFFFFFFFFFFFFFFFFFFFFF3FE8
:10A04800FFFFFFFFFFFFFFFFFFFFFFFFFFFFFFFF18
:10A05800FFFFFFFFFFFFFFFFFFFFFFFFFFFFFFFF08
:10A06800FFFFFFFFFFFFFFFFFFFFFFFFFFFFFFFFF8
:10A07800FFFFFFFFFFFFFFFFFFFFFFFFFFFFFFFFE8
:10A08800FFFFFFFFFFFFFFFFFFFFFFFFFFFFFFFFD8
:10A09800FFFFFFFFFFFFFFFFFFFFFFFFFFFFFF3F88
:10A0A800FFFFFFFFFFFFFFFFFFFFFFFFFFFFFFFFB8
:10A0B800FFFFFFFFFFFFFFFFFFFFFFFFFFFFFFFFA8
:10A0C800FFFFFFFFFFFFFFFFFFFFFFFFFFFFFFFF98
:10A0D800FFFFFFFFFFFFFFFFFFFFFFFFFFFFFFFF88
:10A0E800FFFFFFFFFFFFFFFFFFFFFFFFFFFFFFFF78
:10A0F800FFFFFFFFFFFFFFFFFFFFFFFFFFFFFF3F28
:10A10800FFFFFFFFFFFFFFFFFFFFFFFFFFFFFFFF57
:10A11800FFFFFFFFFFFFFFFFFFFFFFFFFFFFFFFF47
:10A12800FFFFFFFFFFFFFFFFFFFFFFFFFFFFFFFF37
:10A13800FFFFFFFFFFFFFFFFFFFFFFFFFFFFFFFF27
:10A14800FFFFFFFFFFFFFFFFFFFFFFFFFFFFFFFF17
:10A15800FFFFFFFFFFFFFFFFFFFFFFFFFFFFFF3FC7
:10A16800FFFFFFFFFFFFFFFFFFFFFFFFFFFFFFFFF7
:10A17800FFFFFFFFFFFFFFFFFFFFFFFFFFFFFFFFE7
:10A18800FFFFFFFFFFFFFFFFFFFFFFFFFFFFFFFFD7
:10A19800FFFFFFFFFFFFFFFFFFFFFFFFFFFFFFFFC7
:10A1A800FFFFFFFFFFFFFFFFFFFFFFFFFFFFFFFFB7
:10A1B800FFFFFFFFFFFFFFFFFFFFFFFFFFFFFF3F67
:10A1C800FFFFFFFFFFFFFFFFFFFFFFFFFFFFFFFF97
:10A1D800FFFFFFFFFFFFFFFFFFFFFFFFFFFFFFFF87
:10A1E800FFFFFFFFFFFFFFFFFFFFFFFFFFFFFFFF77
:10A1F800FFFFFFFFFFFFFFFFFFFFFFFFFFFFFFFF67
:10A20800FFFFFFFFFFFFFFFFFFFFFFFFFFFFFFFF56
:10A21800FFFFFFFFFFFFFFFFFFFFFFFFFFFFFF3F06
:10A22800FFFFFFFFFFFFFFFFFFFFFFFFFFFFFFFF36
:10A23800FFFFFFFFFFFFFFFFFFFFFFFFFFFFFFFF26
:10A24800FFFFFFFFFFFFFFFFFFFFFFFFFFFFFFFF16
:10A25800FFFFFFFFFFFFFFFFFFFFFFFFFFFFFFFF06
:10A26800FFFFFFFFFFFFFFFFFFFFFFFFFFFFFFFFF6
:10A27800FFFFFFFFFFFFFFFFFFFFFFFFFFFFFF3FA6
:10A28800FFFFFFFFFFFFFFFFFFFFFFFFFFFFFFFFD6
:10A29800FFFFFFFFFFFFFFFFFFFFFFFFFFFFFFFFC6
:10A2A800FFFFFFFFFFFFFFFFFFFFFFFFFFFFFFFFB6
:10A2B800FFFFFFFFFFFFFFFFFFFFFFFFFFFFFFFFA6
:10A2C800FFFFFFFFFFFFFFFFFFFFFFFFFFFFFFFF96
:10A2D800FFFFFFFFFFFFFFFFFFFFFFFFFFFFFF3F46
:10A2E800FFFFFFFFFFFFFFFFFFFFFFFFFFFFFFFF76
:10A2F800FFFFFFFFFFFFFFFFFFFFFFFFFFFFFFFF66
:10A30800FFFFFFFFFFFFFFFFFFFFFFFFFFFFFFFF55
:10A31800FFFFFFFFFFFFFFFFFFFFFFFFFFFFFFFF45
:10A32800FFFFFFFFFFFFFFFFFFFFFFFFFFFFFFFF35
:10A33800FFFFFFFFFFFFFFFFFFFFFFFFFFFFFF3FE5
:10A34800FFFFFFFFFFFFFFFFFFFFFFFFFFFFFFFF15
:10A35800FFFFFFFFFFFFFFFFFFFFFFFFFFFFFFFF05
:10A36800FFFFFFFFFFFFFFFFFFFFFFFFFFFFFFFFF5
:10A37800FFFFFFFFFFFFFFFFFFFFFFFFFFFFFFFFE5
:10A38800FFFFFFFFFFFFFFFFFFFFFFFFFFFFFFFFD5
:10A39800FFFFFFFFFFFFFFFFFFFFFFFFFFFFFF3F85
:10A3A800FFFFFFFFFFFFFFFFFFFFFFFFFFFFFFFFB5
:10A3B800FFFFFFFFFFFFFFFFFFFFFFFFFFFFFFFFA5
:10A3C800FFFFFFFFFFFFFFFFFFFFFFFFFFFFFFFF95
:10A3D800FFFFFFFFFFFFFFFFFFFFFFFFFFFFFFFF85
:10A3E800FFFFFFFFFFFFFFFFFFFFFFFFFFFFFFFF75
:10A3F800FFFFFFFFFFFFFFFFFFFFFFFFFFFFFF3F25
:10A40800FFFFFFFFFFFFFFFFFFFFFFFFFFFFFFFF54
:10A41800FFFFFFFFFFFFFFFFFFFFFFFFFFFFFFFF44
:10A42800FFFFFFFFFFFFFFFFFFFFFFFFFFFFFFFF34
:10A43800FFFFFFFFFFFFFFFFFFFFFFFFFFFFFFFF24
:10A44800FFFFFFFFFFFFFFFFFFFFFFFFFFFFFFFF14
:10A45800FFFFFFFFFFFFFFFFFFFFFFFFFFFFFF3FC4
:10A46800FFFFFFFFFFFFFFFFFFFFFFFFFFFFFFFFF4
:10A47800FFFFFFFFFFFFFFFFFFFFFFFFFFFFFFFFE4
:10A48800FFFFFFFFFFFFFFFFFFFFFFFFFFFFFFFFD4
:10A49800FFFFFFFFFFFFFFFFFFFFFFFFFFFFFFFFC4
:10A4A800FFFFFFFFFFFFFFFFFFFFFFFFFFFFFFFFB4
:10A4B800FFFFFFFFFFFFFFFFFFFFFFFFFFFFFF3F64
:10A4C800FFFFFFFFFFFFFFFFFFFFFFFFFFFFFFFF94
:10A4D800FFFFFFFFFFFFFFFFFFFFFFFFFFFFFFFF84
:10A4E800FFFFFFFFFFFFFFFFFFFFFFFFFFFFFFFF74
:10A4F800FFFFFFFFFFFFFFFFFFFFFFFFFFFFFFFF64
:10A50800FFFFFFFFFFFFFFFFFFFFFFFFFFFFFFFF53
:10A51800FFFFFFFFFFFFFFFFFFFFFFFFFFFFFF3F03
:10A52800FFFFFFFFFFFFFFFFFFFFFFFFFFFFFFFF33
:10A53800FFFFFFFFFFFFFFFFFFFFFFFFFFFFFFFF23
:10A54800FFFFFFFFFFFFFFFFFFFFFFFFFFFFFFFF13
:10A55800FFFFFFFFFFFFFFFFFFFFFFFFFFFFFFFF03
:10A56800FFFFFFFFFFFFFFFFFFFFFFFFFFFFFFFFF3
:10A57800FFFFFFFFFFFFFFFFFFFFFFFFFFFFFF3FA3
:10A58800FFFFFFFFFFFFFFFFFFFFFFFFFFFFFFFFD3
:10A59800FFFFFFFFFFFFFFFFFFFFFFFFFFFFFFFFC3
:10A5A800FFFFFFFFFFFFFFFFFFFFFFFFFFFFFFFFB3
:10A5B800FFFFFFFFFFFFFFFFFFFFFFFFFFFFFFFFA3
:10A5C800FFFFFFFFFFFFFFFFFFFFFFFFFFFFFFFF93
:10A5D800FFFFFFFFFFFFFFFFFFFFFFFFFFFFFF3F43
:10A5E800FFFFFFFFFFFFFFFFFFFFFFFFFFFFFFFF73
:10A5F800FFFFFFFFFFFFFFFFFFFFFFFFFFFFFFFF63
:10A60800FFFFFFFFFFFFFFFFFFFFFFFFFFFFFFFF52
:10A61800FFFFFFFFFFFFFFFFFFFFFFFFFFFFFFFF42
:10A62800FFFFFFFFFFFFFFFFFFFFFFFFFFFFFFFF32
:10A63800FFFFFFFFFFFFFFFFFFFFFFFFFFFFFF3FE2
:10A64800FFFFFFFFFFFFFFFFFFFFFFFFFFFFFFFF12
:10A65800FFFFFFFFFFFFFFFFFFFFFFFFFFFFFFFF02
:10A66800FFFFFFFFFFFFFFFFFFFFFFFFFFFFFFFFF2
:10A67800FFFFFFFFFFFFFFFFFFFFFFFFFFFFFFFFE2
:10A68800FFFFFFFFFFFFFFFFFFFFFFFFFFFFFFFFD2
:10A69800FFFFFFFFFFFFFFFFFFFFFFFFFFFFFF3F82
:10A6A800FFFFFFFFFFFFFFFFFFFFFFFFFFFFFFFFB2
:10A6B800FFFFFFFFFFFFFFFFFFFFFFFFFFFFFFFFA2
:10A6C800FFFFFFFFFFFFFFFFFFFFFFFFFFFFFFFF92
:10A6D800FFFFFFFFFFFFFFFFFFFFFFFFFFFFFFFF82
:10A6E800FFFFFFFFFFFFFFFFFFFFFFFFFFFFFFFF72
:10A6F800FFFFFFFFFFFFFFFFFFFFFFFFFFFFFF3F22
:10A70800FFFFFFFFFFFFFFFFFFFFFFFFFFFFFFFF51
:10A71800FFFFFFFFFFFFFFFFFFFFFFFFFFFFFFFF41
:10A72800FFFFFFFFFFFFFFFFFFFFFFFFFFFFFFFF31
:10A73800FFFFFFFFFFFFFFFFFFFFFFFFFFFFFFFF21
:10A74800FFFFFFFFFFFFFFFFFFFFFFFFFFFFFFFF11
:10A75800FFFFFFFFFFFFFFFFFFFFFFFFFFFFFF3FC1
:10A76800FFFFFFFFFFFFFFFFFFFFFFFFFFFFFFFFF1
:10A77800FFFFFFFFFFFFFFFFFFFFFFFFFFFFFFFFE1
:10A78800FFFFFFFFFFFFFFFFFFFFFFFFFFFFFFFFD1
:10A79800FFFFFFFFFFFFFFFFFFFFFFFFFFFFFFFFC1
:10A7A800FFFFFFFFFFFFFFFFFFFFFFFFFFFFFFFFB1
:10A7B800FFFFFFFFFFFFFFFFFFFFFFFFFFFFFF3F61
:10A7C800FFFFFFFFFFFFFFFFFFFFFFFFFFFFFFFF91
:10A7D800FFFFFFFFFFFFFFFFFFFFFFFFFFFFFFFF81
:10A7E800FFFFFFFFFFFFFFFFFFFFFFFFFFFFFFFF71
:10A7F800FFFFFFFFFFFFFFFFFFFFFFFFFFFFFFFF61
:10A80800FFFFFFFFFFFFFFFFFFFFFFFFFFFFFFFF50
:10A81800FFFFFFFFFFFFFFFFFFFFFFFFFFFFFF3F00
:10A82800FFFFFFFFFFFFFFFFFFFFFFFFFFFFFFFF30
:10A83800FFFFFFFFFFFFFFFFFFFFFFFFFFFFFFFF20
:10A84800FFFFFFFFFFFFFFFFFFFFFFFFFFFFFFFF10
:10A85800FFFFFFFFFFFFFFFFFFFFFFFFFFFFFFFF00
:10A86800FFFFFFFFFFFFFFFFFFFFFFFFFFFFFFFFF0
:10A87800FFFFFFFFFFFFFFFFFFFFFFFFFFFFFF3FA0
:10A88800FFFFFFFFFFFFFFFFFFFFFFFFFFFFFFFFD0
:10A89800FFFFFFFFFFFFFFFFFFFFFFFFFFFFFFFFC0
:10A8A800FFFFFFFFFFFFFFFFFFFFFFFFFFFFFFFFB0
:10A8B800FFFFFFFFFFFFFFFFFFFFFFFFFFFFFFFFA0
:10A8C800FFFFFFFFFFFFFFFFFFFFFFFFFFFFFFFF90
:10A8D800FFFFFFFFFFFFFFFFFFFFFFFFFFFFFF3F40
:10A8E800FFFFFFFFFFFFFFFFFFFFFFFFFFFFFFFF70
:10A8F800FFFFFFFFFFFFFFFFFFFFFFFFFFFFFFFF60
:10A90800FFFFFFFFFFFFFFFFFFFFFFFFFFFFFFFF4F
:10A91800FFFFFFFFFFFFFFFFFFFFFFFFFFFFFFFF3F
:10A92800FFFFFFFFFFFFFFFFFFFFFFFFFFFFFFFF2F
:10A93800FFFFFFFFFFFFFFFFFFFFFFFFFFFFFF3FDF
:10A94800FFFFFFFFFFFFFFFFFFFFFFFFFFFFFFFF0F
:10A95800FFFFFFFFFFFFFFFFFFFFFFFFFFFFFFFFFF
:10A96800FFFFFFFFFFFFFFFFFFFFFFFFFFFFFFFFEF
:10A97800FFFFFFFFFFFFFFFFFFFFFFFFFFFFFFFFDF
:10A98800FFFFFFFFFFFFFFFFFFFFFFFFFFFFFFFFCF
:10A99800FFFFFFFFFFFFFFFFFFFFFFFFFFFFFF3F7F
:10A9A800FFFFFFFFFFFFFFFFFFFFFFFFFFFFFFFFAF
:10A9B800FFFFFFFFFFFFFFFFFFFFFFFFFFFFFFFF9F
:10A9C800FFFFFFFFFFFFFFFFFFFFFFFFFFFFFFFF8F
:10A9D800FFFFFFFFFFFFFFFFFFFFFFFFFFFFFFFF7F
:10A9E800FFFFFFFFFFFFFFFFFFFFFFFFFFFFFFFF6F
:10A9F800FFFFFFFFFFFFFFFFFFFFFFFFFFFFFF3F1F
:10AA0800FFFFFFFFFFFFFFFFFFFFFFFFFFFFFFFF4E
:10AA1800FFFFFFFFFFFFFFFFFFFFFFFFFFFFFFFF3E
:10AA2800FFFFFFFFFFFFFFFFFFFFFFFFFFFFFFFF2E
:10AA3800FFFFFFFFFFFFFFFFFFFFFFFFFFFFFFFF1E
:10AA4800FFFFFFFFFFFFFFFFFFFFFFFFFFFFFFFF0E
:10AA5800FFFFFFFFFFFFFFFFFFFFFFFFFFFFFF3FBE
:10AA6800FFFFFFFFFFFFFFFFFFFFFFFFFFFFFFFFEE
:10AA7800FFFFFFFFFFFFFFFFFFFFFFFFFFFFFFFFDE
:10AA8800FFFFFFFFFFFFFFFFFFFFFFFFFFFFFFFFCE
:10AA9800FFFFFFFFFFFFFFFFFFFFFFFFFFFFFFFFBE
:10AAA800FFFFFFFFFFFFFFFFFFFFFFFFFFFFFFFFAE
:10AAB800FFFFFFFFFFFFFFFFFFFFFFFFFFFFFF3F5E
:10AAC800FFFFFFFFFFFFFFFFFFFFFFFFFFFFFFFF8E
:10AAD800FFFFFFFFFFFFFFFFFFFFFFFFFFFFFFFF7E
:10AAE800FFFFFFFFFFFFFFFFFFFFFFFFFFFFFFFF6E
:10AAF800FFFFFFFFFFFFFFFFFFFFFFFFFFFFFFFF5E
:10AB0800FFFFFFFFFFFFFFFFFFFFFFFFFFFFFFFF4D
:10AB1800FFFFFFFFFFFFFFFFFFFFFFFFFFFFFF3FFD
:10AB2800FFFFFFFFFFFFFFFFFFFFFFFFFFFFFFFF2D
:10AB3800FFFFFFFFFFFFFFFFFFFFFFFFFFFFFFFF1D
:10AB4800FFFFFFFFFFFFFFFFFFFFFFFFFFFFFFFF0D
:10AB5800FFFFFFFFFFFFFFFFFFFFFFFFFFFFFFFFFD
:10AB6800FFFFFFFFFFFFFFFFFFFFFFFFFFFFFFFFED
:10AB7800FFFFFFFFFFFFFFFFFFFFFFFFFFFFFF3F9D
:10AB8800FFFFFFFFFFFFFFFFFFFFFFFFFFFFFFFFCD
:10AB9800FFFFFFFFFFFFFFFFFFFFFFFFFFFFFFFFBD
:10ABA800FFFFFFFFFFFFFFFFFFFFFFFFFFFFFFFFAD
:10ABB800FFFFFFFFFFFFFFFFFFFFFFFFFFFFFFFF9D
:10ABC800FFFFFFFFFFFFFFFFFFFFFFFFFFFFFFFF8D
:10ABD800FFFFFFFFFFFFFFFFFFFFFFFFFFFFFF3F3D
:10ABE800FFFFFFFFFFFFFFFFFFFFFFFFFFFFFFFF6D
:10ABF800FFFFFFFFFFFFFFFFFFFFFFFFFFFFFFFF5D
:10AC0800FFFFFFFFFFFFFFFFFFFFFFFFFFFFFFFF4C
:10AC1800FFFFFFFFFFFFFFFFFFFFFFFFFFFFFFFF3C
:10AC2800FFFFFFFFFFFFFFFFFFFFFFFFFFFFFFFF2C
:10AC3800FFFFFFFFFFFFFFFFFFFFFFFFFFFFFF3FDC
:10AC4800FFFFFFFFFFFFFFFFFFFFFFFFFFFFFFFF0C
:10AC5800FFFFFFFFFFFFFFFFFFFFFFFFFFFFFFFFFC
:10AC6800FFFFFFFFFFFFFFFFFFFFFFFFFFFFFFFFEC
:10AC7800FFFFFFFFFFFFFFFFFFFFFFFFFFFFFFFFDC
:10AC8800FFFFFFFFFFFFFFFFFFFFFFFFFFFFFFFFCC
:10AC9800FFFFFFFFFFFFFFFFFFFFFFFFFFFFFF3F7C
:10ACA800FFFFFFFFFFFFFFFFFFFFFFFFFFFFFFFFAC
:10ACB800FFFFFFFFFFFFFFFFFFFFFFFFFFFFFFFF9C
:10ACC800FF0F0000000000000000E0FFFFFFFFFF93
:10ACD800FFFFFFFFFFFFFFFFFFFFFFFFFFFFFFFF7C
:10ACE800FFFFFFFFFFFFFFFFFFFFFFFFFFFFFFFF6C
:10ACF800FFFFFFFFFFFFFFFFFFFFFFFFFFFFFF3F1C
:10AD0800FFFFFFFFFFFFFFFFFFFFFFFFFFFFFFFF4B
:10AD1800FFFFFFFFFFFFFFFFFFFFFFFFFFFFFFFF3B
:10AD2800FF0F0000000000000000E0FFFFFFFFFF32
:10AD3800FFFFFFFFFFFFFFFFFFFFFFFFFFFFFFFF1B
:10AD4800FFFFFFFFFFFFFFFFFFFFFFFFFFFFFFFF0B
:10AD5800FFFFFFFFFFFFFFFFFFFFFFFFFFFFFF3FBB
:10AD6800FFFFFFFFFFFFFFFFFFFFFFFFFFFFFFFFEB
:10AD7800FFFFFFFFFFFFFFFFFFFFFFFFFFFFFFFFDB
:10AD8800FF0F0000000000000000E0FFFFFFFFFFD2
:10AD9800FFFFFFFFFFFFFFFFFFFFFFFFFFFFFFFFBB
:10ADA800FFFFFFFFFFFFFFFFFFFFFFFFFFFFFFFFAB
:10ADB800FFFFFFFFFFFFFFFFFFFFFFFFFFFFFF3F5B
:10ADC800FFFFFFFFFFFFFFFFFFFFFFFFFFFFFFFF8B
:10ADD800FFFFFFFFFFFFFFFFFFFFFFFFFFFFFFFF7B
:10ADE800FF0F0000000000000000E0FFFFFFFFFF72
:10ADF800FFFFFFFFFFFFFFFFFFFFFFFFFFFFFFFF5B
:10AE0800FFFFFFFFFFFFFFFFFFFFFFFFFFFFFFFF4A
:10AE1800FFFFFFFFFFFFFFFFFFFFFFFFFFFFFF3FFA
:10AE2800FFFFFFFFFFFFFFFFFFFFFFFFFFFFFFFF2A
:10AE3800FFFFFFFFFFFFFFFFFFFFFFFFFFFFFFFF1A
:10AE4800FF0F0000000000000000E0FFFFFFFFFF11
:10AE5800FFFFFFFFFFFFFFFFFFFFFFFFFFFFFFFFFA
:10AE6800FFFFFFFFFFFFFFFFFFFFFFFFFFFFFFFFEA
:10AE7800FFFFFFFFFFFFFFFFFFFFFFFFFFFFFF3F9A
:10AE8800FFFFFFFFFFFFFFFFFFFFFFFFFFFFFFFFCA
:10AE9800FFFFFFFFFFFFFFFFFFFFFFFFFFFFFFFFBA
:10AEA800FF0FE0FF1F0000700000E0FFFFFFFFFF43
:10AEB800FFFFFFFFFFFFFFFFFFFFFFFFFFFFFFFF9A
:10AEC800FFFFFFFFFFFFFFFFFFFFFFFFFFFFFFFF8A
:10AED800FFFFFFFFFFFFFFFFFFFFFFFFFFFFFF3F3A
:10AEE800FFFFFFFFFFFFFFFFFFFFFFFFFFFFFFFF6A
:10AEF800FFFFFFFFFFFFFFFFFFFFFFFFFFFFFFFF5A
:10AF0800FF0FE0FF1F0080FF0000E0FFFFFFFFFFD3
:10AF1800FFFFFFFFFFFFFFFFFFFFFFFFFFFFFFFF39
:10AF2800FFFFFFFFFFFFFFFFFFFFFFFFFFFFFFFF29
:10AF3800FFFFFFFFFFFFFFFFFFFFFFFFFFFFFF3FD9
:10AF4800FFFFFFFFFFFFFFFFFFFFFFFFFFFFFFFF09
:10AF5800FFFFFFFFFFFFFFFFFFFFFFFFFFFFFFFFF9
:10AF6800FF0FE0FF1F00F8FF0000E0FFFFFFFFFFFB
:10AF7800FFFFFFFFFFFFFFFFFFFFFFFFFFFFFFFFD9
:10AF8800FFFFFFFFFFFFFFFFFFFFFFFFFFFFFFFFC9
:10AF9800FFFFFFFFFFFFFFFFFFFFFFFFFFFFFF3F79
:10AFA800FFFFFFFFFFFFFFFFFFFFFFFFFFFFFFFFA9
:10AFB800FFFFFFFFFFFFFFFFFFFFFFFFFFFFFFFF99
:10AFC800FF0FE0FF1F80F3FF0100E0FFFFFFFFFF1F
:10AFD800FFFFFFFFFFFFFFFFFFFFFFFFFFFFFFFF79
:10AFE800FFFFFFFFFFFFFFFFFFFFFFFFFFFFFFFF69
:10AFF800FFFFFFFFFFFFFFFFFFFFFFFFFFFFFF3F19
:10B00800FFFFFFFFFFFFFFFFFFFFFFFFFFFFFFFF48
:10B01800FFFFFFFFFFFFFFFFFFFFFFFFFFFFFFFF38
:10B02800FF0FE0FF1FF8F3FF0300E0FFFFFFFFFF44
:10B03800FFFFFFFFFFFFFFFFFFFFFFFFFFFFFFFF18
:10B04800FFFFFFFFFFFFFFFFFFFFFFFFFFFFFFFF08
:10B05800FFFFFFFFFFFFFFFFFFFFFFFFFFFFFF3FB8
:10B06800FFFFFFFFFFFFFFFFFFFFFFFFFFFFFFFFE8
:10B07800FFFFFFFFFFFFFFFFFFFFFFFFFFFFFFFFD8
:10B08800FF0FE0FF1FFEE3FF0700E0FFFFFFFFFFEA
:10B09800FFFFFFFFFFFFFFFFFFFFFFFFFFFFFFFFB8
:10B0A800FFFFFFFFFFFFFFFFFFFFFFFFFFFFFFFFA8
:10B0B800FFFFFFFFFFFFFFFFFFFFFFFFFFFFFF3F58
:10B0C800FFFFFFFFFFFFFFFFFFFFFFFFFFFFFFFF88
:10B0D800FFFFFFFFFFFFFFFFFFFFFFFFFFFFFFFF78
:10B0E800FF0FE0FFC0FFC3FF0700E0FFFFFFFFFF08
:10B0F800FFFFFFFFFFFFFFFFFFFFFFFFFFFFFFFF58
:10B10800FFFFFFFFFFFFFFFFFFFFFFFFFFFFFFFF47
:10B11800FFFFFFFFFFFFFFFFFFFFFFFFFFFFFF3FF7
:10B12800FFFFFFFFFFFFFFFFFFFFFFFFFFFFFFFF27
:10B13800FFFFFFFFFFFFFFFFFFFFFFFFFFFFFFFF17
:10B14800FF0FE00FC0FFC3FF0F00E0FFFFFFFFFF8F
:10B15800FFFFFFFFFFFFFFFFFFFFFFFFFFFFFFFFF7
:10B16800FFFFFFFFFFFFFFFFFFFFFFFFFFFFFFFFE7
:10B17800FFFFFFFFFFFFFFFFFFFFFFFFFFFFFF3F97
:10B18800FFFFFFFFFFFFFFFFFFFFFFFFFFFFFFFFC7
:10B19800FFFFFFFFFFFFFFFFFFFFFFFFFFFFFFFFB7
:10B1A800FF0FE001C0FF83FF1F00E0FFFFFFFFFF6D
:10B1B800FFFFFFFFFFFFFFFFFFFFFFFFFFFFFFFF97
:10B1C800FFFFFFFFFFFFFFFFFFFFFFFFFFFFFFFF87
:10B1D800FFFFFFFFFFFFFFFFFFFFFFFFFFFFFF3F37
:10B1E800FFFFFFFFFFFFFFFFFFFFFFFFFFFFFFFF67
:10B1F800FFFFFFFFFFFFFFFFFFFFFFFFFFFFFFFF57
:10B20800FF0F0000C0FF03FF1F00E0FFFFFFFFFF6D
:10B21800FFFFFFFFFFFFFFFFFFFFFFFFFFFFFFFF36
:10B22800FFFFFFFFFFFFFFFFFFFFFFFFFFFFFFFF26
:10B23800FFFFFFFFFFFFFFFFFFFFFFFFFFFFFF3FD6
:10B24800FFFFFFFFFFFFFFFFFFFFFFFFFFFFFFFF06
:10B25800FFFFFFFFFFFFFFFFFFFFFFFFFFFFFFFFF6
:10B26800FF0F0000C0FF03FE3F00E0FF0FFC3FFEA2
:10B27800FFFFFF7F3FC7FF3F3FFFFFFFFFFFFFFFCE
:10B28800FFFFFFFFFFFFFFFFFFFFFFFFFFFFFFFFC6
:10B29800FFFFFFFFFFFFFFFFFFFFFFFFFFFFFF3F76
:10B2A800FFFFFFFFFFFFFFFFFFFFFFFFFFFFFFFFA6
:10B2B800FFFFFFFFFFFFFFFFFFFFFFFFFFFFFFFF96
:10B2C800FF0F6000C0FF03FE7F00E0FF0FFC3FFEA2
:10B2D800FFFFFF7F3FC7FF3F3FFFFFFFFFFFFFFF6E
:10B2E800FFFFFFFFFFFFFFFFFFFFFFFFFFFFFFFF66
:10B2F800FFFFFFFFFFFFFFFFFFFFFFFFFFFFFF3F16
:10B30800FFFFFFFFFFFFFFFFFFFFFFFFFFFFFFFF45
:10B31800FFFFFFFFFFFFFFFFFFFFFFFFFFFFFFFF35
:10B32800FF0FE001C0FF03FCFF00E0FF3FFF9FFCB1
:10B33800FFFFFF3FFFCFFF1F1FFFFFFFFFFFFFFFC5
:10B34800FFFFFFFFFFFFFFFFFFFFFFFFFFFFFFFF05
:10B35800FFFFFFFFFFFFFFFFFFFFFFFFFFFFFF3FB5
:10B36800FFFFFFFFFFFFFFFFFFFFFFFFFFFFFFFFE5
:10B37800FFFFFFFFFFFFFFFFFFFFFFFFFFFFFFFFD5
:10B38800FF0FE007C0FF03F8FF00E0FF3FFF9FFC4F
:10B39800FFFFFF3FFFCFFF1F1FFFFFFFFFFFFFFF65
:10B3A800FFFFFFFFFFFFFFFFFFFFFFFFFFFFFFFFA5
:10B3B800FFFFFFFFFFFFFFFFFFFFFFFFFFFFFF3F55
:10B3C800FFFFFFFFFFFFFFFFFFFFFFFFFFFFFFFF85
:10B3D800FFFFFFFFFFFFFFFFFFFFFFFFFFFFFFF97B
:10B3E800FF0FE00FC0FF03F0FF01E0FF3F0F9E1FBC
:10B3F80046CE1C1E1CCFFC3F3FFFFFFFFFFFFFFF99
:10B40800FFFFFFFFFFFFFFFFFFFFFFFFFFFFFFFF44
:10B41800FFFFFFFFFFFFFFFFFFFFFFFFFFFFFF3FF4
:10B42800FFFFFFFFFFFFFFFFFFFFFFFFFFFFFFFF24
:10B43800FFFFFFFFFFFFFFFFFFFFFFFFFFFFFFF91A
:10B44800FF0FE03FC0FF03F0FF03E0FF3F0F9E1F29
:10B4580046CE1C1E1CCFFC3F3FFFFFFFFFFFFFFF38
:10B46800FFFFFFFFFFFFFFFFFFFFFFFFFFFFFFFFE4
:10B47800FFFFFFFFFFFFFFFFFFFFFFFFFFFFFF3F94
:10B48800FFFFFFFFFFFFFFFFFFFFFFFFFFFFFFFFC4
:10B49800FFFFFFFFFFFFFFFFFFFFFFFFFFFFFFFFB4
:10B4A800FF0FE07FC0FF03E0FF07E0FF3FCF0CCFB7
:10B4B8008C8CF83C3F4FFE3F3FFFFFFFFFFFFFFF35
:10B4C800FFFFFFFFFFFFFFFFFFFFFFFFFFFFFFFF84
:10B4D800FFFFFFFFFFFFFFFFFFFFFFFFFFFFFF3F34
:10B4E800FFFFFFFFFFFFFFFFFFFFFFFFFFFFFFFF64
:10B4F800FFFFFFFFFFFFFFFFFFFFFFFFFFFFFFFF54
:10B50800FF0FE0FFC1FF0FC0FF07E0FF3FCF0CCFE9
:10B518008C8CF83C3F4FFE3F3FFFFFFFFFFFFFFFD4
:10B52800FFFFFFFFFFFFFFFFFFFFFFFFFFFFFFFF23
:10B53800FFFFFFFFFFFFFFFFFFFFFFFFFFFFFF3FD3
:10B54800FFFFFFFFFFFFFFFFFFFFFFFFFFFFFFFF03
:10B55800FFFFFFFFFFFFFFFFFFFFFFFFFFFFFFFFF3
:10B56800FF0FE0FFC7FF3FC0FF0FE0FF3FCF9CCFBB
:10B57800CC4C393C3F0FFF3F3FFFFFFFFFFFFFFF72
:10B58800FFFFFFFFFFFFFFFFFFFFFFFFFFFFFFFFC3
:10B59800FFFFFFFFFFFFFFFFFFFFFFFFFFFFFF3F73
:10B5A800FFFFFFFFFFFFFFFFFFFFFFFFFFFFFFFFA3
:10B5B800FFFFFFFFFFFFFFFFFFFFFFFFFFFFFFFF93
:10B5C800FF0FE0FFDFFF7F80FF1FE0FF3FCF9CCF33
:10B5D800CC4C393C3F0FFF3F3FFFFFFFFFFFFFFF12
:10B5E800FFFFFFFFFFFFFFFFFFFFFFFFFFFFFFFF63
:10B5F800FFFFFFFFFFFFFFFFFFFFFFFFFFFFFF3F13
:10B60800FFFFFFFFFFFFFFFFFFFFFFFFFFFFFFFF42
:10B61800FFFFFFFFFFFFFFFFFFFFFFFFFFFFFFFF32
:10B62800FF0FE0FFFFFFFF01FF3FE0FF3FCF9CCF91
:10B63800CCCFC93C3D4FFE3F3FFFFFFFFFFFFFFF61
:10B64800FFFFFFFFFFFFFFFFFFFFFFFFFFFFFFFF02
:10B65800FFFFFFFFFFFFFFFFFFFFFFFFFFFFFF3FB2
:10B66800FFFFFFFFFFFFFFFFFFFFFFFFFFFFFFFFE2
:10B67800FFFFFFFFFFFFFFFFFFFFFFFFFFFFFFFFD2
:10B68800FF0FE0FFFFFFFF07FE3FE0FF3FCF9CCF2C
:10B69800CCCFC93C3D4FFE3F3FFFFFFFFFFFFFFF01
:10B6A800FFFFFFFFFFFFFFFFFFFFFFFFFFFFFFFFA2
:10B6B800FFFFFFFFFFFFFFFFFFFFFFFFFFFFFF3F52
:10B6C800FFFFFFFFFFFFFFFFFFFFFFFFFFFFFFFF82
:10B6D800FFFFFFFFFFFFFFFFFFFFFFFFFFFFFFFF72
:10B6E800FF0FE0FFFFFFFF0FFE3FE0FF0FCC0C1F37
:10B6F80086CF19791EC6FC0F0CFCFFFFFFFFFFFF6A
:10B70800FFFFFFFFFFFFFFFFFFFFFFFFFFFFFFFF41
:10B71800FFFFFFFFFFFFFFFFFFFFFFFFFFFFFF3FF1
:10B72800FFFFFFFFFFFFFFFFFFFFFFFFFFFFFFFF21
:10B73800FFFFFFFFFFFFFFFFFFFFFFFFFFFFFFFF11
:10B74800FF0FE0FFFFFFFF3FFC07E0FF0FCC0C1FE0
:10B7580086CF19791EC6FC0F0CFCFFFFFFFFFFFF09
:10B76800FFFFFFFFFFFFFFFFFFFFFFFFFFFFFFFFE1
:10B77800FFFFFFFFFFFFFFFFFFFFFFFFFFFFFF3F91
:10B78800FFFFFFFFFFFFFFFFFFFFFFFFFFFFFFFFC1
:10B79800FFFFFFFFFFFFFFFFFFFFFFFFFFFFFFFFB1
:10B7A800FF0FE0FFFFFFFFFF3800E0FFFFFFFFFF95
:10B7B800FFFFFFFFFFFFFFFFFFFFFFFFFFFFFF7F11
:10B7C800FEFFFFFFFFFFFFFFFFFFFFFFFFFFFFFF82
:10B7D800FFFFFFFFFFFFFFFFFFFFFFFFFFFFFF3F31
:10B7E800FFFFFFFFFFFFFFFFFFFFFFFFFFFFFFFF61
:10B7F800FFFFFFFFFFFFFFFFFFFFFFFFFFFFFFFF51
:10B80800FF0FE0FFFFFFFFFF0100E0FFFFFFFFFF6B
:10B81800FFFFFFFFFFFFFFFFFFFFFFFFFFFFFFFF30
:10B82800FFFFFFFFFFFFFFFFFFFFFFFFFFFFFFFF20
:10B83800FFFFFFFFFFFFFFFFFFFFFFFFFFFFFF3FD0
:10B84800FFFFFFFFFFFFFFFFFFFFFFFFFFFFFFFF00
:10B85800FFFFFFFFFFFFFFFFFFFFFFFFFFFFFFFFF0
:10B86800FF0FE0FFFFFFFB3F0000E0FFFFFFFFFFD0
:10B87800FFFFFFFFFFFFFFFFFFFFFFFFFFFFFFFFD0
:10B88800FFFFFFFFFFFFFFFFFFFFFFFFFFFFFFFFC0
:10B89800FFFFFFFFFFFFFFFFFFFFFFFFFFFFFF3F70
:10B8A800FFFFFFFFFFFFFFFFFFFFFFFFFFFFFFFFA0
:10B8B800FFFFFFFFFFFFFFFFFFFFFFFFFFFFFFFF90
:10B8C800FF0FE0FFFFFFF3070000E0FFFFFFFFFFB0
:10B8D800FFFFFFFFFFFFFFFFFFFFFFFFFFFFFFFF70
:10B8E800FFFFFFFFFFFFFFFFFFFFFFFFFFFFFFFF60
:10B8F800FFFFFFFFFFFFFFFFFFFFFFFFFFFFFF3F10
:10B90800FFFFFFFFFFFFFFFFFFFFFFFFFFFFFFFF3F
:10B91800FFFFFFFFFFFFFFFFFFFFFFFFFFFFFFFF2F
:10B92800FF0FE0FFFFFF43000000E0FFFFFFFFFF06
:10B93800FFFFFFFFFFFFFFFFFFFFFFFFFFFFFFFF0F
:10B94800FFFFFFFFFFFFFFFFFFFFFFFFFFFFFFFFFF
:10B95800FFFFFFFFFFFFFFFFFFFFFFFFFFFFFF3FAF
:10B96800FFFFFFFFFFFFFFFFFFFFFFFFFFFFFFFFDF
:10B97800FFFFFFFFFFFFFFFFFFFFFFFFFFFFFFFFCF
:10B98800FF0FE0FFFFFF03000000E0FFFFFFFFFFE6
:10B99800FFFFFFFFFFFFFFFFFFFFFFFFFFFFFFFFAF
:10B9A800FFFFFFFFFFFFFFFFFFFFFFFFFFFFFFFF9F
:10B9B800FFFFFFFFFFFFFFFFFFFFFFFFFFFFFF3F4F
:10B9C800FFFFFFFFFFFFFFFFFFFFFFFFFFFFFFFF7F
:10B9D800FFFFFFFFFFFFFFFFFFFFFFFFFFFFFFFF6F
:10B9E800FF0FE0FFFF7F00000000E0FFFFFFFFFF09
:10B9F800FFFFFFFFFFFFFFFFFFFFFFFFFFFFFFFF4F
:10BA0800FFFFFFFFFFFFFFFFFFFFFFFFFFFFFFFF3E
:10BA1800FFFFFFFFFFFFFFFFFFFFFFFFFFFFFF3FEE
:10BA2800FFFFFFFFFFFFFFFFFFFFFFFFFFFFFFFF1E
:10BA3800FFFFFFFFFFFFFFFFFF3FFFFFFFFFFFFFCE
:10BA4800FF0FE0FFFF0700000000E0FFFFFFFFFF20
:10BA5800FFFFFFFFFFFFFFFFFFFFFFFFFFFFFFFFEE
:10BA6800FFFFFFFFFFFFFFFFFFFFFFFFFFFFFFFFDE
:10BA7800FFFFFFFFFFFFFFFFFFFFFFFFFFFFFF3F8E
:10BA8800FFFFFFFFFFFFFFFFFFFFFFFFFFFFFFFFBE
:10BA9800FFFFFFFFFFFFFFFFFF3FFFFFFFFFFFFF6E
:10BAA800FF0FE0FF7F0000000000E0FFFFFFFFFF47
:10BAB800FFFFFFFFFFFFFFFFFFFFFFFFFFFFFFFF8E
:10BAC800FFFFFFFFFFFFFFFFFFFFFFFFFFFFFFFF7E
:10BAD800FFFFFFFFFFFFFFFFFFFFFFFFFFFFFF3F2E
:10BAE800FFFFFFFFFFFFFFFFFFFFFFFFFFFFFFFF5E
:10BAF800FFFFFFFFFFFFFFFFFFFFFFFFFFFFFFFF4E
:10BB0800FF0F0000000000000000E0FFFFFFFFFF44
:10BB1800FFFFFFFFFFFFFFFFFFFFFFFFFFFFFFFF2D
:10BB2800FFFFFFFFFFFFFFFFFFFFFFFFFFFFFFFF1D
:10BB3800FFFFFFFFFFFFFFFFFFFFFFFFFFFFFF3FCD
:10BB4800FFFFFFFFFFFFFFFFFFFFFFFFFFFFFFFFFD
:10BB5800FFFFFFFFFFFFFFFFFFFFFFFFFFFFFFFFED
:10BB6800FF0F0000000000000000E0FFFFFFFFFFE4
:10BB7800FFFFFFFFFFFFFFFFFFFFFFFFFFFFFFFFCD
:10BB8800FFFFFFFFFFFFFFFFFFFFFFFFFFFFFFFFBD
:10BB9800FFFFFFFFFFFFFFFFFFFFFFFFFFFFFF3F6D
:10BBA800FFFFFFFFFFFFFFFFFFFFFFFFFFFFFFFF9D
:10BBB800FFFFFFFFFFFFFFFFFFFFFFFFFFFFFFFF8D
:10BBC800FF0F0000000000000000E0FFFFFFFFFF84
:10BBD800FFFFFFFFFFFFFFFFFFFFFFFFFFFFFFFF6D
:10BBE800FFFFFFFFFFFFFFFFFFFFFFFFFFFFFFFF5D
:10BBF800FFFFFFFFFFFFFFFFFFFFFFFFFFFFFF3F0D
:10BC0800FFFFFFFFFFFFFFFFFFFFFFFFFFFFFFFF3C
:10BC1800FFFFFFFFFFFFFFFFFFFFFFFFFFFFFFFF2C
:10BC2800FF0F0000000000000000E0FFFFFFFFFF23
:10BC3800FFFFFFFFFFFFFFFFFFFFFFFFFFFFFFFF0C
:10BC4800FFFFFFFFFFFFFFFFFFFFFFFFFFFFFFFFFC
:10BC5800FFFFFFFFFFFFFFFFFFFFFFFFFFFFFF3FAC
:10BC6800FFFFFFFFFFFFFFFFFFFFFFFFFFFFFFFFDC
:10BC7800FFFFFFFFFFFFFFFFFFFFFFFFFFFFFFFFCC
:10BC8800FF0F0000000000000000E0FFFFFFFFFFC3
:10BC9800FFFFFFFFFFFFFFFFFFFFFFFFFFFFFFFFAC
:10BCA800FFFFFFFFFFFFFFFFFFFFFFFFFFFFFFFF9C
:10BCB800FFFFFFFFFFFFFFFFFFFFFFFFFFFFFF3F4C
:10BCC800FFFFFFFFFFFFFFFFFFFFFFFFFFFFFFFF7C
:10BCD800FFFFFFFFFFFFFFFFFFFFFFFFFFFFFFFF6C
:10BCE800FFFFFFFFFFFFFFFFFFFFFFFFFFFFFFFF5C
:10BCF800FFFFFFFFFFFFFFFFFFFFFFFFFFFFFFFF4C
:10BD0800FFFFFFFFFFFFFFFFFFFFFFFFFFFFFFFF3B
:10BD1800FFFFFFFFFFFFFFFFFFFFFFFFFFFFFF3FEB
:10BD2800FFFFFFFFFFFFFFFFFFFFFFFFFFFFFFFF1B
:10BD3800FFFFFFFFFFFFFFFFFFFFFFFFFFFFFFFF0B
:10BD4800FFFFFFFFFFFFFFFFFFFFFFFFFFFFFFFFFB
:10BD5800FFFFFFFFFFFFFFFFFFFFFFFFFFFFFFFFEB
:10BD6800FFFFFFFFFFFFFFFFFFFFFFFFFFFFFFFFDB
:10BD7800FFFFFFFFFFFFFFFFFFFFFFFFFFFFFF3F8B
:10BD8800FFFFFFFFFFFFFFFFFFFFFFFFFFFFFFFFBB
:10BD9800FFFFFFFFFFFFFFFFFFFFFFFFFFFFFFFFAB
:10BDA800FFFFFFFFFFFFFFFFFFFFFFFFFFFFFFFF9B
:10BDB800FFFFFFFFFFFFFFFFFFFFFFFFFFFFFFFF8B
:10BDC800FFFFFFFFFFFFFFFFFFFFFFFFFFFFFFFF7B
:10BDD800FFFFFFFFFFFFFFFFFFFFFFFFFFFFFF3F2B
:10BDE800FFFFFFFFFFFFFFFFFFFFFFFFFFFFFFFF5B
:10BDF800FFFFFFFFFFFFFFFFFFFFFFFFFFFFFFFF4B
:10BE0800FFFFFFFFFFFFFFFFFFFFFFFFFFFFFFFF3A
:10BE1800FFFFFFFFFFFFFFFFFFFFFFFFFFFFFFFF2A
:10BE2800FFFFFFFFFFFFFFFFFFFFFFFFFFFFFFFF1A
:10BE3800FFFFFFFFFFFFFFFFFFFFFFFFFFFFFF3FCA
:10BE4800FFFFFFFFFFFFFFFFFFFFFFFFFFFFFFFFFA
:10BE5800FFFFFFFFFFFFFFFFFFFFFFFFFFFFFFFFEA
:10BE6800FFFFFFFFFFFFFFFFFFFFFFFFFFFFFFFFDA
:10BE7800FFFFFFFFFFFFFFFFFFFFFFFFFFFFFFFFCA
:10BE8800FFFFFFFFFFFFFFFFFFFFFFFFFFFFFFFFBA
:10BE9800FFFFFFFFFFFFFFFFFFFFFFFFFFFFFF3F6A
:10BEA800FFFFFFFFFFFFFFFFFFFFFFFFFFFFFFFF9A
:10BEB800FFFFFFFFFFFFFFFFFFFFFFFFFFFFFFFF8A
:10BEC800FFFFFFFFFFFFFFFFFFFFFFFFFFFFFFFF7A
:10BED800FFFFFFFFFFFFFFFFFFFFFFFFFFFFFFFF6A
:10BEE800FFFFFFFFFFFFFFFFFFFFFFFFFFFFFFFF5A
:10BEF800FFFFFFFFFFFFFFFFFFFFFFFFFFFFFF3F0A
:10BF0800FFFFFFFFFFFFFFFFFFFFFFFFFFFFFFFF39
:10BF1800FFFFFFFFFFFFFFFFFFFFFFFFFFFFFFFF29
:10BF2800FFFFFFFFFFFFFFFFFFFFFFFFFFFFFFFF19
:10BF3800FFFFFFFFFFFFFFFFFFFFFFFFFFFFFFFF09
:10BF4800FFFFFFFFFFFFFFFFFFFFFFFFFFFFFFFFF9
:10BF5800FFFFFFFFFFFFFFFFFFFFFFFFFFFFFF3FA9
:10BF6800FFFFFFFFFFFFFFFFFFFFFFFFFFFFFFFFD9
:10BF7800FFFFFFFFFFFFFFFFFFFFFFFFFFFFF7FFD1
:10BF8800FFFFFFFFFFFFFFFFFFFFFFFFFFFFFFFFB9
:10BF9800FFFFFFFFFFFFFFFFFFFFFFFFFFFFFFFFA9
:10BFA800FFFFFFFFFFFFFFFFFFFFFFFFFFFFFFFF99
:10BFB800FFFFFFFFFFFFFFFFFFFFFFFFFFFFFF3F49
:10BFC800FFFFFFFFFFFFFFFFFFFFFFFFFFFFFFFF79
:10BFD800FFFFFFFFFFFFFFFFFFFFFFFFFFFFF7FF71
:10BFE800FFFFFFFFFFFFFFFFFFFFFFFFFFFFFFFF59
:10BFF800FFFFFFFFFFFFFFFFFFFFFFFFFFFFFFFF49
:10C00800FFFFFFFFFFFFFFFFFFFFFFFFFFFFFFFF38
:10C01800FFFFFFFFFFFFFFFFFFFFFFFFFFFFFF3FE8
:10C02800FFFFFFFFFFFFFFFFFFFFFFFFFFFFFFFF18
:10C03800FFFFFFFFFFFFFFFFFFFFFFFFFFFFFFFF08
:10C04800FFFFFFFFFFFFFFFFFFFFFFFFFFFFFFFFF8
:10C05800FFFFFFFFFFFFFFFFFFFFFFFFFFFFFFFFE8
:10C06800FFFFFFFFFFFFFFFFFFFFFFFFFFFFFFFFD8
:10C07800FFFFFFFFFFFFFFFFFFFFFFFFFFFFFF3F88
:10C08800FFFFFFFFFFFFFFFFFFFFFFFFFFFFFFFFB8
:10C09800FFFFFFFFFFFFFFFFFFFFFFFFFFFFFFFFA8
:10C0A800FFFFFFFFFFFFFFFFFFFFFFFFFFFFFFFF98
:10C0B800FFFFFFFFFFFFFFFFFFFFFFFFFFFFFFFF88
:10C0C800FFFFFFFFFFFFFFFFFFFFFFFFFFFFFFFF78
:10C0D800FFFFFFFFFFFFFFFFFFFFFFFFFFFFFF3F28
:10C0E800FFFFFFFFFFFFFFFFFFFFFFFFFFFFFFFF58
:10C0F800FFFFFFFFFFFFFFFFFFFFFFFFFFFFFFFF48
:10C10800FFFFFFFFFFFFFFFFFFFFFFFFFFFFFFFF37
:10C11800FFFFFFFFFFFFFFFFFFFFFFFFFFFFFFFC2A
:10C12800FFFFFFFFFFFFFFFFFFFFFFFFFFFFFFFF17
:10C13800FFFFFFFFFFFFFFFFFFFFFFFFFFFFFF3FC7
:10C14800FFFFFFFFFFFFFFFFFFFFFFFFFFFFFFFFF7
:10C15800FFFFFFFFFFFFFFFFFFFFFFFFFFFFFFFFE7
:10C16800FFFFFFFFFFFFFFFFFFFFFFFFFFFFFFFFD7
:10C17800FFFFFFFFFFFFFFFFFFFFFFFFFFFFFFFFC7
:10C18800FFFFFFFFFFFFFFFFFFFFFFFFFFFFFFFFB7
:10C19800FFFFFFFFFFFFFFFFFFFFFFFFFFFFFF3F67
:10C1A800FFFFFFFFFFFFFFFFFFFFFFFFFFFFFFFF97
:10C1B800FFFFFFFFFFFFFFFFFFFFFFFFFFFFFFFF87
:10C1C800FFFFFFFFFFFFFFFFFFFFFFFFFFFFFFFF77
:10C1D800FFFFFFFFFFFFFFFFFFFFFFFFFFFFFFFF67
:10C1E800FFFFFFFFFFFFFFFFFFFFFFFFFFFFFFFF57
:10C1F800FFFFFFFFFFFFFFFFFFFFFFFFFFFFFF3F07
:10C20800FFFFFFFFFFFFFFFFFFFFFFFFFFFFFFFF36
:10C21800FFFFFFFFFFFFFFFFFFFFFFFFFFFFFFFF26
:10C22800FFFFFFFFFFFFFFFFFFFFFFFFFFFFFFFF16
:10C23800FFFFFFFFFFFFFFFFFFFFFFFFFFFFFFFF06
:10C24800FFFFFFFFFFFFFFFFFFFFFEFFFFFFFFFFF7
:10C25800FFFFFFFFFFFFFFFFFFFFFFFFFFFFFF3FA6
:10C26800FFFFFFFFFFFFFFFFFFFFFFFFFFFFFFFFD6
:10C27800FFFFFFFFFFFFFFFFFFFFFFFFFFFFFFFFC6
:10C28800FFFFFFFFFFFFFFFFFFFFFFFFFFFFFFFFB6
:10C29800FFFFFFFFFFFFBFFFFFFFFFFFFFFFFFFFE6
:10C2A800FFFFFFFFFFFFFFFFFFFFFEFFFFFFFFFF97
:10C2B800FFFFFFFFFFFFFFFFFFFFFFFFFFFFFF3F46
:10C2C800FFFFFFFFFFFFFFFFFFFFFFFFFFFFFFFF76
:10C2D800FFFFFFFFFFFFFFFFFFFFFFFFFFFFFFFF66
:10C2E800FFFFFFFFFFFFFFFFFFFFFFFFFFFFEFFF66
:10C2F800FFFFFFFFFFFFBFFFFFFFFFFFFFFFFFFF86
:10C30800FFFFFFFFFFFFFFFFFFFFFFFFFFFFFFFF35
:10C31800FFFFFFFFFFFFFFFFFFFFFFFFFFFFFF3FE5
:10C32800FFFFFFFFFFFFFFFFFFFFFFFFFFFFFFFF15
:10C33800FFFFFFFFFFFFFFFFFFFFFFFFFFFFFFFF05
:10C34800FFFFFFFFFFFFFFFFFFFFFFFFFFFFEFFF05
:10C35800FFFFFFFFFFFFFFFFFFFFFFFFFFFFFFFFE5
:10C36800FFFFFFFFFFFFFFFFFFFFFFFFFFFFFFFFD5
:10C37800FFFFFFFFFFFFFFFFFFFFFFFFFFFFFF3F85
:10C38800FFFFFFFFFFFFFFFFFFFFFFFFFFFFFFFFB5
:10C39800FFFFFFFFFFFFFFFFFFFFFFFFFFFFFFFFA5
:10C3A800FFFFFFFFFFFFFFFFFFFFFFFFFFFFFFFF95
:10C3B800FFFFFFFFFFFFFFFFFFFFFFFFFFFFFFFF85
:10C3C800FFFFFFFFFFFFFFFFFFFFFFFFFFFFFFFF75
:10C3D800FFFFFFFFFFFFFFFFFFFFFFFFFFFFFF3F25
:10C3E800FFFFFFFFFFFFFFFFFFFFFFFFFFFFFFFF55
:10C3F800FFFFFFFFFFF7FFFFFFFFFBFFFFFFFFFF51
:10C40800FFFFFFFFFFFFFFFDFFFFFFFFFFFFFFFF36
:10C41800FFFFFFFFFFFFFFFFFFFFFFFFFFFFFFFF24
:10C42800FFFFFFFFFFFFFFFFFFFFFFFFFFFFFFFF14
:10C43800FFFFFFFFFFFFFFFFFFFFFFFFFFFFFF3FC4
:10C44800FFFFFFFFFFFFFFFFFFFFFFFFFFFFFFFFF4
:10C45800FFFFFFFFFFFFFFFFFFFFFBFFFFFFFFFFE8
:10C46800FFFFFFFFFFFFFFFDFFFFFFFFFFFFFFFFD6
:10C47800FFFFFFFFFFFFFFFFFFFFFFFFFFFFFFFFC4
:10C48800FFFFFFFFFFFFFFFFFFFFFFFFFFFFFFFFB4
:10C49800FFFFFFFFFFFFFFFFFFFFFFFFFFFFFF3F64
:10C4A800FFFFFFFFFFFFFFFFFFFFFFFFFFFFFFFF94
:10C4B800FFFFFFFFFFFFFFFFFFFFFFFFFFFFFFFF84
:10C4C800FFFFFFFFFFFFFFFFFFFFFFFFFFFFFFFF74
:10C4D800FFFFFFFFFFFFFFFFFFFFFFFFFFFFFFFF64
:10C4E800FFFFFFFFFFFFFFFFFFFFFFFFFFFFFFFF54
:10C4F800FFFFFFFFFFFFFFFFFFFFFFFFFFFFFF3F04
:10C50800FFFFFFFFFFFFFFFFFFFFFFFFFFFFFFFF33
:10C51800FFFFFFFFFFFFFFFFFFFFFFFFFFFFFFFF23
:10C52800FFFFFFFFFFFFFFFFFFFFFFFFFFFFFFFF13
:10C53800FFFFFFFFFFFFFFFFFFFFFFFFFFFFFFFF03
:10C54800FFFFFFFFFFFFFFFFFFFFFFFFFFFFFFFFF3
:10C55800FFFFFFFFFFFFFFFFFFFFFFFFFFFFFF3FA3
:10C56800FFFFFFFFFFFFFFFFFFFFFFFFFFFFFFFFD3
:10C57800FFFFFFFFFFFFFFFFFFFFFFFFFFFFFFFFC3
:10C58800FFFFFFFFFFFFFFFFFFFFFFFFFFFFFFFFB3
:10C59800FFFFFFFFFFFFFFFFFFFFFFFFFFFFFFFFA3
:10C5A800FFFFFFFFFFFFFFFFFFFFFFFFFFFFFFFF93
:10C5B800FFFFFFFFFFFFFFFFFFFFFFFFFFFFFF3F43
:10C5C800FFFFFFFFFFFFFFFFFFFFFFFFFFFFFFFF73
:10C5D800FFFFFFFFFFFFFFFFFFFFFFFFFFFFFFFF63
:10C5E800FFFFFFFFFFFFFFFFFFFFFFFFFFFFFFFF53
:10C5F800FFFFFFFFFFFFFFFFFFEFFFFFFFFFFFFF53
:10C60800FFFFFFFFFFFFFFFFFFFFFFFFFFFFFFFF32
:10C61800FFFFFFFFFFFFFFFFFFFFFFFFFFFFFF3FE2
:10C62800FFFFFFFFFFFFFFFFFFFFFFFFFFFFFFFF12
:10C63800FFFFFFFFFFFFFFFFFFFFFFFFFFFFFFFF02
:10C64800FFFFFFFFFFFFFFFFFFFFFFFFFFFFFFFFF2
:10C65800FFFFFFFFFFFFFFFFFFEFFFFFFFFFFFFFF2
:10C66800FFFFFDFFFFFFFFFFFFFFFFFFFFFFFFFFD4
:10C67800FFFFFFFFFFFFFFFFFFFFFFFFFFFFFF3F82
:10C68800FFFFFFFFFFFFFFFFFFFFFFFFFFFFFFFFB2
:10C69800FFFFFFFFFFFFFFFFFFFFFFFFFFFFFFFFA2
:10C6A800FFFFFFFFFFFFFFFFFFFFFFFFFFFFFFFF92
:10C6B800FFFFFFFFFFFFFFFFFFFFFFFFFFFFFFFF82
:10C6C800FFFFFFFFFFFFFFFFFFFFFFFFFFFFFFFF72
:10C6D800FFFFFFFFFFFFFFFFFFFFFFFFFFFFFF3F22
:10C6E800FFFFFFFFFFFFFFFFFFFFFFFFFFFFFFFF52
:10C6F800FFFFFFFFFFFFFFFFFFFFFFFFFFFFFFFF42
:10C70800FFFFFFFFFFFFFFFFFFFFFFFFFFFFFFFF31
:10C71800FFFFFFFFFFFFFFFFFFFFFFFFFFFFFFFF21
:10C72800FFFFFFFFFFFFFFFFFFFFFFFFFFFFFFFF11
:10C73800FFFFFFFFFFFFFFFFFFFFFFFFFFFFFF3FC1
:10C74800FFFFFFFFFFFFFFFFFFFFFFFFFFFFFFFFF1
:10C75800FFFFFFFFFFFFFFFFFFFFFFFFFFFFFFFFE1
:10C76800FFFFFFFFFFFFFFFFFFFFFFFFFFFFFFFFD1
:10C77800FFFFFFFFFFFFFFFFFFFFFFFFFFFFFFFFC1
:10C78800FFFFFFFFFFFFFFFFFFFFFFFFFFFFFFFFB1
:10C79800FFFFFFFFFFFFFFFFFFFFFFFFFFFFFF3F61
:10C7A800FFFFFFFFFFFFFFFFFFFFFFFFFFFFFFFF91
:10C7B800FFFFFFFFFFFFFFFFE3FF1FFFFFFFFFFF7D
:10C7C800FFFFFFFFFFFFFFFFFFFFFFFFFFFFFFFF71
:10C7D800FFFFFFFFFFFFFFFFFFFFFFFFFFFFFFFF61
:10C7E800FFFFFFFFFFFFFFFFFFFFFFFFFFFFFFFF51
:10C7F800FFFFFFFFFFFFFFFFFFFFFFFFFFFFFF3F01
:10C80800FFFFFFFFFFFFFFFFFFFFFFFFFFFFFFFF30
:10C81800FFFFFFFFFFFFFFFFE3FF1FFFFFFFFFFF1C
:10C82800FFFFFFFFFFFFFFFFFFFFFFFFFFFFFFFF10
:10C83800FFFFFFFFFFFFFFFFFFFFFFFFFFFFFFFF00
:10C84800FFFFFFFFFFFFFFFFFFFFFFFFFFFFFFFFF0
:10C85800FFFFFFFFFFFFFFFFFFFFFFFFFFFFFF3FA0
:10C86800FFFFFFFFFFFFFFFFFFFFFFFFFFFFFFFFD0
:10C87800FFFFFFFFFFFFFFFFE3FF1FFFFFFFFFFFBC
:10C88800FFFFFFFFFFFFFFFFFFFFFFFFFFFFFFFFB0
:10C89800FFFFFFFFFFFFFFFFFFFFFFFFFFFFFFFFA0
:10C8A800FFFFFFFFFFFFFFFFFFFFFFFFFFFFFFFF90
:10C8B800FFFFFFFFFFFFFFFFFFFFFFFFFFFFFF3F40
:10C8C800FFFFFFFFFFFFFFFFFFFFFFFFFFFFFFFF70
:10C8D800FFFFFFFFFFFFFFFF1FFFE3FFFFFFFFFF5C
:10C8E800FFFFFFFFFFFFFFFFFFFFFFFFFFFFFFFF50
:10C8F800FFFFFFFFFFFFFFFFFFFFFFFFFFFFFFFF40
:10C90800FFFFFFFFFFFFFFFFFFFFFFFFFFFFFFFF2F
:10C91800FFFFFFFFFFFFFFFFFFFFFFFFFFFFFF3FDF
:10C92800FFFFFFFFFFFFFFFFFFFFFFFFFFFFFFFF0F
:10C93800FFFFFFFFFFFFFFFF1FFFE3FFFFFFFFFFFB
:10C94800FFFFFFFFFFFFFFFFFFFFFFFFFFFFFFFFEF
:10C95800FFFFFFFFFFFFFFFFFFFFFFFFFFFFFFFFDF
:10C96800FFFFFFFFFFFFFFFFFFFFFFFFFFFFFFFFCF
:10C97800FFFFFFFFFFFFFFFFFFFFFFFFFFFFFF3F7F
:10C98800FFFFFFFFFFFFFFFFFFFFFFFFFFFFFFFFAF
:10C99800FFFFFFFFFFFFFFFF1FFFE3FFFFFFFFFF9B
:10C9A800FFFFFFFFFFFFFFFFFFFFFFFFFFFFFFFF8F
:10C9B800FFFFFFFFFFFFFFFFFFFFFFFFFFFFFFFF7F
:10C9C800FFFFFFFFFFFFFFFFFFFFFFFFFFFFFFFF6F
:10C9D800FFFFFFFFFFFFFFFFFFFFFFFFFFFFFF3F1F
:10C9E800FFFFFFFFFFFFFFFFFFFFFFFFFFFFFFFF4F
:10C9F800FFFFFFFFFFFFFFFF030000FFFFFFFFFF39
:10CA0800FFFFFFFFFFFFFFFFFFFFFFFFFFFFFFFF2E
:10CA1800FFFFFFFFFFFFFFFFFFFFFFFFFFFFFFFF1E
:10CA2800FFFFFFFFFFFFFFFFFFFFFFFFFFFFFFFF0E
:10CA3800FFFFFFFFFFFFFFFFFFFFFFFFFFFFFF3FBE
:10CA4800FFFFFFFFFFFFFFFFFFFFFFFFFFFFFFFFEE
:10CA5800FFFFFFFFFFFFFFFF030000FFFFFFFFFFD8
:10CA6800FFFFFFFFFFFFFFFFFFFFFFFFFFFFFFFFCE
:10CA7800FFFFFFFFFFFFFFFFFFFFFFFFFFFFFFFFBE
:10CA8800FFFFFFFFFFFFFFFFFFFFFFFFFFFFFFFFAE
:10CA9800FFFFFFFFFFFFFFFFFFFFFFFFFFFFFF3F5E
:10CAA800FFFFFFFFFFFFFFFFFFFFFFFFFFFFFFFF8E
:10CAB800FFFFFFFFFFFFFFFF030000FFFFFFFFFF78
:10CAC8007FFFFFFFFFFFFFFFFFFFFFFFFFFFFFFFEE
:10CAD800FFFFFFFFFFFFFFFFFFFFFFFFFFFFFFFF5E
:10CAE800FFFFFFFFFFFFFFFFFFFFFFFFFFFFFFFF4E
:10CAF800FFFFFFFFFFFFFFFFFFFFFFFFFFFFFF3FFE
:10CB0800FFFFFFFFFFFFFFFFFFFFFFFFFFFFFFFF2D
:10CB1800FFFFFFFFFFFFFF7FE0001CFFFFFFFFFF9E
:10CB28007FFFFFFFFFFFFFFFFFFFFFFFFFFFFFFF8D
:10CB3800FFFFFFFFFFFFFFFFFFFFFFFFFFFFFFFFFD
:10CB4800FFFFFFFFFFFFFFFFFFFFFFFFFFFFFFFFED
:10CB5800FFFFFFFFFFFFFFFFFFFFFFFFFFFFFF3F9D
:10CB6800FFFFFFFFFFFFFFFFFFFFFFFFFFFFFFFFCD
:10CB7800FFFFFFFFFFFFFF7FE0001CF8FFFFFFFF45
:10CB8800FFFFFFFFFFFFFFFFFFFFFFFFFFFFFFFFAD
:10CB9800FFFFFFFFFFFFFFFFFFFFFFFFFFFFFFFF9D
:10CBA800FFFFFFFFFFFFFFFFFFFFFFFFFFFFFFFF8D
:10CBB800FFFFFFFFFFFFFFFFFFFFFFFFFFFFFF3F3D
:10CBC800FFFFFFFFFFFFFFFFFFFFFFFFFFFFFFFF6D
:10CBD800FFFFFFFFFFFFFF7FE0001CF8FFFFFFFFE5
:10CBE800FFFFFFFFFFFFFFFFFFFFFFFFFFFBFFFF51
:10CBF800FFFFFFFFFFFFFFFFFFFFFFFFFFFFFFFF3D
:10CC0800FFFFFFFFFFFFFFFFFFFFFFFFFFFFFFFF2C
:10CC1800FFFFFFFFFFFFFFFFFFFFFFFFFFFFFF3FDC
:10CC2800FFFFFFFFFFFFFFFFFFFFFFFFFFFFFFFF0C
:10CC3800FFFFFFFFFFFFFF0F000000F8FFFFFFFFF0
:10CC4800FFFFFFFFFFFFFFFFFFFFFFFFFFFFFFFFEC
:10CC5800FFFFFFFFFFFFFFFFFFFFFFFFFFFFFFFFDC
:10CC6800FFFFFFFFFFFFFFFFFFFFFFFFFFFFFFFFCC
:10CC7800FFFFFFFFFFFFFFFFFFFFFFFFFFFFFF3F7C
:10CC8800FFFFFFFFFFFFFFFFFFFFFFFFFFFFFFFFAC
:10CC9800FFFFFFFFFFFFFF0F000000C0FFFFFFFFC8
:10CCA800FFFFFFFFFFFFFFFFFFFFFFFFFFFFFFFF8C
:10CCB800FFFFFFFFFFFFFFFFFFFFFFFFFFFFFFFF7C
:10CCC800FFFFFFFFFFFFFFFFFFFFFFFFFFFFFFFF6C
:10CCD800FFFFFFFFFFFFFFFFFFFFFFFFFFFFFF3F1C
:10CCE800FFFFFFFFFFFFFFFFFFFFFFFFFFFFFFFF4C
:10CCF800FFFFFFFFFFFFFF0F000000C0FFFFFFFF68
:10CD0800FFFFFFFFFFFFFFFFFFFFFFFFFFFFFFFF2B
:10CD1800FFFFFFFFFFFFFFFFFFFFFFFFFFFFFFFF1B
:10CD2800FFFFFFFFFFFFFFFFFFFFFFFFFFFFFFFF0B
:10CD3800FFFFFFFFFFFFFFFFFFFFFFFFFFFFFF3FBB
:10CD4800FFFFFFFFFFFFFFFFFFFFFFFFFFFFFFFFEB
:10CD5800FFFFFFFFFFFFFF0F000000C0FFFFFFFF07
:10CD6800FFFFFFFFFFFFFFFFFFFFFFFFFFFFFFFFCB
:10CD7800FFFFFFFFFFFFFFFFFFFFFFFFFFFFFFFFBB
:10CD8800FFFFFFFFFFFFFFFFFFFFFFFFFFFFFFFFAB
:10CD9800FFFFFFFFFFFFFFFFFFFFFFFFFFFFFF3F5B
:10CDA800FFFFFFFFFFFFFFFFFFFFFFFFFFFFFFFF8B
:10CDB800FFFFFFFFFFFFFF0F000000C0FFFFFFFFA7
:10CDC800FFFFFFFFFFFFFFFFFFFFFFFFFFFFFFFF6B
:10CDD800FFFFFFFFFFFFFFFFFFFFFFFFFFFFFFFF5B
:10CDE800FFFFFFFFFFFFFFFFFFFFFFFFFFFFFFFF4B
:10CDF800FFFFFFFFFFFFFFFFFFFFFFFFFFFFFF3FFB
:10CE0800FFFFFFFFFFFFFFFFFFFFFFFFFFFFFFFF2A
:10CE1800FFFFFFFFFFFFFF0F000000C0FFFFFFFF46
:10CE2800FFFFFFFFFFFFFFFFFFFFFFFFFFFFFFFF0A
:10CE3800FFFFFFFFFFFFFFFFFFFFFFFFFFFFFFFFFA
:10CE4800FFFFFFFFFFFFFFFFFFFFFFFFFFFFFFFFEA
:10CE5800FFFFFFFFFFFFFFFFFFFFFFFFFFFFFF3F9A
:10CE6800FFFFFFFFFFFFFFFFFFFFFFFFFFFFFFFFCA
:10CE7800FFFFFFFFFFFFFF0F000000C0FFFFFFFFE6
:10CE8800FF000000FEFFFF00000000FCFFFFFF00A6
:10CE980000F8FFFFFFFF010000FFFFFF0100000097
:10CEA80000F8FFFFFFFFFFFFFFFFFFFFFFFFFFFF90
:10CEB800FFFFFFFFFFFFFFFFFFFFFFFFFFFFFF3F3A
:10CEC800FFFFFFFFFFFFFFFFFFFFFFFFFFFFFFFF6A
:10CED800FFFFFFFFFFFFFF8FE3FF1FC7FFFFFFFFFE
:10CEE800FF000000F8FFFF00000000F0FFFF7F00D8
:10CEF80000F0FFFFFFFF000000FEFFFF0100000041
:10CF080000F8FFFFFFFFFFFFFFFFFFFFFFFFFFFF2F
:10CF1800FFFFFFFFFFFFFFFFFFFFFFFFFFFFFF3FD9
:10CF2800FFFFFFFFFFFFFFFFFFFFFFFFFFFFFFFF09
:10CF3800FFFFFFFFFFFFFF8FE3FF1FC7FFFFFFFF9D
:10CF48007F000000F0FFFF00000000E0FFFF7F000F
:10CF580000F0FFFFFF7F000000FCFFFF0100000062
:10CF680000F8FFFFFFFFFFFFFFFFFFFFFFFFFFFFCF
:10CF7800FFFFFFFFFFFFFFFFFFFFFFFFFFFFFF3F79
:10CF8800FFFFFFFFFFFFFFFFFFFFFFFFFFFFFFFFA9
:10CF9800FFFFFFFFFFFFFF8FE3FF1FC7FFFFFFFF3D
:10CFA8007F000000E0FFFF00000000C0FFFF7F00DF
:10CFB80000F0FFFFFF3F000000FCFFFF0000000043
:10CFC80000F8FFFFFFFFFFFFFFFFFFFFFFFFFFFF6F
:10CFD800FFFFFFFFFFFFFFFFFFFFFFFFFFFFFF3F19
:10CFE800FFFFFFFFFFFFFFFFFFFFFFFFFFFFFFFF49
:10CFF800FFFFFFFFFFFFFFFF1F78E0FFFFFFFFFFBF
:10D008007F000000C0FFFF0000000080FFFF7F00DE
:10D0180000E0FFFFFF1F000000F8FFFF0000000016
:10D0280000FCFFFFFFFFFFFFFFFFFFFFFFFFFFFF0A
:10D03800FFFFFFFFFFFFFFFFFFFFFFFFFFFFFF3FB8
:10D04800FFFFFFFFFFFFFFFFFFFFFFFFFFFFFFFFE8
:10D05800FFFFFFFFFFFFFFFF1F78E0FFFFFFFFFF5E
:10D068003F00000080FFFF0100000000FFFF7F007D
:10D0780000E0FFFFFF0F000000F0FFFF00000000CE
:10D0880000FCFFFFFFFFFFFFFFFFFFFFFFFFFFFFAA
:10D09800FFFFFFFFFFFFFFFFFFFFFFFFFFFFFF3F58
:10D0A800FFFFFFFFFFFFFFFFFFFFFFFFFFFFFFFF88
:10D0B800FFFFFFFFFFFFFFFF1F78E0FFFFFFFFFFFE
:10D0C8003F00000000FFFF0100000000FEFF3F00DE
:10D0D80000E0FFFFFF07000000F0FFFF0000000076
:10D0E80000FCFFFFFFFFBFFFFFFFFFFFFFFFFFFF8A
:10D0F800FFFFFFFFFFFFFFFFFFFFFFFFFFFFFF3FF8
:10D10800FFFFFFFFFFFFFFFFFFFFFFFFFFFFFFFF27
:10D11800FFFFFFFFFFFFFFFFFFFFFFFFFFFFFFFF17
:10D128001F00000000FEFF0100000000FEFF3F009E
:10D1380000E0FFFFFF03000000E0FFFF0000000029
:10D1480000FCFFFFFFFFFFFFFFCFFFFFFFFFFFFF19
:10D15800FFFFFFFFFFFFFFFFFFFFFFFFFFFFFF3F97
:10D16800FFFFFFFFFFFFFFFFFFFFFFFFFFFFFFFFC7
:10D17800FFFFFFFFFFFFFFFFFFFFFFFFFFFFFFFFB7
:10D188001F00000000FCFF0100000000FCFF3F0042
:10D1980000C0FFFFFF01000000E0FF7F000000006B
:10D1A80000FE7FFFFFFFFFFFFFFFFFFFFFFFFFFF07
:10D1B800FFFFFFFFFFFFFFFFFFFFFFFFFFFFFF3F37
:10D1C800FFFFFFFFFFFFFFFFFFFFFFFFFFFFFFFF67
:10D1D800FFFFFFFFFFFFFFFFFFFFFFFFFFFFFFFF57
:10D1E8000F00000000F8FF0300000000F0FF3F0000
:10D1F80000C0FFFFFF00000000C0FF7F000000002C
:10D2080000FEFFFFFFFFFFFFFFFFFFFFFFFFFFFF26
:10D21800FFFFFFFFFFFFFFFFFFFFFFFFFFFFFF3FD6
:10D22800FFFFFFFFFFFFFFFFFFFFFFFFFFFFFFFF06
:10D23800FFFFFFFFFFFFFFFFFFFFFFFFFFFFFFFFF6
:10D248000F00000000F0FF0300000000F0FF3F00A7
:10D2580000C0FFFF7F0000000080FF7F000000008B
:10D2680000FEFFFFFDFFFFFFFFFFFFFFFFFFFFFFC8
:10D27800FFFFFFFFFFFFFFFFFFFFFFFFFFFFFF3F76
:10D28800FFFFFFFFFFFFFFFFFFFFFFFFFFFFFFFFA6
:10D29800FFFFFFFFFFFFFFFFFFFFFFFFFFFFFFFF96
:10D2A8000700000000E0FF0300000000E0FF1D0091
:10D2B80000C0FFFF3F0000000080FF7F000000006B
:10D2C80000FEFFFFFFFFFFFFFFFFFFFFFFFFFFFF66
:10D2D800FFFFFFFFFFFFFFFFFFFFFFFFFFFFFF3F16
:10D2E800FFFFFFFFFFFFFFFFFFFFFFFFFFFFFFFF46
:10D2F800FFFFFFFFFFFFFFFFFFFFFFFFFFFFFFFF36
:10D308000700000000C0FF0300000000C0FF1F006E
:10D318000080FFFF1F0000000000FF3F000000002A
:10D3280000FEFFFFFFFFFFFFFFFFFFFFFFFFFFFF05
:10D33800FFFFFFFFFFFFFFFFFFFFFFFFFFFFFF3FB5
:10D34800FFFFFFFFFFFFFFFFFFFFFFFFFFFFFFFFE5
:10D35800FFFFFFFFFFFFFFFFFFFFFFFFFFFFFFFFD5
:10D368000300000000C0FF0700C01F0080FF1F006F
:10D378000080FFFF0F0000000000FF3F00000000DA
:10D3880000FFFFFFFFFFFFFFFFFFFFFFFFFFFFFFA4
:10D39800FFFFFFFFFFFFFFFFFFFFFFFFFFFFFF3F55
:10D3A800FFFFFFFFFFFFFFFFFFFFFFFFFFFFFFFF85
:10D3B800FFFFFFFFFFFFFFFFFFFFFFFFFFFFFFFF75
:10D3C8000700E07F0080FF0700E01F0080FF1F00CC
:10D3D8000080FFFF0F00E03F0000FF3F0080FFFFDD
:10D3E800FFFFFFFFFFFFFFFFFFFFFFFFFFFFFFFF45
:10D3F800FFFFFFFFFFFFFFFFFFFFFFFFFFFFFF3FF5
:10D40800FFFFFFFFFFFFFFFFFFFFFFFFFFFFFFFF24
:10D41800FFFFFFFFFFFFFFFFFFFFFFFFFFFFFFFF14
:10D428000700E07F0080FF0700E03F0000FF0F00DB
:10D438000000FFF70F00E03F0000FF3F0080FFFF04
:10D44800FFFFFFFFFFFFFFFFFFFFFFFFFFFFFFFFE4
:10D45800FFFFFFFFFFFFFFFFFFFFFFFFFFFFFF3F94
:10D46800FFFFFFFFFFFFFFFFFFFFFFFFFFFFFFFFC4
:10D47800FFFFFFFFFFFFFFFFFFFFFFFFFFFFFFFFB4
:10D488000700C07F0080FF0700E03F0000FF0F009B
:10D498000000FFFF0F00E03F0000FF3F0080FFFF9C
:10D4A800FFFFFFFFFFFFFFFFFFFFFFFFFFFFFFFF84
:10D4B800FFFFFFFFFFFFFFFFFFFFFFFFFFFFFF3F34
:10D4C800FFFFFFFFFFFFFFFFFFFFFFFFFFFFFFFF64
:10D4D800FFFFFFFFFFFFFFFFFFFFFFFFFFFFFFFF54
:10D4E8000F00C0FF0080FF0700E03F0000FF0F00B3
:10D4F8000000FFFF0F00E03F0000FF1F00C0FFFF1C
:10D50800FFFFFFFFFFFFFFFFFFFFFFFFFFFFFFFF23
:10D51800FFFFFFFFFFFFFFFFFFFFFFFFFFFFFF3FD3
:10D52800FFFFFFFFFFFFFFFFFFFFFFFFFFFFFFFF03
:10D53800FFFFFFFFFFFFFFFFFFFFFFFFFFFFFFFFF3
:10D548000F00C0FF0000FF0F00E03F0000FF0F00CA
:10D558000000FFFF0F00E03F0000FF1F00C0FFFFBB
:10D56800FFFFFFFFFFFFFFFFFFFFFFFFFFFFFFFFC3
:10D57800FFFFFFFFFFFFFFFFFFFFFFFFFFFFFF3F73
:10D58800FFFFFFFFFFFFFFFFFFFFFFFFFFFFFFFFA3
:10D59800FFFFFFFFFFFFFFFFFFFFFFFFFFFFFFFF93
:10D5A8000F0080FF0000FF0F00C03F0000FF0F00CA
:10D5B8000000FEFF0F00E03F0000FF1F00C0FFFF5C
:10D5C800FFFFFFFFFFFFFFFFFFFFFFFFFFFFFFFF63
:10D5D800FFFFFFFFFFFFFFFFFFFFFFFFFFFFFF3F13
:10D5E800FFFFFFFFFFFFFFFFFFFFFFFFFFFFFFFF43
:10D5F800FFFFFFFFFFFFFFFFFFFFFFFFFFFFFFFF33
:10D608001F0080FF0000FF0F00C03F0000FF070061
:10D618000000FEFF0F00E03F0080FF1F00C0FFFF7B
:10D62800FFFFFFFFFFFFFFFFFFFFFFFFFFFFFFFF02
:10D63800FFFFFFFFFFFFFFFFFFFFFFFFFFFFFF3FB2
:10D64800FFFFFFFFFFFFFFFFFFFFFFFFFFFFFFFFE2
:10D65800FFFFFFFFFFFFFFFFFFFFFFFFFFFFFFFFD2
:10D668001F0080FF0100FE0F00C03F0000FF070001
:10D678000000FEFF0700E03F0080FF1F00E0FFFF03
:10D68800FFFFFFFFFFFFFFFFFFFFFFFFFFFFFFFFA2
:10D69800FFFFFFFFFFFFFFFFFFFFFFFFFFFFFF3F52
:10D6A800FFFFFFFFFFFFFFFFFFFFFFFFFFFFFFFF82
:10D6B800FFFFFFFFFFFFFFFFFFFFFFFFFFFFFFFF72
:10D6C8003F0000FF0100FE1F00C07F0000FF0700B1
:10D6D8000000FEFF0700E01F0080FF0F00E0FFFFD3
:10D6E800FFFFFFFFFFFFFFFFFFFFFFFFFFFFFFFF42
:10D6F800FFFFFFFFFFFFFFFFFFFFFFFFFFFFFF3FF2
:10D70800FFFFFFFFFFFFFFFFFFFFFFFFFFFFFFFF21
:10D71800FFFFFFFFFFFFFFFFFFFFFFFFFFFFFFFF11
:10D728003F0000FF0100FE1F00C07F0000FF070050
:10D738000000FCFF0700E01F0080FF0F00E0FFFF74
:10D74800FFFFFFFFFFFFFFFFFFFFFFFFFFFFFFFFE1
:10D75800FFFFFFFFFFFFFFFFFFFFFFFFFFFFFF3F91
:10D76800FFFFFFFFFFFFFFFFFFFFFFFFFFFFFFFFC1
:10D77800FFFFFFFFFFFFFFFFFFFFFFFFFFFFFFFFB1
:10D788003F0000FFFFFFFF1F00C07F0000FF0700F2
:10D798000000FCFF0700E01F0080FF0F00E0FFFF14
:10D7A800FFFFFFFFFFFFFFFFFFFFFFFFFFFFFFFF81
:10D7B800FFFFFFFFFFFFFFFFFFFFFFFFFFFFFF3F31
:10D7C800FFFFFFFFFFFFFFFFFFFFFFFFFFFFFFFF61
:10D7D800FFFFFFFFFFFFFFFFFFFFFFFFFFFFFFFF51
:10D7E8007F0000FEFFFFFF1F00807F0000FF030097
:10D7F8000000FCFF0700F01F0080FF0F00F0FFFF94
:10D80800FFFFFFFFFFFFFFFFFFFFFFFFFFFFFFFF20
:10D81800FFFFFFFFFFFFFFFFFFFFFFFFFFFFFF3FD0
:10D82800FFFFFFFFFFFFFFFFFFFFFFFFFFFFFFFF00
:10D83800FFFFFFFFFFFFFFFFFFFFFFFFFFFFFFFFF0
:10D848007F0000FEFFFFFF1F00807F0000FF030036
:10D858000000FCFF0700F01F0080FF0F00F0FFFF33
:10D86800FFFFFFFFFFFFFFFFFFFFFFFFFFFFFFFFC0
:10D87800FFFFFFFFFFFFFFFFFFFFFFFFFFFFFF3F70
:10D88800FFFFFFFFFFFFFFFFFFFFFFFFFFFFFFFFA0
:10D89800FFFFFFFFFFFFFFFFFFFFFFFFFFFFFFFF90
:10D8A800FF0000FEFFFFFF3F00807F0000FF030036
:10D8B8000400F8FF0700F01F0080FF0700F0FFFFDB
:10D8C800FFFFFFFFFFFFFFFFFFFFFFFFFFFFFFFF60
:10D8D800FFFFFFFFFFFFFFFFFFFFFFFFFFFFFF3F10
:10D8E800FFFFFFFFFFFFFFFFFFFFFFFFFFFFFFFF40
:10D8F800FFFFFFFFFFFFFFFFFFFFFFFFFFFFFFFF30
:10D90800FF0000FCFFFFFF3F00807F0000FE0300D8
:10D918000600F8FF0700F0FFFFFFFF0700F0FFFD1C
:10D92800FFFFFFFFFFFFFFFFFFFFFFFFFFFFFFFFFF
:10D93800FFFFFFFFFFFFFFFFFFFFFFFFFFFFFF3FAF
:10D94800FFFFFFFFFFFFFFFFFFFFFFFFFFFFFFFFDF
:10D95800FFFFFFFFFFFFFFFFFFFFFFFFFFFFFFFFCF
:10D96800FF00000000F0FF3F00807F0000FE010084
:10D978000600F8FF0700F0FFFFFFFF07000000FCAC
:10D98800FFFFFFFFFFFFFFFFFFFFFFFFFFFFFFFF9F
:10D99800FFFFFFFFFFFFFFFFFFFFFFFFFFFFFF3F4F
:10D9A800FFFFFFFFFFFFFFFFFFFFFFFFFFFFFFFF7F
:10D9B800FFFFFFFFFFFFFFFFFFFFFFFFFFFFFFFF6F
:10D9C800FF01000000E0FF3F00007F0000FE0100B3
:10D9D8000600F8FF0700F0FFFFFFFF07000000FC4C
:10D9E800FFFFFFFFFFFFFFFFFFFFFFFFFFFFFFFF3F
:10D9F800FFFFFFFFFFFFFFFFFFFFFFFFFFFFFF3FEF
:10DA0800FFFFFFFFFFFFFFFFFFFFFFFFFFFFFFFF1E
:10DA1800FFFFFFFFFFFFFFFFFFFFFFFFFFFFFFFF0E
:10DA2800FF01000000C0FF7F0000FF0000FE0100B2
:10DA38000E00F0E30700F0FFFFFFFF03000000FC0B
:10DA4800FFFFFFFFFFFFFFFFFFFFFFFFFFFFFFFFDE
:10DA5800FFFFFFFFFFFFFFFFFFFFFFFFFFFFFF3F8E
:10DA6800FFFFFFFFFFFFFFFFFFFFFFFFFFFFFFFFBE
:10DA7800FFFFFFFFFFFFFFFFFFFFFFFFFFFFFFFFAE
:10DA8800FF0300000080FF7F0000FF0000FE010090
:10DA98000E00F0F30700F0FFFFFFFF03000000FE99
:10DAA800FFDFFFFFFFFFFFFFFFFFFFFFFFFFFFFF9E
:10DAB800FFFFFFFFFFFFFFFFFFFFFFFFFFFFFF3F2E
:10DAC800FFFFFFFFFFFFFFFFFFFFFFFFFFFFFFFF5E
:10DAD800FFFFFFFFFFFFFFFFFFFFFFFFFFFFFFFF4E
:10DAE800FF0F00000000FF7F0000FF0000FE0100A4
:10DAF8000F00F0FF0700F0FFFFFFFF03000000FE2C
:10DB0800FFFFBFFFFFFFFFFFFFFFFFFFFFFFFFFF5D
:10DB1800FFFFFFFFFFFFFFFFFFFFFFFFFFFFFF3FCD
:10DB2800FFFFFFFFFFFFFFFFFFFFFFFFFFFFFFFFFD
:10DB3800FFFFFFFFFFFFFFFFFFFFFFFFFFFFFFFFED
:10DB4800FF1F00000000FE7F0000FF0000FE010034
:10DB58000F00F0FF0700F0FFFFFFFF03000000FECB
:10DB6800FFFFFFFFFFFFFFFFFFFFFFFFFFFFFFFFBD
:10DB7800FFFFFFFFFFFFFFFFFFFFFFFFFFFFFF3F6D
:10DB8800FFFFFFFFFFFFFFFFFFFFFFFFFFFFFFFF9D
:10DB9800FFFFFFFFFFFFFFFFFFFFFFFFFFFFFFFF8D
:10DBA800FF3F00000000FC7F0000FF0000FE0000B7
:10DBB8001F00E0FF0700F0FFFFFFFF03000000FE6B
:10DBC800FFFFFFFFFFFFFFFFFFFFFFFFFFFFFFFF5D
:10DBD800FFFFFFFFFFFFFFFFFFFFFFFFFFFFFF3F0D
:10DBE800FFFFFFFFFFFFFFFFFFFFFFFFFFFFFFFF3D
:10DBF800FFFFFFFFFFFFFFFFFFFFEFFFFFFF7FFFBD
:10DC0800FF7F00000000F87F0000FE0000FE00001B
:10DC18001F00E0FF0700F0FFFFFFFF01000000FE0C
:10DC2800FFFFFFFFFFFFFFFFFFFFFFFFFFFFFFFFFC
:10DC3800FFFFFFFFFFFFFFFFFFFFFFFFFFFFFF3FAC
:10DC4800FFFFFFFFFFFFFFFFFFFFFFFFFFFFFFFFDC
:10DC5800FFFFFFFFFFFFFFFF1FFFFFFFFFFFFFFFAC
:10DC6800FFFF00000000F0FF0000FE0000FE0000C3
:10DC78001F00E0FF0300F0FFFFFFFF01000000FFAF
:10DC8800FFFFFFFFFFFFFEFFFFFFFFFFFFFFFFFF9D
:10DC9800FFFFFFFFFFFFFFFFFFFFFFFFFFFFFF3F4C
:10DCA800FFFFFFFFFFFFFFFFFFFFFFFFFFFFFFFF7C
:10DCB800FFFFFFFFFFFFFFFF1FFFFFFFFFFFFFFF4C
:10DCC800FFFF03000000E0FF0000C00000FE0000AE
:10DCD8001F00E0FF0300F0FFFFFFFF01000000FF4F
:10DCE800FFFFFFFFFFFFFFFFFFFFFFFFFFFFFFFF3C
:10DCF800FFFFFFFFFFFFFFFFFFFFFFFFFFFFFF3FEC
:10DD0800FFFFFFFFFFFFFFFFFFFFFFFFFFFFFFFF1B
:10DD1800FFFFFFFFFFDFFFFF1FFFFFFFFFFFFFFF0B
:10DD28007FFE07000000E0FF00000000007F008089
:10DD38003F00C0FF0300F0FFFFFFFF01000000FFEE
:10DD4800FFFFFFFFFFFFFFFFFFFFFFFFFFFFFFFFDB
:10DD5800FFFFFFFFFFFFFFFFFFFFFFFFFFFFFF3F8B
:10DD6800FFFFFFFFFFFFFFFFFFFFFFFFFFFFFFFFBB
:10DD7800FFFFFFFFFFDFFFFFFFF8FFFFFFFFFFFFD2
:10DD8800FFFF0F000000C0FF00000000007F0080C0
:10DD98003F00C0FF0300F0FFFFFFFF01000000FF8E
:10DDA800FFFFFFFFFFFFFFFFFFFFFFFFFFFFFFFF7B
:10DDB800FFFFFFFFFFFFFFFFFFFFFFFFFFFFFF3F2B
:10DDC800FFFFFFFFFFFFFFFFFFFFFFFFFFFFFFFF5B
:10DDD800FFFFFFFFFFFFFFFFFFF8FFFFFFFFFFFF52
:10DDE800FFFF1F000000C0FF01000000807F0080CF
:10DDF8003F00C0FF0300F8FFFFFFFF00000080FFA7
:10DE0800FFFFFFFFFFFFFFFFFFFFFFFFFFFFFFFF1A
:10DE1800FFFFFFFFFFFFFFFFFFFFFFFFFFFFFF3FCA
:10DE2800FFFFFFFFFFFFFFFFFFFFFFFFFFFFFFFFFA
:10DE3800FFFFFFFFFFFFFFFFFFF8FFFFFFFFFFFFF1
:10DE4800FFFFFFFF7F00C0FF01000000C07F000050
:10DE58000000C0FF0300F80F00F0FF0000FEFFFF06
:10DE6800FFFFFFFFFFFFFFFFFFFFFFFFFFFFFFFFBA
:10DE7800FFFFFFFFFFFFFFFFFFFFFFFFFFFFFF3F6A
:10DE8800FFFFFFFFFFFFFFFFFFFFFFFFFFFFFFFF9A
:10DE9800FFFFFFFFFFFFFFFF1FFFFFFFFFFFFFFF6A
:10DEA800FFFFFFFF7F0080FF01000000C07F000030
:10DEB800000080FF0300F80F00F0FF0000FFFFFFE5
:10DEC800FFFFFFFFFFFFFFFFFFFFFFFFFFFFFFFF5A
:10DED800FFFFFFFFFFFFFFFFFFFFFFFFFFFFFF3F0A
:10DEE800FFFFFFFFFFFFFFFFFFFFFFFFFFFFFFFF3A
:10DEF800FFFFFFFFFFFFFFFF1FFFFFF3FFFFFFFF16
:10DF0800FFFFFFFF7F0080FF01000000E03F0000EF
:10DF1800000080FF0300F80F00F0FF0000FFFFFF84
:10DF2800FFFFFFFFFFFFFFFFFFFFFFFFFFFFFFFFF9
:10DF3800FFFFFFFFFFFFFFFFFFFFFFFFFFFFFF3FA9
:10DF4800FFFFFFFFFFFFFFFFFFFFFFFFFFFFFFFFD9
:10DF5800FFFFFFFFFFFFFFFF1FFFFFFFFFFFFFFFA9
:10DF6800FFFFFFFF7F0080FF03000000F03F00007D
:10DF7800000080FF0300F80700F07F0000FFFFFFAC
:10DF8800FFFFFFFFFFFFFFFFFFFFFFFFFFFFFFFF99
:10DF9800FFFFFFFFFFFFFFFFFFFFFFFFFFFFFF3F49
:10DFA800FFFFFFFFFFFFFFFFFFFFFFFFFFFFFFFF79
:10DFB800FFFFFFFFFFFFFFFFFFF8FFFFFFFFFFFF70
:10DFC800FF7F0080FF0080FF03000000F83F000093
:10DFD800000000FF0300F80700F07F0000FFFFFFCC
:10DFE800FFFFFFFFFFFFFFFFFFFFFFFFFFFFFFFF39
:10DFF800FFFFFFFFFFFFFFFFFFFFFFFFFFFFFF3FE9
:10E00800FFFFFFFFFFFFFFFFFFFFFFFFFFFFFFFF18
:10E01800FFFFFFFFFFFFFFFFFFF8FFFFFFFFFFFF0F
:10E02800FF7F0000FF0000FF03000000F83F000032
:10E03800000000FF0300F80700F07F0000FFFFFF6B
:10E04800FFFFFF7FFFFFFFFFFFFFFFFFFFFFFFFF58
:10E05800FFFFFFFFFFFFFFFFFFFFFFFFFFFFFF3F88
:10E06800FFFFFFFFFFFFFFFFFFFFFFFFFFFFFFFFB8
:10E07800FFFFFFFFFFFFFFFFFFF8FFFFFFFFFFFFAF
:10E08800FFFF0000FF0000FF0300F8FFFF3F000054
:10E09800000000FF0300F80700F07F0080FFFFFF8B
:10E0A800FFFFFFFFFFFFFFFFFFFFFFFFFFFFFFFF78
:10E0B800FFFFFFFFFFFFFFFFFFFFFFFFFFFFFF3F28
:10E0C800FFFFFFFFFFFFFFFFFFFFFFFFFFFFFFFF58
:10E0D800FFFFFFFFFFFFFFFF1FFFFFFFFFFFFFFF28
:10E0E800FFFF0000FF0000FF0300F8FFFF1F000014
:10E0F800000000FF0300F80700F03F0080FFFFFF6B
:10E10800FFFFFFFFFFFFFFFFFFFFFFFFFFFFFFFF17
:10E11800FFFFFFFFFFFFFFFFFFFFFFFFFFFFFF3FC7
:10E12800FFFFFFFFFFFFFFFFFFFFFFFFFFFFFFFFF7
:10E13800FFFFFFFFFFFFFFFF1FFFFFFFFFFFFFFFC7
:10E14800EFFF0100FF0100FE0700F8FFFF1F0000BE
:10E15800000000FE0300F80700F03F0080FFFFFF0B
:10E16800FFFFFFFFFFFFFFFFFFFFFFFFFFFFFFFFB7
:10E17800FFFFFFFFFFFFFFFFFFFFFFFFFFFFFF3F67
:10E18800FFFFFFFFFFFFFFFFFFFFFFFFFFFFFFFF97
:10E19800FFFFFFFFFFFFFFFF1FFFFFFFFFFFFFFF67
:10E1A800FFFF0100FE0100FE0700F8FFFD1F000051
:10E1B800000000FE0300F80700F83F0080FFFFEFB3
:10E1C800FFFFFFFFFFFFFFFFFFFFFFFFFFFFFFFF57
:10E1D800FFFFFFFFFFFFFFFFFFFFFFFFFFFFFF3F07
:10E1E800FFFFFFFFFFFFFFFFFFFFFFFFFFFFFFFF37
:10E1F800FFFFFFFFFFFFFFFFFFF8FFFFFFFFFFFF2E
:10E20800FFFF0100FE0100FE0700F8FFFD1F00F000
:10E21800FF0100FE0300F80700F83F00C0FFFFFF02
:10E22800FFFFFFFFFFFFFFFFFFFFFFFFFFFFFFFFF6
:10E23800FFFFFFFFFFFFFFFFFFFFFFFFFFFFFF3FA6
:10E24800FFFFFFFFFFFFFFFFFFFFFFFFFFFFFFFFD6
:10E25800FFFFFFFFFFFFFFFFFFF8FFFFFFFFFFFFCD
:10E26800FFFF0300FC0100FE0700F8FFFF0F00F0AE
:10E27800FF0100FE0300F80700F83F00C0FFFFFFA2
:10E28800FFFFFFFFFFFFFFFFFFFFFFFFFFFFFFFF96
:10E29800FFFFFFFFFFFFFFFFFFFFFFFFFFFFFF3F46
:10E2A800FFFFFFFFFFFFFFFFFFFFFFFFFFFFFFFF76
:10E2B800FFFFFFFFFFFFFFFFFFF8FFFFFFFFFFFF6D
:10E2C800FFFF0300FC0300FC0F00F8FFFF0F00F046
:10E2D800FF0300FC0300FC0700F81F00C0FFFFFF5E
:10E2E800FFFFFFFFFFFFFFFFFFFFFFFFFFFFFFFF36
:10E2F800FFFFFFFFFFFFFFFFFFFFFFFFFFFFFF3FE6
:10E30800FFFFFFFFFFFFFFFFFFFFFFFFFFFFFFFF15
:10E31800FFFFFFFFFFFFFFFFFFFFFFFFFFFFFFFF05
:10E32800FFFF0300FC0300FC0F00F0FFFF0F00F0ED
:10E33800FF0300FC0300FC0700F81F00C0FFFFFFFD
:10E34800FFFFFFFFFFFFFFFFFFFFFFFFFFFFFFFFD5
:10E35800FFFFFFFFFFFFFFFFFFFFFFFFFFFFFF3F85
:10E36800FFFFFFFFFFFFFFFFFFFFFFFFFFFFFFFFB5
:10E37800FFFFFFFFFFFFFFFFFFFFFFFFFFFFBFFFE5
:10E38800FFFF0700000000FE0F00F0FFFF0F00F086
:10E39800FF0300FC0300000000FC1F00000000FE5B
:10E3A8003FFFFFFFFFFFFFFFFFFFFFFFFFFFFFFF35
:10E3B800FFFFFFFFFFFFFFFFFFFFFFFFFFFFFF3F25
:10E3C800FFFFFFFFFFFFFFFFFFFFFFFFFFFFFFFF55
:10E3D800FFFFFFFFFFFFFFFFFFFFFFFFFFFFBFFF85
:10E3E800FFFF0700000000FF0F00F0FFFF0F00F81D
:10E3F800FF0300FC0700000000FE1F00000000FEF5
:10E408003FFFFFFFFFFFFFFFFFFFFFFFFFFFFFFFD4
:10E41800FFFFFFFFFFFFFFFFFFFFFFFFFFFFFF3FC4
:10E42800FFFFFFFFFFFFFFFFFFFFFFFFFFFFFFFFF4
:10E43800FFFFFFFFFFFFFFFFFFFFFFFFFFFFFFFFE4
:10E44800FFFF1F00000000FF0F00F0FFFC0F00F8A7
:10E45800FF0700F80700000000FF1F00000000FE93
:10E46800FFFFFFFFFFFFFFFFFFFFFFFFFFFFFFFFB4
:10E47800FFFFFFFFFFFFFFFFFFFFFFFFFFFFFF3F64
:10E48800FFFFFFFFFFFFFFFFFFFFFFFFFFFFFFFF94
:10E49800FFFFFFFFFFFFFFFFFFFFFFFFFFFFFFFF84
:10E4A800FFFF3F00000080FF1F00F0FFFF0500F89E
:10E4B800FF0700F80F00000080FF0F00000000FEBB
:10E4C800FFFFFFFFFFFFFFFFFFFFFFFFFFFFFFFF54
:10E4D800FFFFFFFFFFFFFFFFFFFFFFFFFFFFFF3F04
:10E4E800FFFFFFFFFFFFFFFFFFFFFFFFFFFFFFFF34
:10E4F800FFFFFFFFFFFFFFFFFFFFFFFFFFFFFFFF24
:10E50800FFFF7F000000C0FF1F00F0FFFF0700F8BB
:10E51800FF0700F81F000000C0FF0F00000000FF09
:10E52800FFFFFFFFFFFFFFFFFFFFFDFFFFFFFFFFF5
:10E53800FFFFFFFFFFFFFFFFFFFFFFFFFFFFFF3FA3
:10E54800FFFFFFFFFFFFFFFFFFFFFFFFFFFFFFFFD3
:10E55800FFFFFFFFFFFFFFFFFFFFFFFFFFFFFFFFC3
:10E56800FFFFFF010000C0FF1F00E0FFFF0700FCE6
:10E57800FF0700F83F000000E0FF0F00000000FF69
:10E58800FFFFFFFFFFFFFFFFFFFFFFFFFFFFFFFF93
:10E59800FFFFFFFFFFFFFFFFFFFFFFFFFFFFFF3F43
:10E5A800FFFFFFFFFFFFFFFFFFFFFFFFFFFFFFFF73
:10E5B800FFFFFFFFFFFFFFFFFFFFFFFFFFFFFFFF63
:10E5C800FFFFFF070000E0FF1F00E0FFFF0700FC60
:10E5D800FF0F00F83F000000F0FF0F00000000FFF1
:10E5E800FFFFFFFFFFFFFFFFFFFFFFFFFFFFFFFF33
:10E5F800FFFFFFFFFFFFFFFFFFFFFFFFFFFFFF3FE3
:10E60800FFFFFFFFFFFFFFFFFFFFFFFFFFFFFFFF12
:10E61800FFFFFFFFFFFFFFFFFFFFFFFFFFFFFFFF02
:10E62800FFFFFF070000F0FF3F00E0FFFF0300FCD3
:10E63800FF0F00F07F000000F8FF0700000000FF58
:10E64800FFFFFFFFFFFFFFFFFFFFFFFFFFFFFFFFD2
:10E65800FFFFFFFFFFFFFFFFFFFFFFFFFFFFFF3F82
:10E66800FFFFFFFFFFFFFFFFFFFFFFFFFFFFFFFFB2
:10E67800FFFFFFFFFFFFFFFFFFFFFFFFBFFFFFFFE2
:10E68800FFFFFF1F0000D0FF2700E0FFFF0300FC93
:10E69800FF0F00F0FF000000FEFF0700000000FF72
:10E6A800FFFFFFFFFFFFFFFFFFFFFFFFFFFFFFFF72
:10E6B800FFFFFFFFFFFFFFFFFFFFFFFFFFFFFF3F22
:10E6C800FFFFFFFFFFFFFFFFFFFFFFFFFFFFFFFF52
:10E6D800FFFFFFFFFFFFFFFFFFFFFFFFFFFFFFFF42
:10E6E800FFFFFF3F0000D8FF2700E0FFFF0300FC0B
:10E6F800FF0F00F0FF010000FFFD0700000080FF92
:10E70800FFFFFFFFFFFFFFFFFFFFFFFFFFFFFFFF11
:10E71800FFFFFFFFFFFFFFFFFFFFFFFFFFFFFF3FC1
:10E72800FFFFFFFFFFFFFFFFFFFFFFFFFFFFFFFFF1
:10E73800FFFFFFFFFFFFFFFFFFFFFFFFFFFFFFFFE1
:10E74800FFFFFF7F0000FCFF3F00E0FFFF0300FC2E
:10E75800FE1F00F0FF010080FFFD0700000080FFA2
:10E76800FFFFFFFFFFFFFFFFFFFFFFFFFFFFFFFFB1
:10E77800FFFFFFFFFFFFFFFFFFFFFFFFFFFFFF3F61
:10E78800FFFFFFFFFFFFFFFFFFFFFFFFFFFFFFFF91
:10E79800FFFFFFFFFFFFFFFFFFFFFFFFFFFFFFFF81
:10E7A800FFFFFFFFFFFFFFFFFFFFFFFFFFFFFFFF71
:10E7B800FEFFFFFFFFFFFFFFFFFFFFFFFFFFFFFF62
:10E7C800FFFFFFFFFFFFFFFFFFFFFFFFFFFFFFFF51
:10E7D800FFFFFFFFFFFFFFFFFFFFFFFFFFFFFF3F01
:10E7E800FFFFFFFFFFFFFFFFFFFFFFFFFFFFFFFF31
:10E7F800FFFFFFFFFFFFFFFFFFFFFFFFFFFFE7FF39
:10E80800FFFFFFFFFFFFFFFFFFFFFFFFFFFFFFFF10
:10E81800FFFFFFFFFFFFFFFFFFFFFFFFFFFFFFFF00
:10E82800FFFFFFFFFFFFFFFFFFFFFFFFFFFFFFFFF0
:10E83800FFFFFFFFFFFFFFFFFFFFFFFFFFFFFF3FA0
:10E84800FFFFFFFFFFFFFFFFFFFFFFFFFFFFFFFFD0
:10E85800FFFFFFFFFFFFFFFFFFFFFFFFFFFFE7FFD8
:10E86800FFFFFFFFFFFFFFFFFFFFFFFFFFFFFFFFB0
:10E87800FFFDFFFFFFFFFFFFFFFFFFFFFFFFFFFFA2
:10E88800FFFFFFFFFFFFFFFFFFFFFFFFFFFFFFFF90
:10E89800FFFFFFFFFFFFFFFFFFFFFFFFFFFFFF3F40
:10E8A800FFFFFFFFFFFFFFFFFFFFFFFFFFFFFFFF70
:10E8B800FFFFFFFFFFFFFFFFBFFFFFFFFFFFFFFFA0
:10E8C800EFFFFFFFFFFFFFFFFFFFFFFFFFFEFFFF61
:10E8D800FFFDFFFFF7FFFFFFFFFFFFFFFFFFFFFF4A
:10E8E800FFFFFF9FFFFFFFFFFFFFFFFFFFFFFFFF90
:10E8F800FFFFFFFFFFFFFFFFFFFFFFFFFFFFFF3FE0
:10E90800FFFFFFFFFFFFFFFFFFFFFFFFFFFFFFFF0F
:10E91800FFFFFFFFFFFFFFFFFFFFFFFFFFFFFFFFFF
:10E92800EFFFFFEFFFFFFFCFFFFFFFFFFCFEFFFF43
:10E93800FFFFF3FFFFFFFFFFFFFFFFFFFFFFFFFFEB
:10E948007FFFFF9FFFFFFFFFFFFFFFFFFFFFFFFFAF
:10E95800FFFFFFFFFFFFFFFFFFFFFFFFFFFFFF3F7F
:10E96800FFFFFFFFFFFFFFFFFFFFFFFFFFFFFFFFAF
:10E97800FFFFFFFFFFFFFFFFFFFFFFFFFFFFFFFF9F
:10E98800FFFFFFFFFFFFFFCFFFFFFFFFFCFFFFFDC4
:10E99800FFFFFFFFFFFFFFFFFFFFFFFFFFFFFFFF7F
:10E9A800FFFFFFFFFFFFFFFFFFFFFFFFFFFFFFFF6F
:10E9B800FFFFFFFFFFFFFFFFFFFFFFFFFFFFFF3F1F
:10E9C800FFFFFFFFFFFFFFFFFFFFFFFFFFFFFFFF4F
:10E9D800FFFFFFFFFFFFFFFFFFFFFFFFFFFFFFFF3F
:10E9E800FFFFFFFFFFFFFFFFFFFFFFFFFFFFFFFD31
:10E9F800FFFFFFFFFFFFFDFFFFFFE7FFFFFFFFFF39
:10EA0800FFFFFFFFFFFFFFFFFFFFFFFFFFFFFFFF0E
:10EA1800FFFFFFFFFFFFFFFFFFFFFFFFFFFFFF3FBE
:10EA2800FFFFFFFFFFFFFFFFFFFFFFFFFFFFFFFFEE
:10EA3800FFFFFFFFFFFFFFFFFFFFFFFFFFFFFFFFDE
:10EA4800FFFFFFFFFFFFFFFFFFFFFFFFFFFFFFFFCE
:10EA5800FFFFFFFFFFFFFDEFFFFFE7FFFFFFFFFFE8
:10EA6800FFFFFFFFFFFFFFFFFFFFFFFFFFFFFFFFAE
:10EA7800FFFFFFFFFFFFFFFFFFFFFFFFFFFFFF3F5E
:10EA8800FFFFFFFFFFFFFFFFFFFFFFFFFFFFFFFF8E
:10EA9800FFFFFFFFFFFFFFFFFFFFFFFFFFFFFFFF7E
:10EAA800FFFFFFFFFFFFFFFFFFFFFFFFFFFFFFFF6E
:10EAB800FFFFFFFFFFFFFFEFFFFFFFFFFFFFFFFF6E
:10EAC800FFFFFFFFFFBFFFFFFFFFFFFFFFFFFFFF8E
:10EAD800FFFFFFFFFFFFFFFFFFFFFFFFFFFFFF3FFE
:10EAE800FFFFFFFFFFFFFFFFFFFFFFFFFFFFFFFF2E
:10EAF800FFFFFFFFFFFFFFFFFFFFFFFFFFFFFFFF1E
:10EB0800FFFFFFFFFFFFFFFFFFE7FFFFFFFFFFFF25
:10EB1800FEFFFFFFFFFFFFFFFFFFFFFFFFFFFFFFFE
:10EB2800FFFFFFFFFFFFFFFFFFFFFFFFFFFFFFFFED
:10EB3800FFFFFFFFFFFFFFFFFFFFFFFFFFFFFF3F9D
:10EB4800FFFFFFFFFFFFFFFFFFFFFFFFFFFFFFFFCD
:10EB5800FFFFFFFFFFFFFFFFFFFFFFFFFFFFFFFFBD
:10EB6800FFFFFFFFFFFFFFFFFFFFFFFFFFFFFFFFAD
:10EB7800FEFFFFFFFFFFFFFFFFFFFFFFFFFFFFFF9E
:10EB8800FFFFFFFFFFFFFFFFFFFFFFFFFFFFFFFF8D
:10EB9800FFFFFFFFFFFFFFFFFFFFFFFFFFFFFF3F3D
:10EBA800FFFFFFFFFFFFFFFFFFFFFFFFFFFFFFFF6D
:10EBB800FFFFFFFFFFFFFFFFFFFFFFFF0F00F07FDB
:10EBC80000E0FF0F000E00F0FF3F00F87F0000FF9D
:10EBD800FF0F000000FEFF01000000F01F00008092
:10EBE800FFFFFF070080FFFFFFFFFFFFFFFFFFFFA3
:10EBF800FFFFFFFFFFFFFFFFFFFFFFFFFFFFFF3FDD
:10EC0800FFFFFFFFFFFFFFFFFFFFFFFFFFFFFFFF0C
:10EC1800FFFFFFFFFFFFFFFFFFFFFFFF1F00E07F7A
:10EC280000C0FF0F001E00E07F1F00F03F0000FF44
:10EC3800FF07000000F8FF00000000F00F000000D0
:10EC4800FEFFFF010080FFFFFFFFFFFFFFFFFFFF49
:10EC5800FFFFFFFFFFFFFFFFFFFFFFFFFFFFFF3F7C
:10EC6800FFFFFFFFFFFFFFFFFFFFFFFFFFFFFFFFAC
:10EC7800FFFFFFFFFFFFFFFFFFFFFFFF1F00E07F1A
:10EC88000080FF0F001E00E07F1F00F83F0000FE1D
:10EC9800FF07000000F8FF00000000F00F00000070
:10ECA800FEFF7F000000FFFFFFFFFFFFFFFFFFFFEA
:10ECB800FFFFFFFFFFFFFFFFFFFFFFFFFFFFFF3F1C
:10ECC800FFFFFFFFFFFFFFFFFFFFFFFFFFFFFFFF4C
:10ECD800FFFFFFFFFFFFFFFFFFFFFFFF3F00C0FF3A
:10ECE8000000FF0F003C00C0FF1F00F83F0000FEBF
:10ECF800FF07000000F0FF00000000F80700000018
:10ED0800FCFF3F000000FFFFFFFFFFFFFFFFFFFFCB
:10ED1800FFFFFFFFFFFFFFFFFFFFFFFFFFFFFF3FBB
:10ED2800FFFFFFFFFFFFFFFFFFFFFFFFFFFFFFFFEB
:10ED3800FFFFFFFFFFFFFFFFFFFFFFFF3F00C0FFD9
:10ED48000000FE1F003C0080FF1F00F83F0000FC91
:10ED5800FF07000000E0FF00000000F807000000C7
:10ED6800F8FF0F000000FFFFFFFFFFFFFFFFFFFF9F
:10ED7800FFFFFFFFFFFFFFFFFFFFFFFFFFFFFF3F5B
:10ED8800FFFFFFFFFFFFFFFFFFFFFFFFFFFFFFFF8B
:10ED9800FFFFFFFFFFFFFFFFFFFFFFFF7F0080F385
:10EDA8000100FC1F007C0080FF1F00F81F0000FC12
:10EDB800FF07000000E0FF00000000F80700000067
:10EDC800F0FF03000000FEFFFFFFFFFFFFFFFFFF54
:10EDD800FFFFFFFFFFFFFFFFFFFFFFFFFFFFFF3FFB
:10EDE800FFFFFFFFFFFFFFFFFFFFFFFFFFFFFFFF2B
:10EDF800FFFFFFFFFFFFFFFFFFFFFFFF7F0080F325
:10EE08000100F81F00FC0000FF0F00F81F0000FCC5
:10EE1800FF07000000C0FF00000000F8030000002A
:10EE2800E0FF01000000FEFFFFFFFFFFFFFFFFFF05
:10EE3800FFFFFFFFFFFFFFFFFFFFFFFFFFFFFF3F9A
:10EE4800FFFFFFFFFFFFFFFFFFFFFFFFFFFFFFFFCA
:10EE5800FFFFFFFFFFFFFFFFFFFFFFFFFF0000FFB8
:10EE68000300F03F00F80000FE0F00FC1F0000F850
:10EE7800FF0700000080FF00000000FC0300000006
:10EE8800E07F00000000FEFFFFFFFFFFFFFFFFFF26
:10EE9800FFFFFFFFFFFFFFFFFFFFFFFFFFFFFF3F3A
:10EEA800FFFFFFFFFFFFFFFFFFFFFFFFFFFFFFFF6A
:10EEB800FFFFFFFFFFFFFFFFFFFFFFFFFF0000FF58
:10EEC8000300E03F00F80100FE0F00FC1F0000F8FF
:10EED800FC0700000000FF00000000FC0300000029
:10EEE800E03F00000000FEFFFFFFFFFFFFFFFFFF06
:10EEF800FFFFFFFFFFFFFFFFFFFFFFFFFFFFFF3FDA
:10EF0800FFFFFFFFFFFFFFFFFFFFFFFFFFFFFFFF09
:10EF1800FFFFFFFFFFFFFFFFFFFFFFFFFF0100FEF7
:10EF28000300E03F00F00300FC0F00FC0F0000F8B6
:10EF3800FF07000000007F00000000FC0300000045
:10EF4800E01F00000000FCFFFFFFFFFFFFFFFFFFC7
:10EF5800FFFFFFFFFFFFFFFFFFFFFFFFFFFFFF3F79
:10EF6800FFFFFFFFFFFFFFFFFFFFFFFFFFFFFFFFA9
:10EF7800FFFFFFFFFFFFFFFFFFFFFFFFFF0100FE97
:10EF88000700C03F00F00300FC0F00FC0F0000F07A
:10EF9800FF0700FC00007F0080FFFFFF01001F004B
:10EFA800E01F00F00F00FCFFFFFFFFFFFFFFFFFF68
:10EFB800FFFFFFFFFFFFFFFFFFFFFFFFFFFFFF3F19
:10EFC800FFFFFFFFFFFFFFFFFFFFFFFFFFFFFFFF49
:10EFD800FFFFFFFFFFFFFFFFFFFFFFFFFF0300FC37
:10EFE8000700807F00F00700F80F00FC0F0000F01A
:10EFF800FF0700FC00007F0080FFFFFF01800F007B
:10F00800F00F00F00700FCFFFFFFFFFFFFFFFFFF0F
:10F01800FFFFFFFFFFFFFFFFFFFFFFFFFFFFFF3FB8
:10F02800FFFFFFFFFFFFFFFFFFFFFFFFFFFFFFFFE8
:10F03800FFFFFFFFFFFFFFFFFFFFFFFFFF0300FCD6
:10F048000F00007F00F00F00F00F00FC0F0000F031
:10F05800FF0700FC00007F0080FFFFFF01800F001A
:10F06800F00F00F80300FEFFFFFFFFFFFFFFFFFFA9
:10F07800FFFFFFFFFFFFFFFFFFFFFFFFFFFFFF3F58
:10F08800FFFFFFFFFFFFFFFFFFFFFFFFFFFFFFFF88
:10F09800FFFFFFFFFFFFFFFFFFFFFFFFFF0700F876
:10F0A8000F00007E00E00F00F00F00FC0F0000E0F2
:10F0B800FF0700FC00807F00C0FFFFFF0080070003
:10F0C800F00700F80300FFFFFFFFFFFFFFFFFFFF50
:10F0D800FFFFFFFFFFFFFFFFFFFFFFFFFFFFFF3FF8
:10F0E800FFFFFFFFFFFFFFFFFFFFFFFFFFFFFFFF28
:10F0F800FFFFFFFFFFFFFFFFFFFFFFFDFF0700F818
:10F108001F00007C00E01F00E00F00FE070000E089
:10F11800FF0700FC00807F00C0FFFFFF00800700A2
:10F12800F80700FC0100FFFFFFFFFFFFFFFFFFFFE5
:10F13800FFFFFFFFFFFFFFFFFFFFFFFFFFFFFF3F97
:10F14800FFFFFFFFFFFFFFFFFFFFFFFFFFFFFFFFC7
:10F15800FFFFFFFFFFFFFFFFFFFFFFFFFF0F00F0B5
:10F168001F0000F800E03F00C00700FE070000C0D5
:10F17800FF0700FE00807F00C0FFFFFF00C0070000
:10F18800F80700FC0180FFFFFFFFFFFFFFFFFFFF05
:10F19800FFFFFFFFFFFFFFFFFFFFFFFFFFFFFF3F37
:10F1A800FFFFFFFFFFFFFFFFFFFFFFFFFFFFFFFF67
:10F1B800FFFFFFFFFFFFFFFFFFFFFFFFFF0F00F055
:10F1C8001F0000F000C03F00C00700FE070000C09D
:10F1D800FF0700FE00803F00C0FFFFFF00C00700E0
:10F1E800F80300FC0080FFFFFFFFFFFFFFFFFFFFAA
:10F1F800FFFFFFFFFFFFFFFFFFFFFFFFFFFFFF3FD7
:10F20800FFFFFFFFFFFFFFFFFFFFFFFFFFFFFFFF06
:10F21800FFFFFFFFFFFFFFFFFFFFFFFFFF1F00F0E4
:10F228003F0000E000C07F00800700FE078003C0A9
:10F23800FF0700FE00803F00C0FFFF7F00E00300E3
:10F24800FC0300FEFFFFFFFFFFFFFFFFFFFFFFFFC5
:10F25800FFFFFFFFFFFFFFFFFFFFFFFFFFFFFF3F76
:10F26800FFFFFFFFFFFFFFFFFFFFFFFFFFFFFFFFA6
:10F27800FFFFFFFFFFFFFFFFFFFFFFFFFF1F00E094
:10F288003F0000C001C07F00800700FE07800380A8
:10F29800FF0700FE00803F00C0FFFF7F00E0030083
:10F2A800FC0300FEFFFFFFFFFFFFFFFFFFFFFFFF65
:10F2B800FFFFFFFFFFFFFFFFFFFFFFFFFFFFFF3F16
:10F2C800FFFFFFFFFFFFFFFFFFFFFFFFFFFFFFFF46
:10F2D800FFFFFFFFFFFFFFFFFFFFFFFFFF3F00C034
:10F2E8007F0000C00180FF00000700FE038003804C
:10F2F800CF0700FE00803F000000FE7F00000000F6
:10F30800FE010000E0FFFFFFFFFFFFFFFFFFFFFF21
:10F31800FFFFFFFFFFFFFFFFFFFFFFFFFFFFFF3FB5
:10F32800FFFFFFFFFFFFFFFFFFFFFFFFFFFFFFFFE5
:10F33800FFFFFFFFFFFFFFFFFFFFFFFFFF7F00C093
:10F348007F0000800180FF01000600FF03800300AA
:10F35800CF0700FE00803F000000FE3F00000000D5
:10F36800FE030000C0FFFFFFFFFFFFFFFFFFFFFFDF
:10F37800FFFFFFFFFFFFFFFFFFFFFFFFFFFFFF3F55
:10F38800FFFFFFFFFFFFFFFFFFFFFFFFFFFFFFFF85
:10F39800FFFFFFFFFFFFFFFFFFFFFFFFFF7F008073
:10F3A800FF0000000300FF01000600FF03C0070084
:10F3B800FF0700FE00803F000000FE3F00000080C5
:10F3C800FF03000000FFFFFFFFFFFFFFFFFFFFFF3E
:10F3D800FFFFFFFFFFFFFFFFFFFFFFFFFFFFFF3FF5
:10F3E800FFFFFFFFFFFFFFFFFFFFFFFFFFFFFFFF25
:10F3F800FFFFFFFFFFFFFFFFFFFFFFFFFFFF008093
:10F40800FB0000000200FF03000400FF03C0070028
:10F41800FF0700FE00803F000000FE3F000000E004
:10F42800FF03000000FFFFFFFFFFFFFFFFFFFFFFDD
:10F43800FFFFFFFFFFFFFFFFFFFFFFFFFFFFFF3F94
:10F44800FFFFFFFFFFFFFFFFFFFFFFFFFFFFFFFFC4
:10F45800FFFFFFFFFFFFFFFFF3FFFFFFFFFF0000BE
:10F46800FF0100000000FF07000000FF01C00700C7
:10F47800FE0700FE00801F000000FF3F000000F8AC
:10F48800FF07000000FEFFFFFFFFFFFFFFFFFFFF7A
:10F49800FFFFFFFFFFFFFFFFFFFFFFFFFFFFFF3F34
:10F4A800FFFFFFFFFFFFFFFFFFFFFFFFFFFFFFFF64
:10F4B800FFFFFFFFFFFFFFFFFFFFFFFFFFFF010051
:10F4C800FF0100000000FF07000000FF01C00F005F
:10F4D800FE07007E00C01F000000FF1F000000FCA8
:10F4E800FF07000000FEFFFFFFFFFFFFFFFFFFFF1A
:10F4F800FFFFFFFFFFFFFFFFFFFFFFFFFFFFFF3FD4
:10F50800FFFFFFFFFFFFFFFFFFFFFFFFFFFFFFFF03
:10F51800FFFFFFFFFFFFFFFFFFFFFFFFFFFF0100F0
:10F52800FF0380000000FE0F000000FF01C00F0075
:10F53800FC07007E00C01F000000FF1F000000F84D
:10F54800FF0F000000FEFFFFFFFFFFFFFFFFFFFFB1
:10F55800FFFFFFFFFFFFFFFFFFFFFFFFFFFFFF3F73
:10F56800FFFFFFFFFFFFFFFFFFFFFFFFFFFFFFFFA3
:10F57800FFFFFFFFFFFFFFFFFFFFFFFFFFFF03008E
:10F58800FE0380000000FE1F000000FF01C00F0006
:10F59800FC07007E00C01F000000FF1F000000F0F5
:10F5A800FF0F000000FCFFFFFFFFFFFFFFFFFFFF53
:10F5B800FFFFFFFFFFFFFFFFFFFFFFFFFFFFFF3F13
:10F5C800FFFFFFFFFFFFFFFFFFFFFFFFFFFFFFFF43
:10F5D800FFFFFFFFFFFFFFFFFFFFFFFFFFFF03002E
:10F5E800FC0300010000FE1F000080FF01C01F0097
:10F5F800FC07007E00C01F000000FF0F000000E0B5
:10F60800FF0F000000FEFFFFFFFFFFFFFFFFFFFFF0
:10F61800FFFFFFFFFFFFFFFFFFFFFFFFFFFFFF3FB2
:10F62800FFFFFFFFFFFFFFFFFFFFFFFFFFFFFFFFE2
:10F63800FFFFFFFFFFFFFFFFFFFFFFFFFFFF0700C9
:10F64800FC0700030000FE3F000080FF00000800E8
:10F65800FC07007E00C01F00F0FFFF0F003C00C049
:10F66800FFFFFF0300FEFFFFFFFFFFFFFFFFFFFF9E
:10F67800FFFFFFFFFFFFFFFFFFFFFFFFFFFFFF3F52
:10F68800FFFFFFFFFFFFFFFFFFFFFFFFFFFFFFFF82
:10F69800FFFFFFFFFFFFFFFFFFFFFFFFFFFF070069
:10F6A800FC0700070000FC3F000080FF000000008E
:10F6B800F807007E00C01F00F8FFFF0F003E00C0E3
:10F6C800FFFFFF0300FFFFFFFFFFFFFFFFFFFFFF3D
:10F6D800FFFFFFFFFFFFFFFFFFFFFFFFFFFFFF3FF2
:10F6E800FFFFFFFFFFFFFFFFFFFFFFFFFFFFFFFF22
:10F6F800FFFFFFFFFFFFFFFFFFFFFFFFFFFF0F0001
:10F70800F80F000E0000FC7F000080FF00000000E2
:10F71800F807007E00C00F00F8FFFF07003E00E07A
:10F728001F00F80100FFFFFFFFFFFFFFFFFFFFFFC4
:10F73800FFFFFFFFFFFFFFFFFFFFFFFFFFFFFF3F91
:10F74800FFFFFFFFFFFFFFFFFFFFFFFFFFFFFFFFC1
:10F75800FFFFFFFFFFFFFFFFFFFFFFFFFFFF0F00A0
:10F76800F80F001E0000F8FF000080FF00000000F6
:10F77800F007007E00C00F00F8FFFF07003E00E022
:10F788001F00F80180FFFFCFFFFFFFFFFFFFFFFF14
:10F79800FFFFFFFFFFFFFFFFFFFFFFFFFFFFFF3F31
:10F7A800FFFFFFFFFFFFFFFFFFFFFFFFFFFFFFFF61
:10F7B800FFFFFFFFFFFFFFFFFFFFFFFFFFFF1F0030
:10F7C800F00F003C0000F8FF000080FF0000000080
:10F7D800F007007E00C00F00F8FFFF07001E00F0D2
:10F7E8000F00F80080FFFFFFFFFFFFFFFFFFFFFF95
:10F7F800FFFFFFFFFFFFFFFFFFFFFFFFFFFFFF3FD1
:10F80800FFFFFFFFFFFFFFFFFFFFFFFFFFFFFFFF00
:10F81800FFFFFFFFFFFFFFFFFFFFFFFFFFFF1F00CF
:10F82800F01F007C0000F8FF0100807F000000004E
:10F83800F007007E00C00F00F8FFFF07001F00F070
:10F848000F00FC00C0FFFFFFFFFFFFFFFFFFFFFFF0
:10F85800FFFFFFFFFFFFFFFFFFFFFFFFFFFFFF3F70
:10F86800FFFFFFFFFFFFFFFFFFFFFFFFFFFFFFFFA0
:10F87800FFFFFFFFFFFFFFFFFFFFFFFFFFFF3F004F
:10F88800E03F00F80000F0FF0300C07F0000000028
:10F89800E007007E00C00F00F8FFFF03001F00F024
:10F8A8000F007C00C0FFFFFFFFFFFFFFFFFFFFFF10
:10F8B800FFFFFFFFFFFFFFFFFFFFFFFFFFFFFF3F10
:10F8C800FFFFFFFFFFFFFFFFFFFFFFFFFFFFFFFF40
:10F8D800FFFFFFFFFFFFFFFFFFFFFFFFFFFF3F00EF
:10F8E800E03F00F80100F0FF0300C07F00F07F0058
:10F8F800E007007E00E00F00FCFFFF03000F00F8A8
:10F9080007003E00E0FFFFFFFFFFFFFFFFFFFFFFD5
:10F91800FFFFFFFFFFFFFFFFFFFFFFFFFFFFFF3FAF
:10F92800FFFFFFFFFFFFFFFFFFFFFFFFFFFFFFFFDF
:10F93800FFFFFFFFFFFFFFFFFFFFFFFFFFFF7F004E
:10F94800C07F00F80300F0FF0700C07F00F0FF0051
:10F95800C007007E00E00F00FCFFFF03800F00F8E7
:10F9680006003E00E0FFFFFFFFFFFFFFFFFFFFFF76
:10F97800FFFFFFFFFFFFFFFFFFFFFFFFFFFFFF3F4F
:10F98800FFFFFFFFFFFFFFFFFFFFFFFFFFFFFFFF7F
:10F99800FFFFFFFFFFFFFFFFFFFFFFFFFFFF7F00EE
:10F9A800C07F00F00700E0FF0F00C07F00F0FF00FD
:10F9B800C007000000E00F000000F801800F00F809
:10F9C80007000000F0FFFFFFFFFFFFFFFFFFFFFF43
:10F9D800FFFFFFFFFFFFFFFFFFFFFFFFFFFFFF3FEF
:10F9E800FFFFFFFFFFFFFFFFFFFFFFFFFFFFFFFF1F
:10F9F800FFFFFFFFFFFFFFFFFFFFFFFFFFFFFF000E
:10FA0800807F00F00F00E0FF0F00C03F00F0FF0014
:10FA1800C007000000E00F000000F801C00700FC6C
:10FA280007000000F8FFFFFFFFFFFFFFFFFFFFFFDA
:10FA3800FFFFFFFFFFFFFFFFFFFFFFFFFFFFFF3F8E
:10FA4800FFFFFFFFFFFFFFFFFFFFFFFFFFFFFFFFBE
:10FA5800FFFFFFFFFFFFFFFFFFFFFFFFFFFFFF00AD
:10FA680080FF00E01F00E0FF1F00C03F00F0FF0123
:10FA78008007000000F007000000FC01C00700FC40
:10FA88000F000000FEFFFFFFFFDFFFFFFFFFFFFF8C
:10FA9800FFFFFFFFFFFFFFFFFFFFFFFFFFFFFF3F2E
:10FAA800FFFFFFFFFFFFFFFFFFFFFFFFFFFFFFFF5E
:10FAB800FFFFFFFFFFFFFFFFFFFFFFFFFFFFFF014C
:10FAC80000FF00E03F00E0FF3F00C03F00F0FF0103
:10FAD8008007000000FC07000000FC01C00700FCD4
:10FAE8000F000000FFFFFFFFFFFFFFFFFFFFFFFF0B
:10FAF800FFFFFFFFFFFFFFFFFFFFFFFFFFFFFF3FCE
:10FB0800FFFFFFFFFFFFFFFFFFFFFFFFFFFFFFFFFD
:10FB1800FFFFFFFFFFFFFFFFFFFFFFFFFFFFFF01EB
:10FB280000FF01C03F00C0FF3F00E03F00F8FF01B9
:10FB38008007000000FE07000000FC00C00300FE74
:10FB48001F0000C0FFFFFFFFFFFFFFFFFFFFFFFFDA
:10FB5800FFFFFFFFFFFFFFFFFFFFFFFFFFFFFF3F6D
:10FB6800FFFFFFFFFFFFFFFFFFFFFFFFFFFFFFFF9D
:10FB7800FFFFFFFFFFFFFFFFFFFFFFFFFFFFFF0389
:10FB880000FE01C0FF00C0FF7F00E03F00F8FF015A
:10FB98000007000080FF07000000FC00E00300FEF3
:10FBA8001F0000E0FFFFFFFFFFFFFFFFFFFFFFFF5A
:10FBB800FFFFFFFFFFFFFFFFFFFFFFFFFFFFFF3F0D
:10FBC800FFFFFFFFFFFFFFFFFFFFFFFFFFFFFFFF3D
:10FBD800FFFFFFFFFFFFFFFFFFFFFFFFFFFFFF0329
:10FBE80000FE03C0FF00C0FF7F00E01F00F8FF0316
:10FBF80000070000C0FF07000000FC00E00300FF52
:10FC08003F0000F8FFFFFFFFFFFFFFFFFFFFFFFFC1
:10FC1800FFFFFFFFFFFFFFFFFFFFFFFFFFFFFF3FAC
:10FC2800FFFFFFFFFFFFFFFFFFFFFFFFFFFFFFFFDC
:10FC3800FFFFFFFFFFFFFFFFFFFFFFFFFFFFFF07C4
:10FC480000FC0380FF0180FFFF00E01F00F8FF03B6
:10FC580000070000E0FF07000000FE00F00100FFC1
:10FC68003F0000FCFFFFFFFFFFFFFFFFFFFFFFFF5D
:10FC7800FFFFFFFFFFFFFFFFFFFFFFFFFFFFFF3F4C
:10FC8800FFFFFFFFFFFFFFFFFFFFFFFFFFFFFFFF7C
:10FC9800FFFFFFFFFFFFFFFFFFFFFFFFFFFFFF0764
:10FCA80000FC0780FF0380FFFF01E01F00F8FF074B
:10FCB80000060000F8FF07000000FE00F00180FFCA
:10FCC8007F0000FFFFFFFFFFFFFFFFFFFFFFFFFFBA
:10FCD800FFFFFFFFFFFFFFFFFFFFFFFFFFFFFF3FEC
:10FCE800FFFFFFFFFFFFFFFFFFFFFFFFFFFFFFFF1C
:10FCF800FFFFFFFFFFFFFFFFFFFFFFFFFFFFFFFF0C
:10FD0800FFFFFFFFFFFFFFFFFFFFFFFFFFFFFFFFFB
:10FD1800FFFFFFFFFFFFFFFFFFFFFFFFFFFFFFFFEB
:10FD2800FFFFFFFFFFFFFFFFFFFFFFFFFFFFFFFFDB
:10FD3800FFFFFFFFFFFFFFFFFFFFFFFFFFFFFF3F8B
:10FD4800FFFFFFFFFFFFFFFFFFFFFFFFFFFFFFFFBB
:10FD5800FFFFFFFFFFFFFFFFFFFFFFFFFFFFFFFFAB
:10FD6800FFFFFFFFFFFFFFFFFFFFFFFFFFFFFFFF9B
:10FD7800FFFFFFFFFFFFFFFFFFFFFFFFFFFFFFFF8B
:10FD8800FFFFFFFFFFFFFFFFFFFFFFFFFFFFFFFF7B
:10FD9800FFFFFFFFFFFFFFFFFFFFFFFFFFFFFF3F2B
:10FDA800FFFFFFFFFFFFFFFFFFFFFFFFFFFFFFFF5B
:10FDB800FFFFFFFFFFFFFFFFFFFFFFFFFFFFFFFF4B
:10FDC800FFFFFFFFFFFFFFFFFFFFFFFFFFFFFFFF3B
:10FDD800FFFFFFFFFFFFFFFFFFFFFFFFFFFFFFFF2B
:10FDE800FFFFFFFFFFFFFFFFFFFFFFFFFFFFFFFF1B
:10FDF800FFFFFFFFFFFFFFFFFFFFFFFFFFFFFF3FCB
:10FE0800FFFFFFFFFFFFFFFFFFFFFFFFFFFFFFFFFA
:10FE1800FFFFFFFFFFFFFFFFFFFFFFBFFFFFFFFF2A
:10FE2800FFFFFFFFFFFFFFFFFFFFFFFFFFFFFBFFDE
:10FE3800FFFFFFFFFFFFFFFFFFFFFFFFFFFFFFFFCA
:10FE4800FFFFFFFFFFFFFFFFFFFFFFFFFFFFFFFFBA
:10FE5800FFFFFFFFFFFFFFFFFFFFFFFFFFFFFF3F6A
:10FE6800FFFFFFFFFFFFFFFFFFFFFFFFFFFFFFFF9A
:10FE7800FFFFFFFFFFFFFFFFFFFFFFFFFFFFFFFF8A
:10FE8800FFFFFFFFFFFFDFFFFFFFFFFFFFFFFFFF9A
:10FE9800FFFFFFFFFFFFFFFFFFFFFFFFFFFFFFFF6A
:10FEA800FFFFFFFFFFFFFFFFFFFFFFFFFFFFFFFF5A
:10FEB800FFFFFFFFFFFFFFFFFFFFFFFFFFFFFF3F0A
:10FEC800FFFFFFFFFFFFFFFFFFFFFFFFFFFFFFFF3A
:10FED800FFFFFFFFFFFFFFFFFFFFE7FFFFFFFFFF42
:10FEE800FFFFFFFFFFFFDFFFFFFFFFFFFFFFFFFF3A
:10FEF800FFFFFFFFFFFFFFFFFFFFFFFFFFFFFFFF0A
:10FF0800FFFFFFFFFFFFFFFFFFFFFFFFFFFFFFFFF9
:10FF1800FFFFFFFFFFFFFFFFFFFFFFFFFFFFFF3FA9
:10FF2800FFFFFFFFFFFFFFFFFFFFFFFFFFFFFFFFD9
:10FF3800FFFFFFFFFFFFFFFFFFFFFFFFFFFFFFFFC9
:10FF4800FFFFFFFFFFFFFFFFFFFFFFFFFFFFFFFFB9
:10FF5800FFFFFFF9FFFFFFFFFFFFFFFFFFFFFFFFAF
:10FF6800FFFFFFFFFFFFFFFFFFFFFFFFFFFFFFFF99
:10FF7800FFFFFFFFFFFFFFFFFFFFFFFFFFFFFF3F49
:10FF8800FFFFFFFFFFFFFFFFFFFFFFFFFFFFFFFF79
:10FF9800FFFFFFFFFFFFFFFFFFFFFFFFFFFFFFFF69
:10FFA800FFFFFFFFFFFFFFFFFFFFFF7FFEFFFFFFDA
:10FFB800FFFFFFF9FFFFFFFFFFFFFFFFFFFFFFFF4F
:10FFC800FFFFFFFFFFFFFFFFFFFFFFFFFFFFFFFF39
:10FFD800FFFFFFFFFFFFFFFFFFFFFFFFFFFFFF3FE9
:10FFE800FFFFFFFFFFFFFFFFFFFFFFFFFFFFFFFF19
:08FFF800FFFFFFFFFFFFFFFF09
:020000041001E9
:10000000FFFFFFFFFFFFFFFFFFFFFFFFFFFFFFFF00
:10001000FFFFFFFFFFFFFFFFFFFFFFFFFFFFFFFFF0
:10002000FFFCFFFFFFFFFFFFFFFFFFFFFFFF1FFFC3
:10003000FFFFFFFFFFFFFFFFFFFFFFFFFFFFFFFFD0
:10004000FFFFFFFFFFFFFF3FFFFFFFFFFFFFFFFF80
:10005000FFFFFFFFFFFFFFFFFFFFFFFFFFFFFFFFB0
:10006000FFFFFFFFFFFFFFFFFFFFFFFFFFFFFFFFA0
:10007000FFFFFFFFFFFFFFFFFFFFFFFFFFFFFFFF90
:10008000FFFFFFFFFFFFFFFFFFFFFFFFFFFF01FC81
:10009000FFFFFFFFFFFFFFFFFFFFFFFFFFFFFFFF70
:1000A000FFFFFFFFFFFFFF3FFFFFFFFFFFFFFFFF20
:1000B000FFFFFFFFFFFFFFFFFFFFFFFFFFFFFFFF50
:1000C000FFFFFFFFFFFFFFFFFFFFFFFFFFFFFFFF40
:1000D000FFFFFFFFFFFFFFFFFFFFFFFFFFFFFFFF30
:1000E000FFFFFFFFFFFFFFFFFFFFFFFFFF0F00FC12
:1000F000FFFFFFFFFFFFFFFFFFFFFFFFFFFFFFFF10
:10010000FFFFFFFFFFFFFF3FFFFFFFFFFFFFFFFFBF
:10011000FFFFFFFFFFFFFFFFFFFFFFFFFFFFFFFFEF
:10012000FFFFFFFFFFFFFFFFFFFFFFFFFFE7FFFFF7
:10013000FFFFFFFFFFFFFFFFFFFFFFFFFFFFFFFFCF
:10014000FFFFFFFFFFFFFFFFFFFFFFFFFF0100F8C3
:10015000FFFFFFFFFFFFFFFFFFFFFFFFFFFFFFFFAF
:10016000FFFFFFFFFFFFFF3FFFFFFFFFFFFFFFFF5F
:10017000FFFFFFFFFFFFFFFFFFFFFFFFFFFFFFFF8F
:10018000FFFFFFFFFFFFFFFFFFFFFFFFFFFFFFFF7F
:10019000FFFFFFFFFFFF7FFFFFFFFFFFBFFFFFFF2F
:1001A000FFFFFFFFFFFFFFFFFFFEFFFF0F0000F855
:1001B000FFFFFFFFFFFFFFFFFFFFFFFFFFFFFFFF4F
:1001C000FFFFFFFFFFFFFF3FFFFFFFFFFFFFFFFFFF
:1001D000FFFFFFFFFFFFFFFFFFFFFFFFFFFFFFFF2F
:1001E000FFFFFFFFFFFFFFFFFFFFFFFFFFFFFFFF1F
:1001F000FFFFFFFFFFFF7FFFFFFFFFFFFFFFFFFF8F
:10020000F7FFFFFFFFFFFFFFFFFFFFFF03000030CF
:10021000FCFFFFFFFFFFFFFFFFFFFFFFFFFFFFFFF1
:10022000FFFFFFFFFFFFFF3FFFFFFFFFFFFFFFFF9E
:10023000FFFFFFFFFFFFFFFFFFFFFFFFFFFFFFFFCE
:10024000FFFFFFFFFFFFFFFFFFFFFFFFFFFFFFFFBE
:10025000FFEFFFFFFFFFFFFFFFFFFFFFFFFFFFF3CA
:10026000F7FFFFFFFFFFFFFFFFFFFFFF01000000A1
:10027000FCFFFFFFFFFFFFFFFFFFFFFFFFFFFFFF91
:10028000FFFFFFFFFFFFFF3FFFFFFFFFFFFFFFFF3E
:10029000FFFFFFFFFFFFFFFFFFFFFFFFFFFFFFFF6E
:1002A000FFFFFFFFFFFFFFFFFFFFFFFFFFFFFFFF5E
:1002B000FFFFFFFFFFFFFFFFFFFF7FFEFFFFFFFFCF
:1002C000FFFFFFFFFFFFFFFFFFFFFFFF0100000039
:1002D000F8FFFFFFFFFFFFFFFFFFFFFFFFFFFFFF35
:1002E000FFFFFFFFFFFFFF3FFFFFFFFFFFFFFFFFDE
:1002F000FFFFFFFFFFFFFFFFFFFFFFFFFFFFFFFF0E
:10030000FFFFFFFFFFFFFFFFFFFFFFFFFFFFFFFFFD
:10031000FFFDFFFFFFFFFFFFFFFF7FFEFFFFFFFF70
:10032000FFFFFFFFFFFFFFFFFFFFFFFF01000000D8
:10033000F0FFFFFFFFFFFFFFFFFFFFFFFFFFFFFFDC
:10034000FFFFFFFFFFFFFF3FFFFFFFFFFFFFFFFF7D
:10035000FFFFFFFFFFFFFFFFFFFFFFFFFFFFFFFFAD
:10036000FFFFFFFFFFFFFFFFFFFFFFFFFFFFFFFF9D
:10037000FFFDFFFFFFFFCFFFFFFFFFFFFFFFFFFFBF
:10038000FFFFFFFFFFFFFFFFFFFFFFFF0100000078
:1003900070FEFFFFFFFFFFFFFFFFFFFFFFFFFFFFFD
:1003A000FFFFFFFFFFFFFF3FFFFFFFFFFFFFFFFF1D
:1003B000FFFFFFFFFFFFFFFFFFFFFFFFFFFFFFFF4D
:1003C000FFFFFFFFFFFFFFFFFFFFFFFFFFFFFFFF3D
:1003D000FFFFFFFFFFFFCFFFFFFFFFFFFFFFFFFF5D
:1003E000FFFFFFFFFFFFFFFFFFFFFFFF0100000018
:1003F00000F8FFFFFFFFFFFFFFFFFFFFFFFFFFFF13
:10040000FFFFFFFFFFFFFF3FFFFFFFFFFFFFFFFFBC
:10041000FFFFFFFFFFFFFFFFFFFFFFFFFFFFFFFFEC
:10042000FFFFFFFFFFFFFFFFFFFFFFFFFFFFFFFFDC
:10043000FFFFFFFFFFFFFFFFFFFFFFFFFFFFFFFFCC
:10044000FFFFFFFFFFFFFFFFFFFFFFFF01000000B7
:1004500000F8FFFFFFFFFFFFFFFFFFFFFFFFFFFFB2
:10046000FFFFFFFFFFFFFF3FFFFFFFFFFFFFFFFF5C
:10047000FFFFFFFFFFFFFFFFFFFFFFFFFFFFFFFF8C
:10048000FFFFFFFFFFFFFFFFFFFFFFFFFFFFFFFF7C
:10049000FFFFFFFFFFFFFFFFFFFFFFFFFFFFFFFF6C
:1004A000FFFFFFFFFFFFFFFFFFFFFFFF0100000057
:1004B00000F8FFFFFFFFFFFFFFFFFFFFFFFFFFFF52
:1004C000FFFFFFFFFFFFFF3FFFFFFFFFFFFFFFFFFC
:1004D000FFFFFFFFFFFFFFFFFFFFFFFFFFFFFFFF2C
:1004E000FFFFFFFFFFFFFFFFFFFFFFFFFFFFFFFF1C
:1004F0007FFEFFFFFFFFFFF7FFFFFFFFFFFFFFFF95
:10050000FFFFFFFFFFFFFFFFFFFFFFFF01000000F6
:100510000070FEFFFFFFFFFFFFFFFFFFFFFFFFFF7A
:10052000FFFFFFFFFFFFFF3FFFFFFFFFFFFFFFFF9B
:10053000FFFFFFFFFFFFFFFFFFFFFFFFFFFFFFFFCB
:10054000FFFFFFFFFFFFFFFFFFFFEFFFFFFFFFFFCB
:10055000FFFFFFFFFFFFFFFFFFFFFFFFFFFFFFFFAB
:10056000FFFFFFFFFFFFFFFFFFFFFF3F0000000057
:100570000010F8FFFFFFFFFFFFFFFFFFFFFFFFFF80
:10058000FFFFFFFFFFFFFF3FFFFFFFFFFFFFFFFF3B
:10059000FFFFFFFFFFFFFFFFFFFFFFFFFFFFFFFF6B
:1005A000FFFFFFFFFFCFFFFFFFFFE1FFFFFFFFFFA9
:1005B000FFFFFFFFFFFFFFFFFFFFFFFFFFFFFFFF4B
:1005C000FFFFFFFFFFFFFFFFFFFFFF07000000002F
:1005D0000000F8FFFFFFFFFFFFFFFFFFFFFFFFFF30
:1005E000FFFFFFFFFFFFFF3FFFFFFFFFFFFFFFFFDB
:1005F000FFFFFFFFFFFFFFFFFFFFFFFFFFFFFFFF0B
:10060000FFFFFFFFFFCFFFFFFF3FE0FBFFFFFFFF0D
:10061000FFFFFFFFFFFFFFFFFFFFFFFFFFFFFFFFEA
:10062000FFFFFFFFFFFFFFFFFFFFFF0700000000CE
:100630000000F0FFFFFFFFFFFFFFFFFFFFFFFFFFD7
:10064000FFFFFFFFFFFFFF3FFFFFFFFFFFFFFFFF7A
:10065000FFFFFFFFFFFFFFFFFFFFFFFFFFFFFFFFAA
:10066000FFFFFFFFFFFFFFFFFF0760F0FFFFFFFF40
:10067000FFFFFFFFFFFFFFFFFBFFFFFFFFFFFFFF8E
:10068000FFFCFFFFFFFFFFFFFFFFFF070000000071
:10069000000070FCFFFFFFFFFFFFFFFFFFFFFFFFFA
:1006A000FFFFFFFFFFFFFF3FFFFFFFFFFFFFFFFF1A
:1006B000FFFFFFFFFFFFFFFFFFFFFFFFFFFFFFFF4A
:1006C000FFFFFFFFFFFFFFFFFF0100F0FFFFFFFF46
:1006D000FFFFFFFFFFFFFFFFFBFFFFFFFFFFFFFF2E
:1006E000FFFFFFFFFFFFFFFFFFFFFF0F0000000006
:1006F000000000F8FFFFFFFFFFFFFFFFFFFFFFFF0E
:10070000FFFFFFFFFFFFFF3FFFFFFFFFFFFFFFFFB9
:10071000FFFFFFFFFFFFFFFFFFFFFFFFFFFFFFFFE9
:10072000FFFFFFFFFFFFFFFFFF0000F0FFFFFFFFE6
:10073000FFFFFFFFFFFFFFFFFFFFFFFFFFFFFFFFC9
:10074000FFFFFFFFFFFFFFFFFFFFFF0F00000000A5
:10075000000000F8FFFFFFFFFFFFFFFFFFFFFFFFAD
:10076000FFFFFFFFFFFFFF3FFFFFFFFFFFFFFFFF59
:10077000FFFFFFFFFFFFFFFFFFFFFFFFFFFFFFFF89
:10078000FFFFFFFFFFFFFFFBFF0000F0FFFFFFFF8A
:10079000FFFFFFFFFFFFFFFFFFFFFFFFFFFFFFFF69
:1007A000FFFFFFFFFFFFFFFFFFFFFF0F0000000045
:1007B0003C0000F0FFFFFFFFFFFFFFFFFFFFFFFF19
:1007C000FFFFFFFFFFFFFF3FFFFFFFFFFFFFFFFFF9
:1007D000FFFFFFFFFFFFFFFFFFFFFFFFFFFFFFFF29
:1007E000FFFFFFFFFFFFFFFFFF0000F0FFFFFFFF26
:1007F000FFFFFFFFFFFFFFFFFFFFFFFFFFFFFFFF09
:10080000FFFFFFFFFFFFFFFFFFFFFF0F00000000E4
:100810003E0000F0FFFFFFFFFFFFFFFFFFFFFFFFB6
:10082000FFFFFFFFFFFFFF3FFFFFFFFFFFFFFFFF98
:10083000FFFFFFFFFFFFFFFFFFFFFFFFFFFFFFFFC8
:10084000FFFFFFFFFFFFFFFFFF0000F0FFFFFFFFC5
:10085000FFFFFFFFFFFFFFFFFFFFFFDFFFFFFFFFC8
:10086000FFFFFFFFFFFFFFFFFFFFFF0F0000000084
:100870007C0000F0FFFFFFFFFFFFFFFFFFFFFFFF18
:10088000FFFFFFFFFFFFFF3FFFFFFFFFFFFFFFFF38
:10089000FFFFFFFFFFFFFFFFFFFFFFFFFFFFFFFF68
:1008A000FFFFFFFFFFFFFFFFFF0000F0FFFFFFFF65
:1008B000FFFFFFFFFFFFFFFFFFFFFFDFFFFFFFFF68
:1008C000FFFFFFFFFFFFFFFFFFFFFF010000000032
:1008D0007C0000F0FFFFFFFFFFFFFFFFFFFFFFFFB8
:1008E000FFFFFFFFFFFFFF3FFFFFFFFFFFFFFFFFD8
:1008F000FFFFFFFFFFFFFFFFFFFFFFFFFFFFFFFF08
:10090000FFE7FFFFFFFFFFFF7F0000F0FFFFFFFF9C
:10091000FFFFFFFFFFFFFFFFFFFFFFFFFFFFFFFFE7
:10092000FFFFFFFFFFFFFFFFFFFF1F000000C001F1
:10093000080000F0FFFFFFFFFFFFFFFFFFFFFFFFCB
:10094000FFFFFFFFFFFFFF3FFFFFFFFFFFFFFFFF77
:10095000FFFFFFFFFFFFFFFFFFFFFFFFFFFFFFFFA7
:10096000FFFFFFFFFFFFFFFF7F0000F0F9FFFFFF2A
:10097000FFFFFFFFFFFFFFFFFFFFFFFFFFFFFFFF87
:10098000FFFFFFFFFFFFFFFFFFFF1F000000FC0155
:10099000000000F0FFFFFFFFFFFFFFFFFFFFFFFF73
:1009A000FFFFFFFFFFFFFF3FFFFFFFFFFFFFFFFF17
:1009B000FFFFFFFFFFFFFFFFFFFFFFFFFFFFFFFF47
:1009C000FFFFFFFFFFFFFFFF7F000000F8FFFFFFBB
:1009D000FFFFFFFFFFFFFFFFFFFFFFFFFFFFFFFF27
:1009E000FFFFFFFFFFFFFFFFFFFF1F000000FC03F3
:1009F000000000FEFFFFFFFFFFFFFFFFFFFFFFFF05
:100A0000FFFFFFFFFFFFFF3FFFFFFFFFFFFFFFFFB6
:100A1000FFFFFFFFFFFFFFFFFFFFFFFFFFFFFFFFE6
:100A2000FFFFFFFFFFFFFFFF7F000000F8FFFFFF5A
:100A3000FFFFBFCFFFFFFFFFFFFFFFFFFFFFFFFF36
:100A4000FFFFFFFFFFFFFFFFFFFF0F000000FC03A2
:100A5000000000FEFFFFFFFFFFFFFFFFFFFFFFFFA4
:100A6000FFFFFFFFFFFFFF3FFFFFFFFFFFFFFFFF56
:100A7000FFFFFFFFFFFFFFFFFFFFFFFFFFFFFFFF86
:100A8000FFFFFFFFFFFFFFFF7F000000F8FFFFFFFA
:100A9000FFFFBFFFFFFFFFFFFFFFFFFFFFFFFFFFA6
:100AA000FFFFFFFFFFFFFFFFFFFF1F000000F80336
:100AB000000000FEFFFFFFFFFFFFFFFFFFFFFFFF44
:100AC000FFFFFFFFFFFFFF3FFFFFFFFFFFFFFFFFF6
:100AD000FFFFFFFFFFFFFFFFFFFFFFFFFFFFFFFF26
:100AE000FFFFFFFFFFFFFFFF7F000000F8FFFFFF9A
:100AF000FFFFFFFFFFFFFFFFFFFFFFFFFFFFFFFF06
:100B0000FFFFFFFFFFFFFFFFFFFF1F008000180038
:100B1000000000FEFFFFFFFFFFFFFFFFFFFFFFFFE3
:100B2000FFFFFFFFFFFFFF3FFFFFFFFFFFFFFFFF95
:100B3000FFFFFFFFFFFFFFFFFFFFFFFFFFFFFFFFC5
:100B4000FFFFFFFFFFFFFFFF7F000000F8FFFFFF39
:100B5000FFFFFFFFFFFFFFFFFFFFFFFFFFFFFFFFA5
:100B6000FFFFFFFFFFFFFFFFFFFF3F00E000000070
:100B7000000000FCFFFFFFFFFFFFFFFFFFFFFFFF85
:100B8000FFFFFFFFFFFFFF3FFFFFFFFFFFFFFFFF35
:100B9000FFFFFFFFFFFFFFFFFFFFFFFFFFFFFFFF65
:100BA000FFFFFFFFFFFFFFFF7F000000F0FFFFFFE1
:100BB000FFFFFFFFFFFFFFFFFFFFFFFFFFFFFFFF45
:100BC000FFFFFFFFFFFFFFFFFFFF3F00FC000000F4
:100BD000000000FCFFFFFFFFFFFFFFFFFFFFFFFF25
:100BE000FFFFFFFFFFFFFF3FFFFFFFFFFFFFFFFFD5
:100BF000FFFFFFFFFFFFFFFFFFFFFFFFFFFFFFFF05
:100C0000FFFFFFFFFFFFFFFF7F000000F0FFFFFF80
:100C1000FFFFFFFFFFFFFFFFFFFFFFFFFFFFFFFFE4
:100C2000FFFFFFFFFFFFFFFFFFFF1F00FC000000B3
:100C3000000000FCFFFFFFFFFFFFFFFFFFFFFFFFC4
:100C4000FFFFFFFFFFFFFF3FFFFFFFFFFFFFFFFF74
:100C5000FFFFFFFFFFFFFFFFFFFFFFFFFFFFFFFFA4
:100C6000FFFFFFFFFFFFFFFF7F000000F0FFFFFF20
:100C7000FFFFFFFFFFFFFFFFFFFFFFFFFFFFFFFF84
:100C8000FFFFFFFFFFF9FFFFFFFF0300F801000078
:100C9000000000FCFFFFFFFFFFFFFFFFFFFFFFFF64
:100CA000FFFFFFFFFFFFFF3FFFFFFFFFFFFFFFFF14
:100CB000FFFFFFFFFFFFFFFFFFFFFFFFFFFFFFFF44
:100CC000FFFFFFFFFFFFFFFF7F000000F0FFFFFFC0
:100CD000FFFFFFFFFFFF0FF8001FF0FFFFFFFFFF09
:100CE000FFFFFFFFFFFFFFFFFFFF00007800000096
:100CF000000080FFFFFFFFFFFFFFFFFFFFFFFFFF81
:100D0000FFFFFFFFFFFFFF3FFFFFFFFFFFFFFFFFB3
:100D1000FFFFFFFFFFFFFFFFFFFFFFFFFFFFFFFFE3
:100D2000FFFFFFFFFFFFFFFF3F000000F0FFFFFF9F
:100D3000FFFFFFFFFFFF0FF8001FF0FFFFFFFFFFA8
:100D4000FFFFFFFFFFFFFFFFFF3F0000100000005D
:100D50001C00C0FFFFFFFFFFFFFFFFFFFFFFFFFFC4
:100D6000FFFFFFFFFFFFFF3FFFFFFFFFFFFFFFFF53
:100D7000FFFFFFFFFFFFFFFFFFFFFFFFFFFFFFFF83
:100D8000FFFFFFFFFFFFFFFF3F000000F0FFFFFF3F
:100D9000FFFFFFFFFFFF0FF8001FF0FFFFFFFFFF48
:100DA000DFFFFFFFFFFFFFFFFF3F0000000000002D
:100DB0001F00E0FFFFFFFFFFFFFFFFFFFFFFFFFF41
:100DC000FFFFFFFFFFFFFF3FFFFFFFFFFFFFFFFFF3
:100DD000FFFFFFFFFFFFFFFFFFFFFFFFFFFFFFFF23
:100DE000FFFFFFFFFFFFFFFF3F000000F8FFFFFFD7
:100DF000FFFFFFFFFFFF0FF8001FF0FFFFFFFFFFE8
:100E0000FFFFFFFFFFFFFFFFFF3F000000000000AC
:100E10003F00C0FFFFFFFFFFFFFFFFFFFFFFFFFFE0
:100E2000FFFFFFFFFFFFFF3FFFFFFFFFFFFFFFFF92
:100E3000FFFFFFFFFFFFFFFFFFFFFFFFFFFFFFFFC2
:100E4000FFFFFFFFFFFFFFFF3F000000FCFFFFFF72
:100E5000FFFFFFFFFFFF0770000EF0FFFFFFFFFF28
:100E6000FFFFFFFFFFFFFFFFFF3F0000000000004C
:100E70003E00C0FFFFFFFFFFFFFFFFFFFFFFFFFF81
:100E8000FFFFFFFFFFFFFF3FFFFFFFFFFFFFFFFF32
:100E9000FFFFFFFFFFFFFFFFFFFFFFFFFFFFFFFF62
:100EA000FFFFFFFFFFFFFFFF3F000080FFFFFFFF8F
:100EB000FFFFFFFFFFFF03200000F0FFFFFFFFFF2A
:100EC000FFFFFFFFFFFFFFFFFF7F000000000000AC
:100ED0007E1C80FFFFFFFFFFFFFFFFFFFFFFFFFF05
:100EE000FFFFFFFFFFFFFF3FFFFFFFFFFFFFFFFFD2
:100EF000FFFFFFFFFFFFFFFFFFFFFFFFFFFFFFFF02
:100F0000FFFFFFFFFFFFFFFF3F0000E0FFFFFFFFCE
:100F1000FFFFFFFFFF3F00000000F0FFFFFFFFFFAC
:100F2000FFFFFFFFFFFFFFFFFF7F0000000000004B
:100F30007E3E80FFFFFFFFFFFFFFFFFFFFFFFFFF82
:100F4000FFFFFFFFFFFFFF3FFFFFFFFFFFFFFFFF71
:100F5000FFFFFFFFFFFFFFFFFFFFFFFFFFFFFFFFA1
:100F6000FFFFFFFFFFFFFFFF3F0000E0FFFFFFFF6E
:100F7000FFFFFFFFFF3F00000000F0FFFFFFFFFF4C
:100F8000FFFFFFFFFFFFFFFFFF7F000000000C00DF
:100F9000FE3F00FFFFFFFFFFFFFFFFFFFFFFFFFF21
:100FA000FFFFFFFFFFFFFF3FFFFFFFFFFFFFFFFF11
:100FB000FFFFFFFFFFFFFFFFFFFFFFFFFFFFFFFF41
:100FC000FFFFFFFFFFFFFFFF3F0000E0FFFFFFFF0E
:100FD000FFFFFFFFFF3F80001000FFFFFFFFFFFF4D
:100FE000FFFFFFFFFFFFFFFFFF7F000000001F006C
:100FF000FE7F80FFFFFFFFFFFFFFFFFFFFFFFFFF01
:10100000FFFFFFFFFFFFFF3FFFFFFFFFFFFFFFFFB0
:10101000FFFFFFFFFFFFFFFFFFFFFFFFFFFFFFFFE0
:10102000FFFFFFFFFFFFFFFF3F0000E0FFFFFFFFAD
:10103000FFFFFFFFFF3FC0013880FFFFFFFFFFFF03
:10104000FFFFFFFFFFFFFFFFFF1F000000801F00EB
:10105000FE7FF0FFFFFFFFFFFFFFFFFFFFFFFFFF30
:10106000FFFFFFFFFFFFFF3FFFFFFFFFFFFFFFFF50
:10107000FFFFFFFFFFFFFFFFFFFFFFFFFFFFFFFF80
:10108000FFFFFFFFFFFBFFFF3F0000E0FFFFFFFF51
:10109000FFFFFFFFFF3FE0037CC0FFFFFFFFFFFFFD
:1010A000FFFFFFFFFFFFFFFFFF07000000801F8023
:1010B000FFFFFDFFFFFFFFFFFFFFFFFFFFFFFFFF42
:1010C000FFFFFFFFFFFFFF3FFFFFFFFFFFFFFFFFF0
:1010D000FFFFFFFFFFFFFFFFFFFFFFFFFFFFFFFF20
:1010E000FFFFFFFFFFFBFFFF3F0000E0FFFFFFFFF1
:1010F000FFFFFFFFFF3FE0037CC0F7FFFFFFFFFFA5
:10110000FFFFFFFFFFFFFFFFFF00000000003FF0B9
:10111000FFFFFFFFFFFFFFFFFFFFFFFFFFFFFFFFDF
:10112000FFFFFFFFFFFFFF3FFFFFFFFFFFFFFFFF8F
:10113000FFFFFFFFFFFFFFFFFFFFFFFFFFFFFFFFBF
:10114000FFFFFBFFFFFFFFFF3F0000E0FFFFFFFF90
:10115000FFFFFFFFFF3FE0037CC0F3FFFFFFFFFF48
:10116000FFFFFFFFFFFFFFFF7F00000000003FFCCD
:10117000FFFFFFFFFFFFFFFFFFFFFFFFFFFFFFFF7F
:10118000FFFFFFFFFFFFFF3FFFFFFFFFFFFFFFFF2F
:10119000FFFFFFFFFFFFFFFFFFFFFFFFFFFFFFFF5F
:1011A000FFFFFFFFFFFFFFFF1F0000E0FFFFFFFF4C
:1011B000FFFFFFFFFF3FE0037CC0FFFFFFFFFFFFDC
:1011C000FFFFFFFFFFFFFFFF3F0000000000FFFFEA
:1011D000FFFFFFFFFFFFFFFFFFFFFFFFFFFFFFFF1F
:1011E000FFFFFFFFFFFFFF3FFFFFFFFFFFFFFFFFCF
:1011F000FFFFFFFFFFFFFFFFFFFFFFFFFFFFFFFFFF
:10120000FFFFFFFFFFFFFFFF1F0000E0FFFFFFFFEB
:10121000FFFFFFFFFFFFFFFFFFFFFFFFFFFFFFFFDE
:10122000FFFFFFFFFFFFFFFF7F0000000000FFFF49
:10123000FFFFFFFFFFFFFFFFFFFFFFFFFFFFFFFFBE
:10124000FFFFFFFFFFFFFF3FFFFFFFFFFFFFFFFF6E
:10125000FFFFFFFFFFFFFFFFFFFFFFFFFFFFFFFF9E
:10126000FFFFFFFFFFFFFFFF1F0000E0FFFFFFFF8B
:10127000FFFFFFFFFFFFFFFFFFFFFFFFFFDFFFFF9E
:10128000FFFFFFFFFFFFFFFF7F0000000000FFFFE9
:10129000FFFFFFFFFFFFFFFFFFFFFFFFFFFFFFFF5E
:1012A000FFFFFFFFFFFFFF3FFFFFFFFFFFFFFFFF0E
:1012B000FFFFFFFFFFFFFFFFFFFFFFFFFFFFFFFF3E
:1012C000FFFFFFFFFFFFFFFF1F0000E0FFFFFFFF2B
:1012D000FFFFFFFFFFFFFFFFFFFFFFFFFFDFFFFF3E
:1012E000FFFFFFFFFFFFFFFFFF0000000000FFFF09
:1012F000FFFFFFFFFFFFFFFFFFFFFFFFFFFFFFFFFE
:10130000FFFFFFFFFFFFFF3FFFFFFFFFFFFFFFFFAD
:10131000FFFFFFFFFFFFFFFFFFFFFFFFFFFFFFFFDD
:10132000FFFFFFFFFFFFFFFF1F0000E0FFFFFFFFCA
:10133000FFFFFFFFFFFFFFFFFFFFFFFFFFFFFFFFBD
:10134000FFFFFFFFFFFFFFFFFF0000000080FFFF28
:10135000FFFFFFFFFFFFFFFFFFFFFFFFFFFFFFFF9D
:10136000FFFFFFFFFFFFFF3FFFFFFFFFFFFFFFFF4D
:10137000FFFFFFFFFFFFFFFFFFFFFFFFFFFFFFFF7D
:10138000FFFFFFFFFFFFFFFF1F0000E0FFFFFFFF6A
:10139000FFFFFFFFFFFFFFFFFFFFFFFFFFFFFFFF5D
:1013A000FFFFFFFFFFFFFFFFFF00000000F0FFFF58
:1013B000FFFFFFFFFFFFFFFFFFFFFFFFFFFFFFFF3D
:1013C000FFFFFFFFFFFFFF3FFFFFFFFFFFFFFFFFED
:1013D000FFFFFFFFFFFFFFFFFFFFFFFFFFFFFFFF1D
:1013E000FFFFFFFFFFFFFFFF1F0000E0FFFFFFFF0A
:1013F000FFFFFFFFFFFFFFFFFFFFFFFFFFFFFFFFFD
:10140000FFFFFFFFFFFFFFFFFF01000000FCFFFFEA
:10141000FFFFFFFFFFFFFFFFFFFFFFFFFFFFFFFFDC
:10142000FFFFFFFFFFFFFF3FFFFFFFFFFFFFFFFF8C
:10143000FFFFFFFFFFFFFFFFFFFFFFFFFFFFFFFFBC
:10144000FFFFFFFFFFFFFFFF1F0000F0FFFFFFFF99
:10145000FFFFFFFFFFFFFFFFFFFFFFFFFFFFFFFF9C
:10146000FFFFFFBFFFFFFFFFFF01060000FFFFFFC1
:10147000FFFFFFFFFFFFFFFFFFFFFFFFFFFFFFFF7C
:10148000FFFFFFFFFFFFFF3FFFFFFFFFFFFFFFFF2C
:10149000FFFFFFFFFFFFFFFFFFFFFFFFFFFFFFFF5C
:1014A000FFFFFFFFFFFFFFFF1F0000FEFFFFFFFF2B
:1014B000FFFFFFFFFFFFFFFFFFFFFFFFFFFFFFFF3C
:1014C000FFFFFFBFFFFFFFFFFFC1070000FEFFFFA1
:1014D000FFFFFFFFFFFFFFFFFFFFFFFFFFFFFFFF1C
:1014E000FFFFFFFFFFFFFF3FFFFFFFFFFFFFFFFFCC
:1014F000FFFFFFFFFFFFFFFFFFFFFFFFFFFFFFFFFC
:10150000FFFF7FFFFFFFFFFF1F00E0FFFFFFFFFF69
:10151000FFFFFFFFFFFFFFFFFFFFFFFFFDFFFFFFDD
:10152000FFFFFFFFFFFFFFFFFFF90F0000FEFFFFC0
:10153000FFFFFFFFFFFFFFFFFFFFFFFFFFFFFFFFBB
:10154000FFFFFFFFFFFFFF3FFFFFFFFFFFFFFFFF6B
:10155000FFFFFFFFFFFFFFFFFFFFFFFFFFFFFFFF9B
:10156000FFFF7FFFFFFFFFFF1F00E0FFFFFFFFFF09
:10157000FFFFFFFFFFFFFFFFFFFFFFFFF9FFFFFF81
:10158000FFFFFFFFFFFFFFFFFFFF0F0000FCFFFF5C
:10159000FFFFFFFFFFFFFFFFFFFFFFFFFFFFFFFF5B
:1015A000FFFFFFFFFFFFFF3FFFFFFFFFFFFFFFFF0B
:1015B000FFFFFFFFFFFFFFFFFFFFFFFFFFFFFFFF3B
:1015C000FFFFFFFFFFFFFFFF1F00E0FFFFFFFFFF29
:1015D000FFFFFFFFFFFFFFFFFFFFFFFFFFFFFFFF1B
:1015E000FFFFFFFFFFFFFFFFFFFF0F0000FCFFFFFC
:1015F000FFFFFFFFFFFFFFFFFFFFFFFFFFFFFFFFFB
:10160000FFFFFFFFFFFFFF3FFFFFFFFFFFFFFFFFAA
:10161000FFFFFFFFFFFFFFFFFFFFFFFFFFFFFFFFDA
:10162000FFFFFFFFFFFFFFFF1F00E0FFFFFFFFFFC8
:10163000FFFFEFFFFFFFFFFFFFFFFFFFFFFFFFFFCA
:10164000FFFFFFFFFFFFFFFFFFFF1F0000F8FFFF8F
:10165000FFFFFFFFFFFFFFFFFFFFFFFFFFFFFFFF9A
:10166000FFFFFFFFFFFFFF3FFFFFFFFFFFFFFFFF4A
:10167000FFFFFFFFFFFFFFFFFFFFFFFFFFFFFFFF7A
:10168000FFFFFFFFFFFFFFFF0F00E0FFFFFFFFFF78
:10169000FFFFFFFFFFFFFFFFFFFFFFFFFFFFFFFF5A
:1016A000FFFFFFFFFFFFFFFFCFFF1F3E00F8FFFF21
:1016B000FFFFFFFFFFFFFFFFFFFFFFFFFFFFFFFF3A
:1016C000FFFFFFFFFFFFFF3FFFFFFFFFFFFFFFFFEA
:1016D000FFFFFFFFFFFFFFFFFFFFFFFFFFFFFFFF1A
:1016E000FFFFFFFFFFFFFFFF0F00E0FFFFFFFFFF18
:1016F000FFFFFFFFFFFFFFFFFFFFFFFFFFFFFFFFFA
:10170000FFFFFFFFFFFFFFFFFFFFFF3F00F8FFFFAF
:10171000FFFFFFFFFFFFFFFFFFFFFFFFFFFFFFFFD9
:10172000FFFFFFFFFFFFFF3FFFFFFFFFFFFFFFFF89
:10173000FFFFFFFFFFFFFFFFFFFFFFFFFFFFFFFFB9
:10174000FFFFFFFFFFFFFFFF0F00E0FFFFFFFDFFB9
:10175000FFFFFFFFFFFFFFFFFFFFFFFFFFFFFFFF99
:10176000FFFFFFFFFFFFFFFFFFFFFF7F00F8FFFF0F
:10177000FFFFFFFFFFFFFFFFFFFFFFFFFFFFFFFF79
:10178000FFFFFFFFFFFFFF3FFFFFFFFFFFFFFFFF29
:10179000FFFFFFFFFFFFFFFFFFFFFFFFFFFFFFFF59
:1017A000FFFFFFFFFFFFFFFF0F00F0FFFFFFFDFF49
:1017B000FFFFFFFFFFFFFFFFFFFFFFFFFFFFFFFF39
:1017C000FFFFFFFFFFFFFFFFFFFFFF7F00FFFFFFA8
:1017D000FFE7FFFFFFFFFFFFFFFFFFFFFFFFFFFF31
:1017E000FFFFFFFFFFFFFF3FFFFFFFFFFFFFFFFFC9
:1017F000FFFFFFFFFFFFFFFFFFFFFFFFFFFFFFFFF9
:10180000FFFFFFFFFFFFFFFF0F00F8FFFFFFFFFFDE
:10181000FFFFFFFFFFFFFFFFFFFFFFFFFFFFFFFFD8
:10182000FFFFFFFFFFFFFFFFFFFFFFFFE1FFFFFFE6
:10183000FFFFFFFFFFFFFFFFFFFFFFFFFFFFFFFFB8
:10184000FFFFFFFFFFFFFF3FFFFFFFFFFFFFFFFF68
:10185000FFFFFFFFFFFFFFFFFFFFFFFFFFFFFFFF98
:10186000FFFFFFFFFFFFFFFF0FC0FFFFFFFFFFFFB7
:10187000FFFFFFFFFFFFFFFFFFF9FFFFFFFFFFFF7E
:10188000FFFFFFFFFFFFFFFFFFFFFFFFF9FFFFFF6E
:10189000FFFFFFFFFFFFFFFFFFFFFFFFFFFFFFFF58
:1018A000FFFFFFFFFFFFFF3FFFFFFFFFFFFFFFFF08
:1018B000FFFFFFFFFFFFFFFFFFFFFFFFFFFFFFFF38
:1018C000FFFFFFFFFFFFFFFF0FFFFFFFFFFFFFFF18
:1018D000FFFFFFFFFFFFFFFFFFFBFFFFFFFFFFFF1C
:1018E000FFFFFFFFFFFFFFFFFFFFFFFFFFFFFFFF08
:1018F000FFFFFFFFFFFFFFFFFFFFFFFFFFFFFFFFF8
:10190000FFFFFFFFFFFFFF3FFFFFFFFFFFFFFFFFA7
:10191000FFFFFFFFFFFFFFFFFFFFFFFFFFFFFFFFD7
:10192000FFFFFFEFFFFFFFFFFFFFFFFFFFFFFFFFD7
:10193000FFFFFFFFFFFFFFFFFFFFFFFFFFFFFFFFB7
:10194000FFFFFFFFFFFFFFFFFFFFFFFFFFFFFFFFA7
:10195000FFFFFFFFFFFFFFFFFFFFFFFFFFFFFFFF97
:10196000FFFFFFFFFFFFFF3FFFFFFFFFFFFFFFFF47
:10197000FFFFFFFFFFFFFFFFFFFFFFFFFFFFFFFF77
:10198000FFFFFFFFFFFFFFFFFFFFFFFFFFFFFFFF67
:10199000FFFFFFFFFFFFFFFFFFFFFFFFFFFFFFFF57
:1019A000FFFFFFFFFFFFFFFFFFFFFFFFFFFFFFFF47
:1019B000FFFFFFFFFFFFFFFFFFFFFFFFFFFFFFFF37
:1019C000FFFFFFFFFFFFFF3FFFFFFFFFFFFFFFFFE7
:1019D000FFFFFFFFFFFFFFFFFFFFFFFFFFFFFFFF17
:1019E000FFFFFFFFFFFFFFFFFFFFFFFFFFFFFFFF07
:1019F000FFFFFFFFFFFFFFFFFFFFFFFFFFFFFFFFF7
:101A0000FFFFFFFFFFFFFFFFFFFFFFFFFFFFFFFFE6
:101A1000FFFFFFFFFFFFFFFFFFFFFFFFFFFFFFFFD6
:101A2000FFFFFFFFFFFFFF3FFFFFFFFFFFFFFFFF86
:101A3000FFFFFFFFFFFFFFFFFFFFFFFFFFFFFFFFB6
:101A4000FFFFFFFFFFFFFFFFFFFFFFFFFFFFFFFFA6
:101A5000FFFFFFFFFFFFFFFFFFFFFFFFFFFFFFFF96
:101A6000FFFFFFFFFFFFFFFFFFFFFFFFFFFFFFFF86
:101A7000FFFFFFFFFFFFFFFFFFFFFFFFFFFFFFFF76
:101A8000FFFFFFFFFFFFFF3FFFFFFFFFFFFFFFFF26
:101A9000FFFFFFFFFFFFFFFFFFFFFFFFFFFFFFFF56
:101AA000FFFFFFFFFFFFFFFFFFFFFFFFFFFFFFFF46
:101AB000FFFFFFFFFFFFFFFFFFFFFFFFFFFFFFFF36
:101AC000FFFFFFFFFFFFFFFFFFFFFFFFFFFFFFFF26
:101AD000FFFFFFFFFFFFFFFFFFFFFFFFFFFFFFFF16
:101AE000FFFFFFFFFFFFFF3FFFFFFFFFFFFFFFFFC6
:101AF000FFFFFFFFFFFFFFFFFFFFFFFFFFFFFFFFF6
:101B0000FFFFFFFFFFFFFFFFFFFFFFFFFFFFFFFFE5
:101B1000FFFFFFFFFFFFFFFFFFFFFFFFFFFFFFFFD5
:101B2000FFFFFFFFFFFFFFFFFFFFFFFFFFFFFFFFC5
:101B3000FFFFFFFFFFFFFFFFFFFFFFFFFFFFFFFFB5
:101B4000FFFFFFFFFFFFFF3FFFFFFFFFFFFFFFFF65
:101B5000FFFFFFFFFFFFFFFFFFFFFFFFFFFFFFFF95
:101B6000FFFFFFFFFFFFFFFFFFFFFFFFFFFFFFFF85
:101B7000FFFFFFFFFFFFFFFFFFFFFFFFFFFFFFFF75
:101B8000FFFFFFFFFFFFFFFFFFFFFFFFFFFFFFFF65
:101B9000FFFFFFFFFFFFFFFFFFFFFFFFFFFFFFFF55
:101BA000FFFFFFFFFFFFFF3FFFFFFFFFFFFFFFFF05
:101BB000FFFFFFFFFFFFFFFFFFFFFFFFFFFFFFFF35
:101BC000FFFFFFFFFFFFFFFFFFFFFFFFFFFFFFFF25
:101BD000FFFFFFFFFFFFFFFFFFFFFFFFFFFFFFFF15
:101BE000FFFFFFFFFFFFFFFFFFFFFFFFFFFFFFFF05
:101BF000FFFFFFFFFFFFFFFFFFFFFFFFFFFFFFFFF5
